:100000000C94322A0C942C2D0C94572D0C94822D88
:100010000C94AD2D0C94D82D0C94032E0C942E2EF4
:100020000C94592E0C94632A0C94632A0C94632A22
:100030000C94632A0C94632A0C94632A0C94632A0C
:100040000C94632A0C944AA90C94632A0C94632A96
:100050000C94632A0C94632A0C94CB9C0C94652A10
:100060000C94632A0C94148B0C94C08B0C94632A0C
:100070000C94632A0C94632A0C94632A0C94632ACC
:100080000C94632A0C94632A0C94632A0C94632ABC
:100090000C94632A0C94632A0C94632A0C94632AAC
:1000A0000C94632A0C94632A0C94632A0C94632A9C
:1000B0000C94632A0C94632A0C94632A0C94632A8C
:1000C0000C94632A0C94632A0C94632A0C94632A7C
:1000D0000C94632A0C94632A0C94632A0C94632A6C
:1000E0000C94632AA22BA72BAC2BB62BC02B392C3C
:1000F000CA2BD22BDA2BE42BEE2BF82B072C112C4E
:10010000392C1B2C252C2F2C5D2C602C4F2C532C88
:10011000592C972C642C682C6E2C722C762C7C2CF1
:10012000802C842C972C8A2C8E2C922C335A195A82
:10013000165A1C5A1F5A225A2E5A255A3F5A285AC2
:100140002B5A478B4D8B5E8B698B718B868B758B96
:10015000868B798B7D8B868B838BA997A997B0979C
:10016000B097B097B797B797B797C497BE97BE9712
:10017000BE97084AD73B3BCE016E84BCBFFDC12F62
:100180003D6C74319ABD56833DDA3D00C77F11BE88
:10019000D9E4BB4C3E916BAAAABE000000803F058B
:1001A000A84CCDB2D44EB93836A9020C50B99186BC
:1001B00088083CA6AAAA2ABE000000803F000D9431
:1001C000A12C0D94A1270D94C80B4E414E494E49C8
:1001D0005459494E46CDCCCC3D0AD7233C17B7D114
:1001E0003877CC2B329595E6241FB14F0A000020BA
:1001F000410000C84200401C4620BCBE4CCA1B0E39
:100200005AAEC59D7400000A0B02090C0D0E0807BA
:1002100003040100000000000000000000000000D6
:1002200000000000000000000000000000000000CE
:10023000001211100000000000000000000000008B
:10024000000000000000000000000001021020205B
:10025000080810204010204080020102010804021A
:100260000101020408102040808040201008040290
:1002700001800402018040201008040201080402E9
:1002800001010204081020408001020408102040EF
:100290008005050505070508080808020202020A8C
:1002A0000A08080404040401010101010101010319
:1002B00003030303030303040707070C0C0C0C0CD4
:1002C0000C0C0C0202020206060606060606060BC7
:1002D0000B0B0B0B0B0B0B0000200023002600293F
:1002E000002C002F0032000001000003010601096C
:1002F0000100002200250028002B002E00310034D0
:100300000002010000050108010B0100002100248A
:100310000027002A002D00300033000101000004F6
:100320000107010A0101060D00FE09016602D6203F
:10033000FFFE0BFE0AFE0D0060221969808080809E
:100340008080800080183363A0A0A00357675050BE
:10035000F850F850500259692078A0A0702828F071
:100360002002596948A85010204050A890025868AF
:1003700040A0A040A0989068281363808080113B23
:100380006B2040408080808080404020113B6B800B
:100390004040202020202040408006556520A87045
:1003A000A8200455652020F8202011336360408088
:1003B000065161F811336340E040025969080810A2
:1003C00010204040808002596920508888888888A1
:1003D00050200259692060A02020202020F80259D6
:1003E000697088880810204080F8025969F8081060
:1003F000207008088870025969101030505090F829
:100400001010025969F88080B0C808088870025935
:100410006970888080F088888870025969F80810AF
:100420001020204040400259697088888870888870
:10043000887002596970888888780808887011382F
:100440006840E040000040E04011386840E0400073
:100450000060408002596908102040804020100848
:10046000045464F80000F802596980402010081014
:1004700020408002596970888808102020002002DE
:10048000596970888898A8A8B08078025969205066
:10049000888888F8888888025969F04848487048F0
:1004A0004848F00259697088808080808088700296
:1004B0005969F048484848484848F0025969F88066
:1004C0008080F0808080F8025969F8808080F08018
:1004D0008080800259697088808080988888700246
:1004E000596988888888F888888888123969E0403E
:1004F000404040404040E002596938101010101050
:10050000109060025969888890A0C0A090888802E5
:1005100059698080808080808080F802596988884D
:10052000D8A8A88888888802596988C8C8A8A898BF
:1005300098888802596970888888888888887002B5
:100540005969F0888888F080808080015A6A7088B4
:100550008888888888A87008025969F0888888F097
:10056000A090888802596970888080700808887017
:10057000025969F820202020202020200259698873
:10058000888888888888887002596988888888500F
:100590005050202002596988888888A8A8A8A850A7
:1005A00002596988885050205050888802596988BB
:1005B0008850502020202020025969F8081010206F
:1005C000404080F8113B6BE080808080808080809C
:1005D00080E0025969808040402010100808113BDB
:1005E0006BE0202020202020202020E008536320E2
:1005F0005088015161F82A226280400256667008D4
:1006000078889868025969808080F088888888F0A6
:1006100002566670888080887002596908080878D8
:1006200088888888780256667088F88088700259B1
:100630006930484040F04040404000586870888829
:100640008878088870025969808080B0C888888856
:10065000881238684000C040404040E0004A6A10BC
:1006600000301010101090906002596980808090C6
:10067000A0C0A09088123969C0404040404040402E
:10068000E0025666D0A8A8A8A888025666B0C88816
:10069000888888025666708888888870005868F054
:1006A000888888F0808080005868788888887808F2
:1006B0000808025666B0C88080808002566670883E
:1006C000601088700258684040F040404048300256
:1006D0005666888888889868025666888888505048
:1006E000200256668888A8A8A8500256668850201E
:1006F0002050880058688888889868088870025652
:1007000066F810204080F8015B6B1820202020C084
:10071000202020201822196980808080808080809D
:1007200080015B6BC0202020201820202020C008E2
:10073000536348A890FFFFFFFFFFFFFFFFFFFFFF8E
:10074000FFFFFFFFFFFFFFFFFFFFFFFFFFFFFFFFB9
:10075000FFFFFFFFFFFF0D0060221969800080800E
:1007600080808080800358682070A8A0A0A8702096
:1007700002596930484040E0404048B0035666881E
:10078000705050708802596988885050F820F820BD
:1007900020221969808080800080808080124A6ACF
:1007A000609080609090601090601A3262A0A00308
:1007B00059697088A8D8C8D8A88870045767700885
:1007C00078887800F80356662850A0A05028045373
:1007D00063F80808163161E00359697088E8D8D8D1
:1007E000E8D888700A5161F81744646090906003FB
:1007F00057672020F8202000F807356540A02040EA
:10080000E007356540A04020C02A226240800058A1
:10081000688888888898E8808002596978E8E8E8DC
:10082000E868282828262161C020226240800735F8
:100830006540C04040E0045767708888887000F8C1
:10084000035666A050282850A0025A6A40C0404073
:10085000E00818283808025A6A40C04040E01028D2
:10086000081038025A6A40A04020A04818283808CA
:10087000025969200020204080888870025A6A400E
:10088000200020508888F88888025A6A10200020AA
:10089000508888F88888025A6A3048002050888832
:1008A000F88888025A6A28500020508888F888887A
:1008B000025A6A50500020508888F88888025A6A84
:1008C00020502020508888F8888802596958A0A0B4
:1008D000A0B0E0A0A0B8005B6B70888080808080B2
:1008E00088702040025A6A402000F88080F08080A2
:1008F000F8025A6A102000F88080F08080F8025ACE
:100900006A304800F88080F08080F8025A6A5050BF
:1009100000F88080F08080F8123A6A804000E04061
:1009200040404040E0123A6A204000E040404040F1
:1009300040E0124A6A609000E04040404040E012CF
:100940003A6AA0A000E04040404040E0025969F00F
:10095000484848E8484848F0025A6A2850008888C1
:10096000C8A8988888025A6A4020007088888888B9
:100970008870025A6A1020007088888888887002FF
:100980005A6A30480070888888888870025A6A28B5
:10099000500070888888888870025A6A50500070A9
:1009A0008888888888700355658850205088015B46
:1009B0006B08709898A8A8A8C8C87080025A6A40A6
:1009C000200088888888888870025A6A10200088E9
:1009D000888888888870025A6A30480088888888A1
:1009E000888870025A6A5050008888888888887081
:1009F000025A6A102000888850202020200259695D
:100A000080F0888888F0808080025969609090A08A
:100A1000A0908888B00259694020007008788898B2
:100A2000680259691020007008788898680259692E
:100A3000304800700878889868025969285000701A
:100A4000087888986802596950500070087888982A
:100A500068025A6A304830007008788898680256F0
:100A600066702870A0A850005868708880808870D0
:100A700020400259694020007088F880887002592F
:100A8000691020007088F880887002596930480029
:100A90007088F88088700259695050007088F8801A
:100AA0008870123969804000C040404040E01239EF
:100AB00069204000C040404040E012496960900019
:100AC000C040404040E0123969A0A000C040404012
:100AD00040E0025A6A50206010708888888870024E
:100AE0005969285000B0C888888888025969402010
:100AF0000070888888887002596910200070888882
:100B00008888700259693048007088888888700227
:100B10005969285000708888888870025969505037
:100B200000708888888870035767202000F80020AC
:100B300020015868087098A8A8C8708002596940B8
:100B40002000888888889868025969102000888861
:100B50008888986802596930480088888888986829
:100B6000025969505000888888889868005B6B102B
:100B700020008888889868088870005A6A8080B049
:100B8000C88888C8B08080005B6B50500088888817
:100B9000986808887001050700FE0500FB01F22037
:100BA000FFFE05FE05FE0200400215258080800044
:100BB00080053242A0A002556550F850F850014619
:100BC000562070C030E02002556590102040480249
:100BD0005565608068906805122280800225354046
:100BE000808080400225358040404080043343A00F
:100BF00040A003334340E0400122324080043141B1
:100C0000E002112180025565081020408002455500
:100C10006090909060022535C040404040024555AC
:100C2000E0106080F0024555E0106010E00245558C
:100C30002060A0F020024555F080E010E00245550C
:100C40006080E09060024555F0102040400245551C
:100C500060906090600245556090701060031323AF
:100C6000800080021424800080800235452040806E
:100C70004020033343E000E00235458040204080BF
:100C8000024555E0106000400255657088B8A870B4
:100C9000024555609090F090024555E090E090E05C
:100CA0000235456080808060024555E0909090E07C
:100CB000023545E080E080E0023545E080E080805C
:100CC0000245557080B090700245559090F090901C
:100CD000023545E0404040E002455530101090603C
:100CE00002455590A0C0A09002354580808080E0EC
:100CF00002556588D8A8888802455590D0B0909054
:100D00000245556090909060024555E09090E080DB
:100D1000014656609090906010024555E09090E03A
:100D20009002455570806010E0023545E04040403B
:100D30004002455590909090600245559090A0A03B
:100D40004002556588A8A8A850024555909060902B
:100D5000900245559090701060023545E02040802B
:100D6000E0022535C0808080C0025565804020109B
:100D700008022535C0404040C005324240A0024133
:100D800051F0052232804002445470909070024528
:100D90005580E09090E002344460808060024555C8
:100DA000107090907002445460B0C06002354520CD
:100DB00040E04040004656709090701060024555EB
:100DC00080E0909090021525800080808000273779
:100DD000400040404040800245558090A0E0900295
:100DE00015258080808080025464F0A8A8A8024461
:100DF00054E090909002445460909060004656E019
:100E00009090E080800046567090907010100234F0
:100E100044A0C0808002445470C030E00235454098
:100E2000E0404020024454909090700244549090CE
:100E3000A040025464A8A85050023444A04040A0EE
:100E4000004656909090701060024454F02040F09C
:100E5000023545604080406002152580808080809A
:100E6000023545C0402040C005425250A0FFFFFF60
:100E7000FFFFFFFFFFFFFFFFFFFFFFFFFFFFFFFF82
:100E8000FFFFFFFFFFFFFFFFFFFFFFFFFFFF02006E
:100E900040FFFFFFFFFFFFFFFFFFFFFFFFFFFFFF21
:100EA000FFFFFFFFFFFFFFFFFFFFFFFFFFFFFFFF52
:100EB000FFFFFFFFFFFFFFFFFFFFFFFFFFFFFFFF42
:100EC000FFFFFFFFFFFFFFFFFFFFFFFFFFFFFFFF32
:100ED000FFFFFFFFFFFFFFFFFFFFFFFFFFFFFFFF22
:100EE000FFFFFFFFFFFFFFFFFFFFFFFFFFFFFFFF12
:100EF00001050800FF060121023520FFFF07FF065C
:100F0000FF090050221656808080800080153353E0
:100F1000A0A0A00257575050F850F8505002575711
:100F20002070A07028702013355580A040A02002AA
:100F3000475740A0A040A0A05025135380808012A6
:100F40002656408080808040122656804040404097
:100F5000800245559060F060900255552020F820A1
:100F600020113353604080044151F011335340E06D
:100F70004002465610102040808012365640A0A0F5
:100F8000A0A04012365640C0404040E002465660A5
:100F900090106080F0024656F0206010906002468B
:100FA000562060A0F02020024656F080E0109060AD
:100FB0000246566080E0909060024656F010202075
:100FC00040400246566090609090600246566090A5
:100FD00090701060122555C0C000C0C01136566018
:100FE00060006040801236562040808040200343DD
:100FF00053F000F0123656804020204080123656C2
:1010000040A020400040015858304898A8A890407F
:1010100030024656609090F09090024656E090E084
:101020009090E0024656609080809060024656E0C4
:1010300090909090E0024656F080E08080F002466A
:1010400056F080E0808080024656609080B09060CC
:101050000246569090F0909090123656E0404040F4
:1010600040E002465670202020A04002465690A044
:10107000C0A0A0900246568080808080F002465634
:1010800090F0F090909002465690D0F0B0B0900260
:101090004656609090909060024656E09090E080B6
:1010A00080014757609090D0B06010024656E090A3
:1010B00090E0909002465660904020906012365624
:1010C000E040404040400246569090909090600230
:1010D0004656909090906060024656909090F0F046
:1010E00090024656909060609090025656888850C4
:1010F000202020024656F010204080F0123656E0A4
:1011000080808080E0024656808040201010123699
:1011100056E020202020E016325240A0014151F03C
:1011200016225280400244547090907002465680BD
:1011300080E09090E0123454608080600246561047
:10114000107090907002445460B0C0600246562007
:101150005040E04040014555609070106002465696
:101160008080E09090901236564000C04040E011E0
:1011700037572000202020A040024656808090E073
:101180009090123656C040404040E0025454D0A8DF
:10119000A8A8024454E0909090024454609090605B
:1011A000014555E090E08080014555709070101029
:1011B000024454A0D0808012345460C020C0024643
:1011C000564040E0405020024454909090701234B9
:1011D00054A0A0A04002545488A8A850024454909F
:1011E0006060900145559090709060024454F020EA
:1011F00040F0024757304020C02040302216568031
:101200008080808080024757C02040304020C00648
:10121000425250A0FFFFFFFFFFFFFFFFFFFFFFFF56
:10122000FFFFFFFFFFFFFFFFFFFFFFFFFFFFFFFFCE
:10123000FFFFFFFFFF0900502216568000808080CC
:10124000800146562070A0A070200246562050E033
:101250004050A002555588705070880256568850EC
:10126000F820F82022175780808000808080024775
:10127000577080E0907010E0173151A00256567000
:10128000A8C8C8A87014355560A06000E003435397
:1012900050A050123353E02020143151E002565632
:1012A00070E8D8E8D870173151E015335340A040AA
:1012B00012355540E04000E014355540A02040E094
:1012C000143555C020C020C016225240800145551B
:1012D000909090E08002565678E8E868282824111B
:1012E0005180112252408014355540C04040E014D6
:1012F000355540A04000E0034353A050A00247579B
:10130000808080A060F0200247578080A0D010200D
:101310007002475780408060A0F02012365640008F
:101320004080A04002475740206090F090900247D4
:101330005720406090F0909002475760906090F086
:10134000909002475750A06090F0909002475790BD
:10135000006090F0909002475760906090F09090FD
:1013600002465670A0A0F0A0B00147576090808060
:101370009060400247574020F080E080F0024757DD
:101380002040F080E080F00247576090F080E080DD
:10139000F00247579000F080E080F012375780400D
:1013A000E0404040E01237572040E0404040E0122B
:1013B000375740A0E0404040E0123757A000E040DF
:1013C0004040E00256567048E8484870024757507F
:1013D000A090D0B0909002475740206090909060CD
:1013E000024757204060909090600247576090609D
:1013F0009090906002475750A06090909060024794
:101400005790006090909060123353A040A0024625
:101410005670B0B0D0D0E0024757402090909090E6
:10142000600247572040909090906002475760902C
:10143000909090906002475790009090909060023A
:1014400057571020885020202002465680E0909068
:10145000E0800246566090A0A090A002475740202E
:10146000007090907002475720400070909070027A
:1014700047572050007090907002475750A000705E
:1014800090907002465650007090907002475760DE
:10149000906070909070025454F068B07811355597
:1014A000608080604002475740200060B0C060020A
:1014B000475720400060B0C060024757609000600E
:1014C000B0C060024656500060B0C060123757800E
:1014D0004000C04040E0123757204000C04040E08C
:1014E00012375740A000C04040E0123656A000C05E
:1014F0004040E0024757A040A0107090600247575C
:1015000050A000E0909090024757402000609090DB
:1015100060024757204000609090600247576090FB
:10152000006090906002475750A000609090600269
:1015300046569000609090601235554000E00040A3
:1015400002445470B0D0E002475740200090909081
:10155000700247572040009090907002475760906B
:1015600000909090700246569000909090700148C4
:101570005820400090907090600147578080E09024
:10158000E08080014757900090907090602020206C
:1015900020002020202020200025753A253032759B
:1015A00000253032753A25303275002575642025C6
:1015B0003032753A25303275003FFFF03800703117
:1015C00086302387102787902F87D02F03D0203095
:1015D000102078102078102030102F03D02F87D0C3
:1015E0002787902387103186303800703FFFF03F07
:1015F000FFF038007030FC3020FC102078102030D4
:10160000102C00D02E31D02F7BD02F7BD02E31D07C
:101610002C00D020301020781020FC1030FC303806
:1016200000703FFFF0041040020820020820041060
:101630004008208010410010410008208004104024
:101640000000001FFFF81FFFF81FFFF81FFFF81F23
:10165000E02010201020101020102020102010302A
:10166000300840048003001FE03FF03FF03FF01FD0
:10167000E01FE03FF03FF03FF00FC0078003004560
:1016800072723A207574663820666F6E74206E6FC1
:101690007420696E697469616C697A65642E0045AD
:1016A00072723A207574663820666F6E74206E6FA1
:1016B0007420696E697469616C697A65642E00458D
:1016C00072723A207574663820666F6E74206E6F81
:1016D0007420696E697469616C697A65642E005062
:1016E0006C65617365207265736574005052494E74
:1016F0005445522048414C544544007F80FFC0FF70
:10170000C0FFC07F807F80FFC0FFC0FFC03F001EC2
:10171000000C00FFFFFF0E000E000E000E000E007A
:101720000E000E000E007FC03F801F000E00040060
:1017300004000E001F003F807FC00E000E000E0050
:101740000E000E000E000E000E0000FE0003FF80D3
:101750000783C00E01C00E00E01C00E07F00E03EE9
:1017600000E01C00E00800E00000E00001C00E0105
:10177000C00F078007FF0001FC0003F8000FFE0008
:101780001E0F00380700380380700380700FE07070
:1017900007C0700380700100700000380000380737
:1017A000001E0F000FFE0003F80000060C00FE07ED
:1017B000022603BC017FFE08FE08FE05080806009D
:1017C0000040F0C88888987810050808060000C016
:1017D000F88888888888F80505050600012030F813
:1017E00030200508080600002070F820202020E0A6
:1017F0000509090600FF2070A8A8B8888870200590
:101800000606060001E08CEA8C8A0A050909060032
:10181000FFF8A88888888888A8F8050A0A0600FEC4
:10182000205050505088A8A8887003030306000376
:1018300040A040FFFFFFFFFFFFFFFFFFFFFFFFFF95
:10184000FFFFFFFFFFFFFFFFFF0000000605FF0196
:101850000707060200808080808000800303030663
:101860000105A0A0A005060606000050F85050F89B
:10187000500509090600FF2070A8A07028A8702054
:10188000050707060000C8C81020409898050707FC
:1018900006000040A0A040A89068010303060205CE
:1018A0008080800309090601FF204040808080403D
:1018B00040200309090601FF8040402020204040CD
:1018C0008005070706000020A8702070A8200505E5
:1018D000050600012020F820200203030601FFC0B6
:1018E0004080050101060003F8020202060100C063
:1018F000C0050707060000081010204040800507BB
:1019000007060000708898A8C888700307070601BA
:101910000040C040404040E00507070600007088D6
:1019200008102040F8050707060000F808103008E6
:10193000887005070706000010305090F810100559
:101940000707060000F880F00808887005070706FA
:101950000000304080F0888870050707060000F816
:1019600008101020202005070706000070888870E6
:10197000888870050707060000708888780810605E
:10198000020505060100C0C000C0C002060606012F
:10199000FFC0C000C0408003050506010120408053
:1019A0004020050303060002F800F80305050601C0
:1019B0000180402040800507070600007088102045
:1019C0002000200507070600007088B8A8B88070BE
:1019D000050707060000708888F8888888050707CB
:1019E000060000F04848704848F005070706000068
:1019F00070888080808870050707060000F04848DE
:101A0000484848F0050707060000F88080F080800D
:101A1000F8050707060000F88080F0808080050741
:101A20000706000070888080988870050707060008
:101A300000888888F8888888030707060100E04046
:101A400040404040E0050707060000381010101025
:101A500090600507070600008890A0C0A090880548
:101A60000707060000808080808080F80507070651
:101A7000000088D8A888888888050707060000889D
:101A800088C8A89888880507070600007088888895
:101A9000888870050707060000F08888F08080803D
:101AA00005070706000070888888A8906805070762
:101AB000060000F08888F0A090880507070600005F
:101AC00070888070088870050707060000F82020DD
:101AD000202020200507070600008888888888883D
:101AE0007005070706000088888888505020050781
:101AF0000706000088888888A8A850050707060000
:101B000000888850205088880507070600008888CC
:101B10005020202020050707060000F8081020406C
:101B200080F80309090601FFE080808080808080C2
:101B3000E005070706000080404020101008030958
:101B4000090601FFE020202020202020E0050303DB
:101B50000600052050880501010600FEF803030376
:101B600006010580402005050506000070087888FC
:101B7000780507070600008080F0888888F0050552
:101B800005060000708080887005070706000008C1
:101B90000878888888780505050600007088F08038
:101BA00070050707060000304840E0404040050748
:101BB000070600FE70888888780870050707060009
:101BC000008080F0888888880307070601004000AD
:101BD000C0404040E00409090601FE10003010102A
:101BE0001010906005070706000080808890E09044
:101BF00088030707060100C04040404040E005055B
:101C000005060000D0A8A8A8A8050505060000B094
:101C1000C8888888050505060000708888887005D2
:101C200007070600FEF0888888F080800507070611
:101C300000FE78888888780808050505060000B049
:101C4000C880808005050506000078807008F005D2
:101C500007070600002020F82020201805050506AB
:101C6000000088888898680505050600008888882F
:101C700050200505050600008888A8A85005050520
:101C800006000088502050880507070600FE888857
:101C90008850204080050505060000F8102040F817
:101CA0000309090601FF20404040804040402001D8
:101CB00009090602FF80808080808080808003097F
:101CC000090601FF8040404020404040800503035A
:101CD00006000248A890FF1FFFFFFFFFFFFF600004
:101CE00000000001FF400000000000FF8000000035
:101CF00000007F83CF00000C303F87FF80000C3056
:101D00001F867980000C000F8C30C7838C30E78CE5
:101D100030CFC7CC31F38C30DCECEC33B98C30D81D
:101D20006C6C33198C30D06C0C33198C30D86C0C33
:101D300033198C30DC6C0E3B198C30CF7C079F192B
:101D40008C30C77C038F1940000000000002600047
:101D500000000000061FFFFFFFFFFFF8000000006B
:101D60000000000000000000000000000000000073
:101D70000000000000000000000000000000000C57
:101D8000000000000000000C000000000000001235
:101D900000000000000000230000000000000021FF
:101DA000000000000000004C800000000000005E09
:101DB000800000000000009240000000000000A130
:101DC0004000000000000121200000000000027F10
:101DD000900000000000020010000000000007FF5B
:101DE000F8000000000004000800000000000800E7
:101DF00004000000000008000600000000001000C1
:101E0000020000000000301E010000000000207FE2
:101E100081000000000041FFE0800000000043FC62
:101E2000F08000000000873B7840000000018EDB5E
:101E3000FC60000000010FEBCC20000000021FED51
:101E4000B610000000021FDEB6100000000439CDFD
:101E50007F080000000436E0FF08000000087EC094
:101E6000BB84000000187F005D86000000107FC06A
:101E7000ED82000000203CC07301000000203B33D5
:101E80007F01000000701BE77E03800000C81DEE8C
:101E9000DE04C00000880FDEDC04400001240FDFF8
:101EA0003C092000012607DBF8192000027203E735
:101EB000F0139000025101FFE02290000489007F9E
:101EC000802448000904801E004824000BFE4000C6
:101ED00000DFF40010004000008002001FFFFFFF41
:101EE000FFFFFE00000000000000000000000000F6
:101EF0000000000000000000000000001022103C64
:101F00003C0E1F00102210042211040010221008A1
:101F100022110400102210083C110400102210109D
:101F20002211040010221020221104001E1C1E3C4D
:101F30003C0E040000000000000000000000000053
:101F40000000000000000000000000000000000091
:101F50000000000000000000000000000000000081
:101F60000000000000000000000000000000000071
:101F70000000000000000000000000000000000061
:101F80000000000000000000000000000000000051
:101F90000000000000000000000000060900FE062E
:101FA000018902FE20FFFE07FE06FE00000006007B
:101FB000070106060602008080808000800303037C
:101FC000060103A0A0A00507070600FF5050F85027
:101FD000F850500509090600FE2070A8A07028A836
:101FE00070200608080600FF40A848102048540842
:101FF0000507070600FF6090906098906801030352
:102000000602038080800207070602FF408080806E
:102010008080400207070602FF8040404040408029
:102020000505050600008850F850880505050600DE
:10203000002020F820200204040602FEC040408058
:10204000050101060002F8020202060200C0C004F7
:1020500006060601001010204080800406060601D6
:102060000060909090906003060606010040C0401A
:102070004040E00406060601006090102040F00495
:102080000606060100F020601010E00506060600B6
:102090000010305090F810040606060100F080E0B1
:1020A0001010E00406060601006080E090906004D5
:1020B0000606060100F01010204040040606060146
:1020C00000609060909060040606060100609090A9
:1020D000701060020505060200C0C000C0C0020703
:1020E000070602FEC0C000C040408005050506008E
:1020F000001860806018050303060001F800F80569
:102100000505060000C0300830C0040707060100BE
:10211000609010604000400506060600007090A820
:10212000B08070050606060000205088F8888805F3
:102130000606060000F088F08888F004060606010E
:1021400000609080809060040606060100E0909098
:102150009090E0040606060100F080E08080F00424
:102160000606060100F080E0808080040606060175
:1021700000609080B090600406060601009090F028
:10218000909090030606060100E040404040E005C4
:1021900006060600003810101090600406060601BE
:1021A0000090A0C0A09090040606060100808080E8
:1021B0008080F005060606000088D8A8A888880454
:1021C000060606010090D0B0909090050606060025
:1021D00000708888888870040606060100E09090E8
:1021E000E080800407070601FF609090D0B0601087
:1021F000040606060100E09090E0909004060606B2
:102200000100609040209060050606060000F8205E
:1022100020202020040606060100909090909060F7
:10222000040606060100909090F060600506060620
:1022300000008888A8A8D8880506060600008850EF
:10224000202050880506060600008888502020209F
:10225000040606060100F010204080F00306060682
:102260000100E080808080E0040606060100808096
:1022700040201010030606060100E020202020E088
:102280000503030600032050880501010600FEF83F
:102290000202020602048040040404060100709059
:1022A00090700406060601008080E09090E004042F
:1022B00004060100708080700406060601001010FC
:1022C0007090907004040406010060B0C0700406B1
:1022D00006060100205040E040400406060601FECC
:1022E0006090907010600406060601008080E09007
:1022F00090900306060601004000C04040E003083D
:10230000080601FE200060202020A04004060606EA
:1023100001008080A0C0A090030606060100C04016
:10232000404040E0050404060000D0A8A88804044A
:1023300004060100E09090900404040601006090FF
:1023400090600406060601FEE09090E0808004069E
:10235000060601FE7090907010100404040601003F
:10236000A0D0808004040406010070C030E00406A0
:10237000060601004040E04050200404040601002D
:102380009090907004040406010090906060050431
:102390000406000088A8A850040404060100906008
:1023A00060900406060601FE909090709060040410
:1023B00004060100F02040F003070706010020405A
:1023C00040804040200107070602FF808080808017
:1023D00080800307070601008040402040408004C1
:1023E000020206010350A0FFFFFFFFFFFFFFFFFFF8
:1023F000FFFFFFFFFFFFFFFFFFFFFFFFFFFFFFFFED
:10240000FFFFFFFFFFFFFFFF0000000600070106C0
:10241000060602008000808080800406060601FF18
:102420002070A0A070200507070600FF304840F08C
:102430004040F8050505060000A8508850A805068C
:10244000060600008850F820F8200107070602FF62
:10245000808080008080800407070601FF70806014
:10246000906010E0030101060105A00607070600C1
:1024700000788494A494847803050506010160A083
:102480006000E00505050600002850A05028040360
:1024900003060100F01010040101060102F0060716
:1024A000070600007884B4A4A4847804010106011E
:1024B00005F00403030601026090600507070600AB
:1024C000FF2020F8202000F803050506010140A0A8
:1024D0002040E0030505060101C0204020C00202A3
:1024E0000206020440800405050601FF9090B0D06A
:1024F0008005060606000078E8E868282801010142
:10250000060202800202020602FE40800305050662
:10251000010140C04040E003050506010140A04024
:1025200000E0050505060000A0502850A005080899
:102530000600FF40C04050703078100508080600C3
:10254000FF40C04050680810380508080600FFC06A
:10255000204030F0307810040707060100200020EA
:1025600060809060050707060000402020507088BA
:10257000880507070600001020205070888805078E
:1025800007060000205020507088880507070600C5
:10259000002850205070888805070706000050006A
:1025A00020507088880507070600002050205070D2
:1025B000888805060606000078A0F0A0A0B80408E8
:1025C000080601FE609080809060204004070706A6
:1025D00001004020F080E080F004070706010020A1
:1025E00040F080E080F00407070601002050F080F2
:1025F000E080F00407070601005000F080E080F062
:102600000307070601008040E0404040E003070761
:102610000601002040E0404040E0030707060100BB
:1026200040A0E0404040E0030707060100A000E0B2
:10263000404040E00506060600007048E848487043
:1026400004070706010050A090D0B090900407073F
:10265000060100402060909090600407070601008A
:1026600020406090909060040707060100205060B1
:102670009090906004070706010050A06090909031
:102680006004070706010050006090909060050507
:102690000506000088502050880408080601FF1035
:1026A00070B0B0D0D0E08004070706010040209051
:1026B0009090906004070706010020409090909051
:1026C0006004070706010020509090909060040776
:1026D00007060100500090909090600507070600E3
:1026E000001020885020202004060606010080E00B
:1026F0009090E0800406060601006090A0A090A0E3
:10270000040707060100402000709090700407073E
:102710000601002040007090907004070706010039
:102720002050007090907004070706010050A00030
:102730007090907004060606010050007090907032
:1027400004070706010020502070909070050404D3
:1027500006000070A8B0780406060601FE708080AE
:1027600070204004070706010040200060B0C070E0
:1027700004070706010020400060B0C0700407078E
:1027800006010020500060B0C0700406060601007B
:10279000500060B0C070030707060100804000C011
:1027A0004040E0030707060100204000C04040E031
:1027B00003070706010040A000C04040E0030606F2
:1027C000060100A000C04040E004070706010030F9
:1027D00060107090906004070706010050A000E0B0
:1027E00090909004070706010040200060909060E0
:1027F000040707060100204000609090600407076E
:102800000601002050006090906004070706010058
:1028100050A0006090906004060606010050006021
:102820009090600505050600002000F800200404D3
:102830000406010070B0D0E0040707060100402044
:1028400000909090700407070601002040009090CF
:1028500090700407070601002050009090907004CB
:1028600006060601005000909090700409090601C8
:10287000FE2040009090907090600408080601FED1
:102880008080E09090E080800408080601FE5000FF
:102890009090907090605072696E742066726F6D47
:1028A000205344005072696E742066726F6D20531D
:1028B0004400022E2E004D61696E0046696C616D08
:1028C000656E7400447269766520537472656E6734
:1028D00074680053746570732F6D6D004A65726B78
:1028E00000416363656C65726174696F6E00566563
:1028F0006C6F6369747900436F6E666967757261A6
:1029000074696F6E004573746570732F6D6D00454B
:1029100073746570732F6D6D005A73746570732FC7
:102920006D6D005A73746570732F6D6D00597374FB
:102930006570732F6D6D005973746570732F6D6DB5
:10294000005873746570732F6D6D005873746570E3
:10295000732F6D6D00416476616E6365642053650D
:102960007474696E67730056652D6A65726B0056E4
:10297000652D6A65726B00567A2D6A65726B00561A
:102980007A2D6A65726B0056792D6A65726B0056F6
:10299000792D6A65726B0056782D6A65726B0056E8
:1029A000782D6A65726B00416476616E63656420A0
:1029B00053657474696E677300416D6178204500DA
:1029C000416D6178204500416D6178205A00416D6C
:1029D0006178205A00416D6178205900416D61781D
:1029E000205900416D6178205800416D6178205870
:1029F00000412D74726176656C00412D74726176B0
:102A0000656C00412D7265747261637400412D72B2
:102A100065747261637400416363656C0041636354
:102A2000656C00416476616E6365642053657474FF
:102A3000696E6773005654726176206D696E005638
:102A400054726176206D696E00566D696E00566D28
:102A5000696E00566D6178204500566D617820459D
:102A600000566D6178205A00566D6178205A0056E4
:102A70006D6178205900566D6178205900566D615E
:102A800078205800566D6178205800416476616E58
:102A90006365642053657474696E6773004C6F617D
:102AA00064206D6D004C6F6164206D6D00556E6C1F
:102AB0006F6164206D6D00556E6C6F6164206D6D8B
:102AC00000416476616E6365204B00416476616EFF
:102AD0006365204B00416476616E636564205365D5
:102AE0007474696E677300450045005A005A0058B7
:102AF0005900585900436F6E74726F6C00446973CB
:102B000061626C65207374657070657273004D3816
:102B100034004C6576656C2058204178697300005C
:102B20004175746F20686F6D6500473238004D6FD6
:102B300076652061786973004D61696E004578742F
:102B4000727564657220004D6F7665205A004D6F76
:102B500076652059004D6F76652058004D6F76657B
:102B60006D656E7400457874727564657220004DF1
:102B70006F766520302E316D6D004D6F766520319A
:102B80006D6D004D6F76652031306D6D004D6F7647
:102B900065206178697300486F74656E6420746F96
:102BA0006F20636F6C640045787472756465722081
:102BB000004D6F7665205A004D6F76652059004DA7
:102BC0006F76652058004D6F7665205A004D6F7600
:102BD000652059004D6F7665205800576169742053
:102BE000666F720066696C616D656E7420707572D7
:102BF00067650000506C6561736520776169742EAC
:102C000000507265737320627574746F6E00746F18
:102C100020726573756D65207072696E74005761FE
:102C2000697420666F720066696C616D656E7420F0
:102C30006C6F616400496E736572742066696C61C3
:102C40006D656E7400616E642070726573732062CE
:102C50007574746F6E00746F20636F6E74696E7537
:102C60006500507265737320627574746F6E0074C2
:102C70006F2068656174206E6F7A7A6C65004E6FA4
:102C80007A7A6C652068656174696E6700506C655E
:102C900061736520776169742E2E2E005761697407
:102CA00020666F720066696C616D656E7420756E6A
:102CB0006C6F6164005761697420666F72006669A9
:102CC0006C616D656E74206368616E676500746F1A
:102CD000207374617274004368616E67696E672067
:102CE00046696C616D656E7400554E4C4F414420D1
:102CF00046494C414D454E54004C4F4144204649B5
:102D00004C414D454E540020204E6F7A7A6C653A06
:102D100020002000456E642066696C616D656E74EC
:102D2000206368616E6765005075726765206D6F1E
:102D3000726500004368616E67652066696C616D4D
:102D4000656E7400556E6C6F61642066696C616DB0
:102D5000656E74004C6F61642066696C616D656EB0
:102D600074004D36303020423020542564004D37F9
:102D70003032203B2564004D37303220542564002A
:102D80004D37303120542564005072656865617498
:102D900020437573746F6D005072656865617420AF
:102DA000437573746F6D005072656865617420417E
:102DB0004253005072656865617420504C41004276
:102DC00061636B004E6F2053442063617264005056
:102DD00072696E742066726F6D2053440041626F99
:102DE0007574205072696E746572004368616E6715
:102DF000652066696C616D656E74004368616E671D
:102E0000652066696C616D656E74004D36303020EA
:102E1000423000436F6E66696775726174696F6EE8
:102E20000054656D7065726174757265004D6F76E2
:102E3000656D656E7400526573756D65207072699D
:102E40006E740054756E650053746F7020707269F3
:102E50006E74005061757365207072696E740049FC
:102E60006E666F2073637265656E0053746F7020B9
:102E70007072696E74004D61696E005072696E7493
:102E80002061626F72746564004D3234004D3235DA
:102E900020500A4D32340050726F6265205A204F24
:102EA0006666736574004261627973746570205957
:102EB000004261627973746570205800466C6F77C8
:102EC00000466C6F770046616E2073706565640024
:102ED00046616E20737065656400426564004265FA
:102EE00064004E6F7A7A6C65004E6F7A7A6C65007A
:102EF0005370656564005370656564004D61696E6B
:102F00000042616279737465702059004261627990
:102F100073746570205800436F6F6C646F776E0038
:102F200046616E2073706565640046616E20737043
:102F30006565640042656400426564004E6F7A7A9C
:102F40006C65004E6F7A7A6C65004D61696E005257
:102F50006573746F7265206661696C736166650084
:102F60004C6F61642073657474696E677300537489
:102F70006F72652073657474696E67730050726F49
:102F80006265205A204F66667365740041647661FD
:102F90006E6365642053657474696E6773004D6178
:102FA000696E0050726F6265205A204F66667365C5
:102FB00074004C756C7A426F74204D696E69207292
:102FC000656164792E005072696E74696E672E2E89
:102FD0002E005072696E74207061757365640043D1
:102FE0006172642072656D6F76656400436172641E
:102FF00020696E736572746564004D3331004361FE
:103000006E6E6F7420656E7465722073756264698C
:10301000723A20006F70656E206661696C65642C81
:103020002046696C653A20006175746F25632E67D0
:10303000006572726F722077726974696E672074AE
:103040006F2066696C650A004E6F742053442070CF
:1030500072696E74696E670A005344207072696EFB
:1030600074696E672062797465200044656C6574CC
:10307000696F6E206661696C65642C2046696C65B9
:103080003A200046696C652064656C657465643A35
:103090000057726974696E6720746F2066696C6589
:1030A0003A20006F70656E206661696C65642C2043
:1030B00046696C653A20006F70656E206661696CC8
:1030C00065642C2046696C653A200046696C652071
:1030D00073656C65637465640A002053697A653AA8
:1030E000200046696C65206F70656E65643A20004B
:1030F0002066696C653A2000667265736800646FCB
:10310000696E67004E6F772000454E44205355424C
:10311000524F5554494E450A002220706F730022C9
:1031200020706172656E743A2200535542524F55B9
:1031300054494E452043414C4C207461726765747C
:103140003A2200747279696E6720746F2063616C33
:103150006C207375622D67636F64652066696C65AA
:1031600073207769746820746F6F206D616E7920A9
:103170006C6576656C732E204D4158206C657665C4
:103180006C2069733A310A004D3234004D323320DD
:1031900025730053442063617264206F6B0A006FD3
:1031A00070656E526F6F74206661696C65640A00A9
:1031B000766F6C756D652E696E6974206661696CD9
:1031C00065640A00534420696E6974206661696C05
:1031D0000A00286E6F2066696C65290043616E6E77
:1031E0006F74206F70656E20737562646972200061
:1031F0007C3C3E5E2B3D3F2F5B5D3B2C2A225C00DE
:103200004F4646004F4E006563686F3A0045727244
:103210006F723A004572726F722077726974696ECC
:103220006720746F20454550524F4D210A0050725F
:1032300065737320627574746F6E20286F72204DF1
:103240003130382920746F2068656174206E6F7A80
:103250007A6C650A00507265737320627574746FBE
:103260006E20286F72204D3130382920746F207203
:103270006573756D650A00496E73657274206669C1
:103280006C616D656E7420616E642070726573731D
:1032900020627574746F6E20286F72204D31303843
:1032A000290A004D3630303A20546F6F20636F6C1E
:1032B0006400486F74656E6420746F6F20636F6C78
:1032C000640A00486F74656E6420746F6F20636FCA
:1032D0006C640A00496E736572742066696C616D76
:1032E000656E7420616E6420707265737320627500
:1032F00074746F6E20286F72204D313038290A00A7
:1033000063616E63656C00726573756D65640072F0
:103310006573756D650070617573656400706F77B6
:1033200065726F6666002F2F616374696F6E3A0075
:1033300020573A0020573A004578747275646572D8
:1033400020436F6F6C696E672E2E2E004578747265
:10335000756465722048656174696E672E2E2E0053
:10336000202F002042403A0020403A004D383420BF
:10337000582059205A204500546865726D616C20B0
:1033800052756E6177617900453120544845524D40
:10339000414C2052554E415741590042454420541A
:1033A0004845524D414C2052554E415741590020FD
:1033B0002D20496E76616C6964206578747275643D
:1033C0006572206E756D62657220210A0048656124
:1033D00074696E67206661696C656400426564208B
:1033E00068656174696E67206661696C6564004830
:1033F000656174696E67206661696C65640045315A
:103400002048656174696E67206661696C65640057
:103410004D494E54454D5020747269676765726519
:1034200064004531204572723A204D494E54454D55
:1034300050004572723A204D494E54454D5020423D
:103440004544004D415854454D502074726967679A
:1034500065726564004531204572723A204D4158CD
:1034600054454D50004572723A204D415854454DD7
:103470005020424544006265640A002C2073797331
:1034800074656D2073746F70706564212048656188
:103490007465725F49443A200023646566696E650D
:1034A0002044454641554C545F004B6420004B6915
:1034B00020004B70200000626564005049442041A8
:1034C00075746F74756E652066696E69736865647E
:1034D000212050757420746865206C617374204BD2
:1034E000702C204B6920616E64204B6420636F6EEA
:1034F0007374616E74732066726F6D2062656C6F99
:103500007720696E746F20436F6E666967757261AC
:1035100074696F6E2E680A00504944204175746FBB
:1035200074756E65206661696C6564212074696DCF
:10353000656F75740A00546865726D616C20527510
:103540006E6177617900453120544845524D414CB8
:103550002052554E41574159004245442054484558
:10356000524D414C2052554E4157415900486561DA
:1035700074696E67206661696C6564004531204836
:10358000656174696E67206661696C656400426597
:10359000642068656174696E67206661696C656442
:1035A00000504944204175746F74756E65206661E2
:1035B000696C6564212054656D7065726174757203
:1035C0006520746F6F20686967680A00204B643A51
:1035D0002000204B693A2000204B703A20000A203E
:1035E000436C617373696320504944200A0020547E
:1035F000753A2000204B753A2000206D61783A2002
:1036000000206D696E3A200020643A200020626933
:1036100061733A2000504944204175746F74756E8F
:10362000652073746172740A0050494420417574B6
:103630006F74756E65206661696C656421205465E0
:103640006D706572617475726520746F6F20686942
:1036500067680A001000AD0330016A0150022B01B7
:1036600070030A019004F500B005E500D006D8000B
:10367000F007CE001009C500300ABE00500BB7009D
:10368000700CB100900DAB00B00EA600D00FA200E0
:10369000F0109D0010129900301395005014920004
:1036A00070158E0090168B00B0178700D01884001C
:1036B000F0198100101B7E00301C7B00501D79002A
:1036C000701E7600901F7300B0207000D0216E0035
:1036D000F0226B001024690030256600502663003C
:1036E0007027610090285E00B0295C00D02A590044
:1036F000F02B5600102D5400302E5100502F4E004C
:1037000070304B0090314800B0324500D033420059
:10371000F0343E0010363B0030373700503833006D
:1037200070392E00903A2900B03B2300D03C1B009A
:10373000F03D1100103F0100F03F00001000C902F1
:1037400010012C014001220170011801B0010E018D
:10375000F00104015002FA00B002F0003003E6006C
:10376000D003DC009004D2007005C800A006BE00A3
:103770000008B400B009AA00D00BA000600E9600AB
:1037800060118C000015820020197800C01D6E00A9
:10379000A0226400B0275A00902C5000003146004F
:1037A000E0343C0010383200903A2800603C1E00A3
:1037B000A03D1400803E0A00203F00006F70656E3F
:1037C00000545249474745524544003A20007A5F29
:1037D0006D6178007A5F6D696E00795F6D61780068
:1037E000795F6D696E00785F6D617800785F6D69F3
:1037F0006E005265706F7274696E6720656E6473D7
:10380000746F70207374617475730A00456E64730D
:10381000746F707320256320256320256320256342
:1038200000205A3A0020593A0020583A00656E6448
:1038300073746F7073206869743A2000486F6D6903
:103840006E67206661696C656400496E76616C69BB
:10385000642065787472756465720A0045303A2098
:10386000005A3A2000593A20004D53312C4D533222
:103870002C4D53332050696E730A583A20004D691D
:1038800063726F737465707320756E617661696CB5
:1038900061626C650A00205A3A0020593A002043C0
:1038A0006F756E7420583A00C23100001C2600006B
:1038B000F4190000D80F0000EB080000C00400005D
:1038C000750200004001000024F4D43050C38E2063
:1038D000C2A24017828B7011127A910D816CD90AA5
:1038E000A861E108C7586607615143061E4B5D0594
:1038F000C145A7041A411104093D980371393103E8
:103900004036DB0265339102D4305402802E1D0212
:10391000632CEE01752AC501B028A0011027810192
:103920008F2564012B244B01E0223401AC211F01BF
:103930008D200D01801FFC00841EED00971DDF000F
:10394000B81CD200E61BC600201BBC00641AB200E3
:10395000B219A8000A19A0006A189900D11791009D
:1039600040178B00B516840031167E00B315790020
:103970003A157300C7146F0058146A00EE136600FE
:103980008813630025135E00C7125B006C1257009A
:1039900015125400C111510070114F0021114B003C
:1039A000D61049008D104700461044000210420016
:1039B000C00F4000800F3E00420F3C00060F3B004E
:1039C000CB0E3800930E37005C0E3500270E340006
:1039D000F30D3200C10D3100900D3000600D2E004E
:1039E000320D2D00050D2C00D90C2B00AE0C29003A
:1039F000850C29005C0C2700350C27000E0C2600D6
:103A0000E80B2400C40B2400A00B23007D0B230033
:103A10005A0B2100390B2100180B2000F80A1F0057
:103A2000D90A1E00BB0A1E009D0A1D00800A1D0047
:103A3000630A1C00470A1B002C0A1B00110A1A000B
:103A4000F7091A00DD091900C4091900AB091900AA
:103A5000920917007B091800630917004C0916002A
:103A600036091600200916000A091500F508150088
:103A7000E0081400CC081400B8081400A4081400CE
:103A8000900813007D0812006B08130058081200FC
:103A90004608120034081100230811001208110012
:103AA00001081100F0071000E0071000D007100017
:103AB000C0071000B0070F00A107100091070E000B
:103AC00083070F0074070F0065070E0057070E00ED
:103AD00049070E003B070D002E070E0020070D00C2
:103AE00013070D0006070D00F9060C00ED060D008A
:103AF000E0060C00D4060C00C8060C00BC060C0046
:103B0000B0060C00A4060B0099060C008D060B00F5
:103B100082060B0077060B006C060B0061060A009C
:103B200057060B004C060A0042060A0038060A0037
:103B30002E060A0024060A001A060A0010060900CA
:103B400007060A00FD050900F4050900EB05090058
:103B5000E2050900D9050900D0050900C7050900DB
:103B6000BE050900B5050800AD050800A50509005A
:103B70009C050800940508008C05080084050800D1
:103B80007C050800740508006C0507006505080041
:103B90005D050700560508004E05070047050700AC
:103BA0004005080038050700310507002A05070011
:103BB000230507001C050600160507000F05070072
:103BC0000805060002050700FB040600F5040700CF
:103BD000EE040600E8040600E2040700DB04060029
:103BE000D5040600CF040600C9040600C30406007D
:103BF000BD040600B7040600B1040500AC040600CD
:103C0000A6040600A00405009B0406009504050018
:103C1000900406008A04050085040500800406005F
:103C20007A04050075040500700405006B040500A6
:103C300066040500610405005C04050057040500E6
:103C4000520405004D040500480405004304050026
:103C50003E0404003A040500350405003004040065
:103C60002C04050027040400230405001E0404009E
:103C70001A04040016040500110404000D040400D5
:103C8000090405000404040000040400FC0304000B
:103C9000F8030400F4030400F0030400EC03040040
:103CA000E8030400E4030400E0030400DC03040070
:103CB000D8030400D4030400D0030400CC030400A0
:103CC000C8030300C503030024F404D9201BC40C5B
:103CD0005C0E9804C4095F0265077101F405F900E0
:103CE000FB04B30048048700C10369005803550072
:103CF00003034500BE023A008402310053022A0049
:103D00002902250004022000E4011C00C80119005A
:103D1000AF01170098011400840113007101100015
:103D20006101100051010E0043010D0036010B002E
:103D30002B010B0020010B00150109000C010900EB
:103D400003010800FB000800F3000800EB00070077
:103D5000E4000600DE000600D8000600D2000600DF
:103D6000CC000500C7000500C2000500BD0004002E
:103D7000B9000400B5000400B1000400AD00040067
:103D8000A9000400A5000300A20003009F00040096
:103D90009B000300980003009500020093000300BD
:103DA000900003008D0002008B00030088000200D9
:103DB0008600020084000300810002007F000200F0
:103DC0007D0002007B000200790002007700010004
:103DD000760002007400020072000100710002000F
:103DE0006F0002006D0001006C0002006A0001001B
:103DF0006900020067000100660001006500010023
:103E00006400020062000100610001006000010026
:103E10005F0002005D0001005C0001005B0001002A
:103E20005A0001005900010058000100570001002C
:103E3000560001005500010054000100530000002D
:103E40005300010052000100510001005000010028
:103E50004F0001004E0000004E0001004D00010027
:103E60004C0001004B0000004B0001004A00010023
:103E7000490001004800000048000100470001001F
:103E8000460000004600010045000000450001001A
:103E90004400010043000000430001004200000014
:103EA000420001004100000041000100400001000B
:103EB0003F0000003F0001003E0000003E00010006
:103EC0003D0000003D0001003C0000003C000000FF
:103ED0003C0001003B0000003B0001003A000000F4
:103EE0003A000100390000003900010038000000EC
:103EF00038000000380001003700000037000100E2
:103F000036000000360000003600010035000000D9
:103F100035000000350001003400000034000000CE
:103F200034000100330000003300000033000100C2
:103F300032000000320000003200010031000000B9
:103F400031000000310001003000000030000000AE
:103F5000300001002F0000002F0000002F000000A3
:103F60002F0001002E0000002E0000002E00010096
:103F70002D0000002D0000002D0000002D0001008C
:103F80002C0000002C0000002C0000002C00010080
:103F90002B0000002B0000002B0000002B00010074
:103FA0002A0000002A0000002A0000002A00010068
:103FB000290000002900000029000000290000005D
:103FC000290001002800000028000000280000004F
:103FD0002800000028000100270000002700000042
:103FE0002700000027000000270001002600000035
:103FF0002600000026000000260000002600010028
:10400000250000002500000025000000250000001C
:10401000250000002500010024000000240000000D
:104020002400000024000000240001002300000000
:1040300023000000230000002300000023000000F4
:1040400023000000230001002200000022000000E5
:1040500022000000220000002200000022000100D7
:1040600021000000210000002100000021000000CC
:1040700021000000210000002100010020000000BC
:1040800020000000200000002000000020000000B0
:104090002000000020000000200001001F000000A0
:1040A0001F0000001F0000001F0000001F00000094
:1040B0001F0000001F0001001E0000001E00000085
:1040C0001E0000001E0000003A0A0020286D6D2925
:1040D000002055004C0046696C616D656E74206C63
:1040E0006F61642F756E6C6F6164206C656E6774B0
:1040F00068733A0A00204500205A0020204D3930CC
:104100003720580053746570706572206D6F746F3E
:10411000722063757272656E74733A0A0020204DC6
:10412000393030204B004C696E65617220416476F5
:10413000616E63653A0A0020204D383531205A00FF
:104140005A2D50726F6265204F6666736574002049
:10415000440020490020204D3330342050002044BA
:104160000020490020204D33303120500050494478
:104170002073657474696E67733A0A0020460020E4
:10418000420020480020204D3134352053004D613D
:1041900074657269616C2068656174757020706106
:1041A00072616D65746572733A0A0020204D343275
:1041B000302053004175746F20426564204C657651
:1041C000656C696E673A0A00204500205A00205944
:1041D0000020580020540020530020204D3230355C
:1041E00020420020453C6D61785F655F6A65726BB7
:1041F0003E0020583C6D61785F785F6A65726B3E67
:1042000020593C6D61785F795F6A65726B3E205A18
:104210003C6D61785F7A5F6A65726B3E00416476DF
:10422000616E6365643A20423C6D696E5F736567D9
:104230006D656E745F74696D655F75733E20533C88
:104240006D696E5F66656564726174653E20543C9D
:104250006D696E5F74726176656C5F6665656472C8
:104260006174653E0020540020520020204D323001
:1042700034205000416363656C65726174696F6ED0
:104280002028756E6974732F7332293A20503C7060
:1042900072696E745F616363656C3E20523C726547
:1042A00074726163745F616363656C3E20543C7437
:1042B000726176656C5F616363656C3E0A002045E0
:1042C00000205A0020590020204D32303120580063
:1042D0004D6178696D756D20416363656C657261D0
:1042E00074696F6E2028756E6974732F7332293A62
:1042F0000A00204500205A0020590020204D32306D
:10430000332058004D6178696D756D206665656470
:1043100072617465732028756E6974732F73293AFE
:104320000A0053746570732070657220756E69742D
:104330003A0A0020204D3134392043203B20556E6D
:1043400069747320696E2043656C736975730A0024
:104350002020473231202020203B20556E69747385
:1043600020696E206D6D0020204D363033200048CE
:10437000617264636F6465642044656661756C7422
:104380002053657474696E6773204C6F6164656453
:104390000A00282300002823000064000000E8032E
:1043A000000000009643000096430000004100001A
:1043B00020420000C9420000C9420000C844000079
:1043C000D243290A002062797465733B20637263CB
:1043D00020002073746F7265642073657474696E55
:1043E00067732072657472696576656420280020A1
:1043F0002863616C63756C6174656429210A00200F
:10440000213D2000454550524F4D20435243206DE1
:1044100069736D61746368202D202873746F7265F1
:10442000642920002053697A653A2000496E64654A
:10443000783A2000204D61726C696E3D5636342901
:104440000A0028454550524F4D3D00454550524FBA
:104450004D2076657273696F6E206D69736D61743E
:1044600063682000290A002062797465733B206329
:104470007263200053657474696E67732053746FA0
:10448000726564202800454550524F4D2064617488
:104490006173697A65206572726F722E0A005072BC
:1044A0006F62696E67206661696C65640A005072AC
:1044B0006F62696E67206661696C6564005761723E
:1044C0006E696E673A20486F6D696E672042756D40
:1044D000702044697669736F72203C20310A0002B3
:1044E0000204486F6D652025732573257320666966
:1044F000727374002066697273740A005A0059005E
:104500005800486F6D65200020746F6F206C6F6ECF
:104510006720657874727573696F6E207072657646
:10452000656E7465640A0020636F6C64206578743E
:10453000727573696F6E2070726576656E746564EE
:104540000A0020453A00205A3A0020593A00583AC9
:10455000000000F0410000F04100000041FF0101B7
:104560000000A0400000A0400000004000002543E3
:104570000000454300002143000040C000003E43CE
:1045800000001F430000224300003E4300001F4381
:10459000000040C00000E0C0000000C020746F6F49
:1045A000206C6F6E6720657874727573696F6E200A
:1045B00070726576656E7465640A0020636F6C6462
:1045C00020657874727573696F6E20707265766598
:1045D0006E7465640A00627573793A207061757350
:1045E000656420666F7220696E7075740A0062756A
:1045F00073793A2070617573656420666F722075F7
:104600007365720A00627573793A2070726F636520
:104610007373696E670A004D3131372050726F62D3
:1046200065207375636365737366756C0A00204952
:104630006E76616C69642065787472756465722049
:1046400000205A3A200020593A2000426564205840
:104650003A200050726F6265205A204F666673657B
:10466000743A20003F5A206F7574206F6620726183
:104670006E676520282D3220746F2035290A004D81
:1046800031343520533C696E6465783E206F757413
:10469000206F662072616E67652028302D31290AEF
:1046A00000436C69636B20746F20726573756D6570
:1046B0002E2E2E00556E6B6E6F776E20636F6D6DB4
:1046C000616E643A202200454550524F4D204F4BB9
:1046D0000A004E6F206D6F76652E004543484F00EF
:1046E000494E464F004552524F5253004452595280
:1046F000554E00434F4D4D554E49434154494F4E41
:10470000006F666600DB46E046E546EC46F346444D
:10471000454255473A004C756C7A426F74204D699A
:104720006E69204C4344204F46462E00205A0020FC
:104730005900580020204D61783A2000205A00206E
:104740005900580020204D696E3A2000536F66745E
:1047500020656E6473746F70733A2000256973006E
:1047600025696D20256973002569682025696D20FC
:1047700025697300256964202569682025696D20F5
:1047800025697300256979202569642025696820D9
:1047900025696D20256973005072696E74207469F3
:1047A0006D653A20004D3131332053002F2F20000A
:1047B0004361703A004D4F54494F4E5F4D4F444551
:1047C0005300544845524D414C5F50524F5445435D
:1047D00054494F4E004155544F5245504F52545F2B
:1047E00053445F5354415455530050524F4D50540D
:1047F0005F535550504F525400454D455247454E1A
:1048000043595F50415253455200434153455F4C19
:10481000494748545F4252494748544E4553530014
:10482000544F47474C455F4C494748545300534FFA
:104830004654574152455F504F57455200425549E3
:104840004C445F50455243454E54004C4556454CF0
:10485000494E475F44415441005A5F50524F4245D0
:10486000004155544F4C4556454C005052494E540A
:104870005F4A4F420050524F4752455353004155F3
:10488000544F5245504F52545F54454D5000564F6F
:104890004C554D455452494300454550524F4D00EB
:1048A00053455249414C5F584F4E5F584F46460062
:1048B0004649524D574152455F4E414D453A4D6133
:1048C000726C696E20204649524D574152455F56E1
:1048D000455253494F4E3A322E302E302E39352024
:1048E00045585452554445525F545950453A4165D4
:1048F000726F7374727564657220534F55524345DD
:104900005F434F44455F55524C3A68747470733A34
:104910002F2F636F64652E616C6570686F626A65C6
:104920006374732E636F6D2F646966667573696F48
:104930006E2F4D41524C494E2050524F544F434FD1
:104940004C5F56455253494F4E3A312E30204D411F
:104950004348494E455F545950453A4C756C7A422C
:104960006F74204D696E69204C4344204558545261
:10497000554445525F434F554E543A3120555549A1
:10498000443A30383366363866312D303238652D4A
:10499000343934632D393865312D663265306466BB
:1049A0006165653961350A0020284E6F742079658C
:1049B00074206D65617375726564290020204176ED
:1049C0006572616765206D656173757265642062EB
:1049D00061636B6C61736820286D6D293A0020203B
:1049E000536D6F6F7468696E6720286D6D293A206A
:1049F00020202020202020202020202020202020B7
:104A0000530020204261636B6C61736820446973BA
:104A100074616E636520286D6D293A202020202066
:104A20002020200020202020202846312E30203D2C
:104A30002066756C6C2C2046302E30203D206E6F29
:104A40006E65290A002020436F7272656374696F76
:104A50006E20416D6F756E742F466164652D6F75A4
:104A6000743A202020202046006163746976653AFC
:104A70000A00696E004261636B6C61736820636F4A
:104A80007272656374696F6E2069732000205A002A
:104A900020506F736974696F6E616C204572726F1C
:104AA000723A0A004E6F7A7A6C6520546970204F12
:104AB000757465722044696D656E73696F6E733AC3
:104AC0000A002020546F703A2000202046726F6E3A
:104AD000743A200020204C6566743A2000426163DD
:104AE0006B6C6173683A0A00205A0043656E746506
:104AF000723A0A00202046726F6E743A200020201D
:104B00004C6566743A20002020546F703A200053A0
:104B1000696465733A0A00426564204C6576656C89
:104B2000696E6720004661696C656420746F20655A
:104B30006E61626C6520426564204C6576656C69C7
:104B40006E670A00426564204C6576656C20436F91
:104B50007272656374696F6E204D61747269783A20
:104B6000000A0A426564204C6576656C20436F72CA
:104B700072656374696F6E204D61747269783A0072
:104B8000202B000A436F727265637465642042656E
:104B900064204865696768742076732E20426564D6
:104BA00020546F706F6C6F67793A0A00202B000AEF
:104BB0004265642048656967687420546F706F6748
:104BC00072617068793A0A2020202B2D2D2D204209
:104BD00041434B202D2D2B0A2020207C20202020FB
:104BE000202020202020207C0A204C207C202020F7
:104BF00020282B29202020207C20520A2045207CA0
:104C000020202020202020202020207C20490A2035
:104C100046207C20282D29204E20282B29207C204E
:104C2000470A2054207C20202020202020202020E3
:104C3000207C20480A2020207C20202020282D298C
:104C4000202020207C20540A2020207C202020208E
:104C5000202020202020207C0A2020204F2D2D20C5
:104C600046524F4E54202D2D2B0A2028302C30290F
:104C70000A003474682070726F626520706F696E0C
:104C8000742C2064697374616E63652066726F6D45
:104C900020706C616E653A200020284452595255AC
:104CA0004E2900473239204175746F2042656420D7
:104CB0004C6576656C696E67003F20284C2C522C41
:104CC000462C4229206F7574206F6620626F756EC6
:104CD00064732E0A003F50726F626520706F696EB8
:104CE00074732028592920697320696D706C61756F
:104CF0007369626C652028322D32292E0A003F50DC
:104D0000726F626520706F696E7473202858292055
:104D1000697320696D706C61757369626C652028B8
:104D2000322D32292E0A003F2856296572626F7390
:104D300065206C6576656C20697320696D706C61A7
:104D4000757369626C652028302D34292E0A004362
:104D5000757272656E742066696C653A2000456EE6
:104D6000642066696C65206C6973740A004265672B
:104D7000696E2066696C65206C6973740A00416411
:104D800076616E6365204B3D003F4B2076616C750C
:104D900065206F7574206F662072616E67652028CC
:104DA000302D3130292E0A004D31313720486F74B3
:104DB00020456E642048656174696E672E2E2E0A48
:104DC0004D31303420533137302054300A47323897
:104DD000204F310A473120593235205A3130204690
:104DE000353030300A4D313039205231373020548F
:104DF000300A4D313137205265776970696E67200E
:104E00006E6F7A7A6C650A54300A4731205834350F
:104E100020593137322046353030300A4731205A58
:104E2000310A4D31303920523137300A473120585C
:104E3000343520593137322046343030300A47314A
:104E40002058343520593137322046343030300A3A
:104E500047312058343520593137322046343030EC
:104E6000300A473120583435205931373220463402
:104E70003030300A4731205834352059313732200C
:104E800046343030300A47312058343520593137D4
:104E9000322046343030300A4731205834352059DA
:104EA0003137322046343030300A473120583435DB
:104EB00020593137322046343030300A47312058BB
:104EC000343520593137322046343030300A4731BA
:104ED0002058343520593137322046343030300AAA
:104EE000473120583435205931373220463430305C
:104EF000300A473120583435205931373220463472
:104F00003030300A4731205A31350A4D31303620A1
:104F100053323535200A47302058302059300A4D59
:104F200031303920523136302054300A4D3130374B
:104F30000A0020466C6F773A200020643A0020690E
:104F40003A0020703A00204500205A0020590020E5
:104F50004D393220580043290A0061626C65642093
:104F6000286D696E2074656D70200064697300653A
:104F70006E00436F6C64206578747275646573208D
:104F80006172652000205400205200416363656C0B
:104F900065726174696F6E3A205000496E76616C7B
:104FA00069642065787472756465720A0020643AD9
:104FB0000020693A0020703A00536C6565702E2E0F
:104FC0002E0047322F473320626164207061726186
:104FD0006D65746572730A0050726F6265205A20A5
:104FE0004F66667365743A2000446F6E6520736186
:104FF00076696E672066696C652E0A0053442072DC
:10500000656164206572726F720A00446F6E65207C
:105010007072696E74696E672066696C650A005308
:10502000544F505045442E20005072696E74657282
:105030002073746F707065642064756520746F20D0
:105040006572726F72732E204669782074686520CD
:105050006572726F7220616E6420757365204D39C0
:10506000393920746F20726573746172742E202830
:1050700054656D7065726174757265206973207214
:10508000657365742E20536574206974206166749D
:1050900065722072657374617274696E67290A00A3
:1050A0004E6F20436865636B73756D207769746814
:1050B000206C696E65206E756D6265722C204C6186
:1050C0007374204C696E653A20004E6F204368650A
:1050D000636B73756D2077697468206C696E6520E9
:1050E0006E756D6265722C204C617374204C696E14
:1050F000653A2000636865636B73756D206D697335
:105100006D617463682C204C617374204C696E650A
:105110003A20004C696E65204E756D62657220699B
:1051200073206E6F74204C617374204C696E65201F
:105130004E756D6265722B312C204C617374204C5E
:10514000696E653A20004D31313000526573656EED
:10515000643A20002042002050006F6B00656E71A1
:1051600075657565696E6720220050494420417558
:10517000746F74756E65206661696C656421204288
:105180006164206578747275646572206E756D62F5
:1051900065720A0042656420636F6F6C696E672EEA
:1051A0002E2E004265642068656174696E672E2E3C
:1051B0002E006F6B00473238205A0A47302058388B
:1051C0003020593139302046333030300A4D3131BA
:1051D00037205072696E742061626F727465642E3C
:1051E000002020506C616E6E657242756666657255
:1051F00042797465733A20002046726565204D65DA
:105200006D6F72793A2000436F6D70696C65643A16
:10521000204D617220203420323031390A00207C48
:1052200020417574686F723A2028416C657068205F
:105230004F626A6563747320496E632E2C204C752F
:105240006C7A426F7420476974205265706F73697D
:10525000746F7279290A0000204C617374205570B4
:1052600064617465643A2000322E302E302E393558
:105270000A004D61726C696E0020536F667477612D
:1052800072652052657365740A0020576174636803
:10529000646F672052657365740A002042726F77ED
:1052A0006E206F75742052657365740A002045780E
:1052B0007465726E616C2052657365740A00506F7C
:1052C00077657255700A0073746172740A004B49F5
:1052D0004C4C45442E20005072696E7465722068F3
:1052E000616C7465642E206B696C6C282920636185
:1052F0006C6C6564210A004B494C4C2063617573EA
:105300006564206279204B494C4C20627574746F3F
:105310006E2F70696E0A004B494C4C2063617573A7
:10532000656420627920746F6F206D7563682069F1
:105330006E6163746976652074696D65202D2063E4
:10534000757272656E7420636F6D6D616E643A2064
:10535000004D3132310A4730205A31300A47323855
:105360002058302059300A4731320A4D3130392027
:10537000523136300A4D3131372050726F62696ECA
:1053800067206265640070726F62655F726577693D
:1053900070650050726F62696E67206661696C6546
:1053A00064004D31313720426564206C6576656C50
:1053B000696E67206661696C65642E0A4730205A01
:1053C00031300A47302045300A4D333030205032DA
:1053D0003520533838300A4D3330302050353020A6
:1053E00053300A4D33303020503235205338383066
:1053F0000A4D333030205035302053300A4D333091
:10540000302050323520533838300A473420533159
:105410000070726F62655F6661696C6564005072EE
:105420006F7465637465642050696E0A0025301DD1
:105430000C1E282924311C0B184527232F1B0A1763
:105440004443222B1A4142043803FF36040806065F
:105450000001CA40BC6C7676A38EF4E3E300E10061
:10546000DF00967611241FBECFEFD1E2DEBFCDBFA5
:1054700000E00CBF14E0A0E0B2E0EAEFF1E702E0E8
:105480000BBF02C007900D92A030B107D9F726E1FB
:10549000A0E0B4E001C01D92AC31B207E1F71AE21E
:1054A000C1E3DAE200E006C021970109802FFE0186
:1054B0000F940731C932D10780E00807A9F70E948D
:1054C00060350D94EC380C9400001F920F920FB6CB
:1054D0000F9211242F933F938F939F93AF93BF937A
:1054E0008091010490910204A0910304B0910404FE
:1054F0003091000423E0230F2D3720F40196A11DE5
:10550000B11D05C026E8230F0296A11DB11D2093F1
:1055100000048093010490930204A0930304B093C9
:1055200004048091050490910604A0910704B091B1
:1055300008040196A11DB11D8093050490930604F3
:10554000A0930704B0930804BF91AF919F918F91EE
:105550003F912F910F900FBE0F901F9018952FB76E
:10556000F894609101047091020480910304909179
:1055700004042FBF08953FB7F894809105049091DB
:105580000604A0910704B091080426B5A89B05C0A5
:105590002F3F19F00196A11DB11D3FBFBA2FA92FB2
:1055A000982F8827820F911DA11DB11DBC01CD012F
:1055B00042E0660F771F881F991F4A95D1F708951B
:1055C0008F929F92AF92BF92CF92DF92EF92FF9213
:1055D0006B017C01D0DF4B015C01C114D104E104FB
:1055E000F104F1F091D3C7DFDC01CB0188199909EF
:1055F000AA09BB09883E9340A105B10570F321E0DB
:10560000C21AD108E108F10888EE880E83E0981EDE
:10561000A11CB11CC114D104E104F10421F7DDCFB8
:10562000FF90EF90DF90CF90BF90AF909F908F90C2
:105630000895789484B5826084BD84B5816084BD0A
:1056400085B5826085BD85B5816085BDEEE6F0E0FB
:10565000808181608083E1E8F0E010828081826057
:105660008083808181608083E0E8F0E080818160D8
:105670008083E1EBF0E0808184608083E0EBF0E008
:10568000808181608083E1E9F0E0808182608083B5
:10569000808181608083E0E9F0E0808181608083A7
:1056A000E1EAF0E080818260808380818160808394
:1056B000E0EAF0E0808181608083E1E2F1E08081D6
:1056C00082608083808181608083E0E2F1E080817C
:1056D00081608083EAE7F0E080818460808380815C
:1056E0008260808380818160808380818068808304
:1056F0001092C10008951F93CF93DF93182FEB01F1
:1057000061E016D1209711F460E004C0CF3FD105CD
:1057100031F461E0812FDF91CF911F9145C1E12FDD
:10572000F0E0EB5FFD4FE4914E2F50E0FA0131972E
:10573000E231F10508F09DC08827EE58FF4F8F4FEA
:105740000D94073184B5806884BDC7BD97C084B50A
:10575000806284BDC8BD92C08091800080688093C3
:105760008000D0938900C093880088C08091800019
:10577000806280938000D0938B00C0938A007EC0AB
:1057800080918000886080938000D0938D00C093CA
:105790008C0074C08091B00080688093B000C0938A
:1057A000B3006CC08091B00080628093B000C09361
:1057B000B40064C080919000806880939000D09382
:1057C0009900C09398005AC08091900080628093A5
:1057D0009000D0939B00C0939A0050C0809190009D
:1057E000886080939000D0939D00C0939C0046C039
:1057F0008091A00080688093A0008091A0008F7BA2
:105800008093A000D093A900C093A80037C08091D6
:10581000A00080628093A000D093AB00C093AA0048
:105820002DC08091A00088608093A000D093AD002F
:10583000C093AC0023C08091200180688093200138
:10584000D0932901C093280119C080912001806262
:1058500080932001D0932B01C0932A010FC0809127
:105860002001886080932001D0932D01C0932C01EA
:1058700005C0C038D1050CF04CCF46CFDF91CF9199
:105880001F91089590E0FC013197E231F10508F095
:105890004EC08827EC57FF4F8F4F0D9407318091F2
:1058A00080008F7703C0809180008F7D809380007F
:1058B000089580918000877FF9CF84B58F7702C0EB
:1058C00084B58F7D84BD08958091B0008F7703C02B
:1058D0008091B0008F7D8093B000089580919000FA
:1058E0008F7707C0809190008F7D03C080919000DA
:1058F000877F8093900008958091A0008F7707C0E4
:105900008091A0008F7D03C08091A000877F80934D
:10591000A0000895809120018F7707C08091200119
:105920008F7D03C080912001877F8093200108959F
:10593000CF93DF9390E0FC01E55BFD4F2491FC01E8
:10594000EF56FD4F8491882361F190E0880F991FF5
:10595000FC01E55FFC4FC591D491FC01EF50FD4F78
:10596000A591B491611109C09FB7F89488812095E1
:1059700082238883EC912E230BC0623061F49FB7A1
:10598000F8943881822F809583238883EC912E2B85
:105990002C939FBF06C08FB7F894E8812E2B2883E5
:1059A0008FBFDF91CF9108951F93CF93DF93282F5F
:1059B00030E0F901EB5FFD4F8491F901E55BFD4FAC
:1059C000D491F901EF56FD4FC491CC23C1F0162FAD
:1059D000811158DFEC2FF0E0EE0FFF1FEF50FD4F6D
:1059E000A591B4918FB7F894111105C09C91ED2F3A
:1059F000E095E92302C0EC91ED2BEC938FBFDF9192
:105A0000CF911F910895CF93DF93282F30E0F901B4
:105A1000EB5FFD4F8491F901E55BFD4FD491F901F6
:105A2000EF56FD4FC491CC2389F081112BDFEC2F71
:105A3000F0E0EE0FFF1FE952FD4FA591B491EC91FC
:105A4000ED2381E090E021F480E002C080E090E06E
:105A5000DF91CF91089508951F920F920FB60F9284
:105A600011240BB60F922F933F934F935F936F9335
:105A70007F938F939F93AF93BF93EF93FF93E091A7
:105A80000402F09105021995FF91EF91BF91AF913A
:105A90009F918F917F916F915F914F913F912F9146
:105AA0000F900BBE0F900FBE0F901F9018951F9276
:105AB0000F920FB60F9211240BB60F922F933F93B4
:105AC0004F935F936F937F938F939F93AF93BF9306
:105AD000EF93FF93E0910602F09107021995FF9171
:105AE000EF91BF91AF919F918F917F916F915F9156
:105AF0004F913F912F910F900BBE0F900FBE0F90C3
:105B00001F9018951F920F920FB60F9211240BB68B
:105B10000F922F933F934F935F936F937F938F9346
:105B20009F93AF93BF93EF93FF93E0910802F0919F
:105B300009021995FF91EF91BF91AF919F918F91BC
:105B40007F916F915F914F913F912F910F900BBE7D
:105B50000F900FBE0F901F9018951F920F920FB6C7
:105B60000F9211240BB60F922F933F934F935F9395
:105B70006F937F938F939F93AF93BF93EF93FF9315
:105B8000E0910A02F0910B021995FF91EF91BF91FC
:105B9000AF919F918F917F916F915F914F913F91C5
:105BA0002F910F900BBE0F900FBE0F901F90189566
:105BB0001F920F920FB60F9211240BB60F922F93D4
:105BC0003F934F935F936F937F938F939F93AF9385
:105BD000BF93EF93FF93E0910002F09101021995BA
:105BE000FF91EF91BF91AF919F918F917F916F91B5
:105BF0005F914F913F912F910F900BBE0F900FBE71
:105C00000F901F9018951F920F920FB60F921124AC
:105C10000BB60F922F933F934F935F936F937F93A6
:105C20008F939F93AF93BF93EF93FF93E091020203
:105C3000F09103021995FF91EF91BF91AF919F9160
:105C40008F917F916F915F914F913F912F910F9025
:105C50000BBE0F900FBE0F901F9018951F920F92C2
:105C60000FB60F9211240BB60F922F933F934F93C1
:105C70005F936F937F938F939F93AF93BF93EF93B4
:105C8000FF93E0910C02F0910D021995FF91EF91B5
:105C9000BF91AF919F918F917F916F915F914F9144
:105CA0003F912F910F900BBE0F900FBE0F901F9042
:105CB00018951F920F920FB60F9211240BB60F92E8
:105CC0002F933F934F935F936F937F938F939F9304
:105CD000AF93BF93EF93FF93E0910E02F0910F0209
:105CE0001995FF91EF91BF91AF919F918F917F9106
:105CF0006F915F914F913F912F910F900BBE0F903D
:105D00000FBE0F901F90189508951F93CF93DF93A8
:105D1000EC011D821C821F821E82198681E0888709
:105D200082E28A871F861E86FE01B396CE01C19647
:105D30002FEF2193E817F907E1F711E018A3CE013F
:105D4000E1D51F8B188E198E80E48A8F1B8E83E518
:105D500092E39AAB89ABDF91CF911F910895DB015C
:105D6000ED91FC911994EF92FF921F93CF93DF93E3
:105D70001F921F92CDB7DEB77C01DC01D196ED9169
:105D8000FC91D29782E069837A83199520E030E014
:105D90004AE069817A81C701E2DF182FD701D196E5
:105DA000ED91FC91D29783E01995D701D196ED91B1
:105DB000FC91D29780E01995812F0F900F90DF9181
:105DC000CF911F91FF90EF9008950F931F93CF9362
:105DD000DF93EC018B01E9A9FAA982E01995E9A901
:105DE000FAA981E0199520E030E044E1B801CE0144
:105DF000B6DF9E012D5C3F4F47E1B801CE01AFDF1A
:105E0000E9A9FAA980E0DF91CF911F910F91199430
:105E1000EF92FF921F93CF93DF93EC017B01E9A9EF
:105E2000FAA982E01995E9A9FAA981E0199520E07B
:105E300030E045E1B701CE0192DF182F882339F019
:105E40009E012D5C3F4F47E1B701CE0188DFE9A9F4
:105E5000FAA980E01995812FDF91CF911F91FF90D2
:105E6000EF900895FC01448F258F9C01245E3F4FE5
:105E700042E375CFCF93DF931F92CDB7DEB79E017C
:105E80002F5F3F4F46E46BDF89810F90DF91CF9109
:105E90000895CF93DF931F92CDB7DEB79E012F5F9A
:105EA0003F4F47E45CDF89810F90DF91CF910895E8
:105EB00020E030E048E453CFCF93DF93EC016A81D8
:105EC0007B81D8DF88836A817B81CE01E2DF898391
:105ED0006A817B81CE01ECDF8B879E012D5C3F4F79
:105EE0006A817B8147E1CE01DF91CF9138CFCF939B
:105EF000DF93EC016A817B8136DF882319F0CE01C4
:105F0000DBDF81E0DF91CF9108958F929F92AF9276
:105F1000BF92CF92EF920F93CF93DF931F921F9276
:105F2000CDB7DEB74C015B012A834983EEDEF40175
:105F3000B382A282498147A32A8120A705A3E4A2B4
:105F4000C3A2C4010F900F90DF91CF910F91EF90FA
:105F5000CF90BF90AF909F908F90C9CFFC0162818E
:105F6000738133CFCF93DF93EC01EE85FF853097BC
:105F700009F019956A817B81CE01DF91CF9148CFDD
:105F8000362F242FFC0162817381432F6BCF0F9337
:105F9000FC0182819381648F458F278F068F9F013B
:105FA000245E3F4F4BE3BC01CF010F91D8CEFC01E3
:105FB00060A30895BF92CF92DF92EF92FF920F936A
:105FC0001F93CF93DF936C01D62FB42EC22F78018D
:105FD000CC2369F0F701049120E04B2D6D2FC60111
:105FE000D6DFFFEFEF1AFF0AC150D85FF1CFDF9184
:105FF000CF911F910F91FF90EF90DF90CF90BF90C6
:1060000008958F929F92AF92BF92CF92DF92EF92BC
:10601000FF920F931F93CF93DF935C01C62EC42F83
:10602000D22ED02F220F220F220F1ED0882379F0DC
:10603000DC0F8D2C912CCD1751F087012D2D4C2F7D
:106040006C2DC501B7DFE80CF91CCF5FF4CFDF91F1
:10605000CF911F910F91FF90EF90DF90CF90BF9065
:10606000AF909F908F9008950F93FC010150040F03
:1060700084A996A9941718F0081728F402C00817E5
:1060800050F0041740F42150260F83A995A99617C4
:1060900020F4281720F480E007C0281720F481E0BE
:1060A000261710F0F8CF81E00F91089581E0089550
:1060B0002EE93FE0009729F0F9013197F1F70197B8
:1060C000F9CF0895FC01128280818150838314826C
:1060D0000895FC0180819281980F9283218192170B
:1060E00060F494819F5F94839381890F821710F0ED
:1060F0008FEF820F838381E0089580E00895FC0193
:1061000091E08381861708F490E031E0461708F0AB
:1061100030E0832F892B21E05281451708F420E0DD
:106120002823832F8923822B0895DC01FB01108211
:1061300012968C911297818315968C9115978150A8
:10614000828313968C9183830895FB01418123817F
:10615000213029F0233031F468EF640F04C0642F3C
:10616000485F01C0642FCBCFDC0115962C911597A9
:106170001696ED91FC911797CF01820F911D820F1A
:10618000911D1192E817F907E1F70895FC01A68126
:10619000B7818281481B8581483018F0A80FB11D56
:1061A0004770382F369536953695562F577080E8BC
:1061B00090E002C0959587955A95E2F7439F402D50
:1061C0001124669566956695E62FF0E0E40FF11DC3
:1061D000EA0FFB1F3081222311F0832B02C0809530
:1061E000832380830895FB014181DC0112962C9169
:1061F0001297421760F013962C911397241738F0DA
:10620000608115962C91621710F42481BFCF0895F8
:10621000CF92DF92FF920F931F93CF93DF936C0186
:10622000EB01FA809B81913051F030F0923049F0CF
:10623000933051F41FEF09C010E001E007C011E0F6
:1062400004C010E00FEF02C010E000E0F7FE03C052
:10625000BE01C601C8DF9881900F98839981910F84
:106260009983FF0C99F7DF91CF911F910F91FF90C8
:10627000DF90CF9008950F931F93CF93DF93890101
:10628000FB01C281D3814233D9F058F44531E1F0AA
:10629000473109F1443141F5CE0166DFCE0112DF0D
:1062A00023C04634E1F04734E1F04B33E9F4B9015F
:1062B000CE014BDF8823C1F0B801CE01A9DF14C0A5
:1062C000B901CE0190DF10C0CE0103DF882369F051
:1062D000CE014ADF09C0B901CE0127DF05C08D819B
:1062E00001C08981F801808381E0DF91CF911F9106
:1062F0000F910895CF92DF92EF92FF920F931F9329
:10630000CF93DF937C01D62FD42EC22F122FC62E0F
:10631000C20E6C2D611B183038F00FEF20E04D2DB0
:10632000C70135DE1850F5CF6C2F687F6D0F2C2F0D
:10633000277071F097E029272F5F27700FEF10E08B
:1063400001C0000F2A95EAF720E04D2DC7011FDE9E
:10635000DF91CF911F910F91FF90EF90DF90CF9041
:106360000895CF92DF92EF92FF920F931F93CF93F6
:10637000DF937C01D62ED42FC22F122FC42EC20E33
:106380004C2D411B183038F00FEF21E06D2DC70167
:10639000FEDD1850F5CF4C2F487F4D0F2C2F277066
:1063A00071F097E029272F5F27700FEF10E001C0F1
:1063B000000F2A95EAF721E06D2DC701E8DDDF9196
:1063C000CF911F910F91FF90EF90DF90CF900895A4
:1063D000DF92EF92FF920F931F93CF93DF937C0195
:1063E000162FC42FD22ED02F3FDE8823F9F02D2D6B
:1063F0004C2F612FC7017EDF2D2F4C2F612FC7013E
:10640000B0DF6FEF6D0D610F2D2F4C2FC701A9DF8E
:106410004FEF4D0F4C0F2D2D612FC701DF91CF9105
:106420001F910F91FF90EF90DF9064CFDF91CF919C
:106430001F910F91FF90EF90DF900895EF92FF92E0
:106440000F931F93CF93DF937C01D62F122FC42F6E
:10645000040F212F4C2F6D2FC7014CDFCF5F0C1382
:10646000F8CFDF91CF911F910F91FF90EF9008959A
:10647000DF92EF92FF920F931F93CF93DF93EC0184
:10648000162FF42EE22EF0DD882329F02E2D4F2D2D
:10649000612FCE01D3DFDF91CF911F910F91FF903C
:1064A000EF90DF9008950895FC01E60FF11D8491AF
:1064B00090E0982F88273196E4918E0F911D0895D2
:1064C000FC0184910895FCDF882321F0823011F0D3
:1064D00083E0089586E0089580E00895FC018081BE
:1064E000089566E0E1CF68E0DFCF0A96FC01849171
:1064F00008950B96FC0184910895DC011496ED91AA
:10650000FC911597319684910895BF92CF92DF92B6
:10651000EF92FF920F931F93CF93DF938C01E62EA0
:10652000DC011496CD91DC911597CE01C9DFF82ED0
:10653000F80184819581C7DFC82EF1E0FF1203C006
:106540002FE0B22E02C0BB24BA94D80114968D91CC
:106550009C911597CADFF82EF80184819581C9DFD7
:10656000D82ED80114968D919C911597BCDFB0E67A
:10657000BE1538F4009729F0C80FD91F91E6F92EFF
:106580000FC0F80184819581ACDFF0E4FE1538F48A
:10659000009729F0C80FD91F81E4F82E01C0619639
:1065A000DE1490F4D80150961C92509753961C928A
:1065B000539754961C92549751961C925197529609
:1065C0001C9280E090E066C0DF1460F38C2D90E0B8
:1065D000FE0124912F3F11F4219657C0FE104CC0AC
:1065E000D80114968D919C9115976ADF9E012F5FBB
:1065F0003F4FFE01882311F08230E1F48491D801ED
:1066000053968C935397F901249154962C93549755
:10661000FE013396E4915096EC935097FE01349628
:10662000E4915196EC935197FE013596E491529680
:10663000EC9320C08491982F9F709250D80152966D
:106640009C93529782958F7051968C935197F90134
:106650002491822F8F7054968C93549722952F708B
:1066600053962C935397FE013296E491E295EF7086
:106670005096EC93CE010EC0FE013296E491EB21D0
:106680009C012E0F311DC20FD31FFD1409F48ACFB8
:10669000F3949ECFDF91CF911F910F91FF90EF90D8
:1066A000DF90CF90BF9008954F925F926F927F924C
:1066B0009F92AF92BF92CF92DF92EF92FF920F9391
:1066C0001F93CF93DF931F92CDB7DEB72C01C62E59
:1066D000942E622F1ADF7C01892B09F43AC0F20153
:1066E00084819581F0DEB82EF201138904898189B5
:1066F000C80E8289981AD92CD01A212F4D2D6C2DB5
:10670000C201B2DC882311F1EB0CF11C195F169564
:1067100016951695612E712CD914C1F03C2D570198
:106720008A2D8E19811770F4F501049120E04D2D0A
:10673000632FC20139832BDCFFEFAF1ABF0A398107
:10674000385FEECFE60CF71CD394E6CFF2018089D8
:1067500001C080E00F90DF91CF911F910F91FF90CA
:10676000EF90DF90CF90BF90AF909F907F906F9011
:106770005F904F9008950F931F93CF93DF9300D0B6
:10678000CDB7DEB78C01DC015596ED91FC915697A3
:106790002B834A83698319954A81480F2B8169812C
:1067A000C8010F900F900F90DF91CF911F910F9123
:1067B0007BCFAF92BF92DF92EF92FF920F931F9326
:1067C000CF93DF931F921F92CDB7DEB77C01D62EF9
:1067D000042FDC015596ED91FC91569729833A835D
:1067E0001995080F2981A22E3A81B32E10E0F501E8
:1067F00021915F01222339F0402F6D2DC70154DF15
:10680000D80E180FF4CF812F0F900F90DF91CF91FA
:106810001F910F91FF90EF90DF90BF90AF90089580
:10682000DF92EF92FF920F931F93CF93DF937C0140
:10683000D62FD42E8901DC015596ED91FC91569707
:106840001995D80EC0E0F8012491222349F04D2D6E
:106850006D2FC70129DFD80FC80F0F5F1F4FF3CF70
:106860008C2FDF91CF911F910F91FF90EF90DF90D0
:106870000895DC0114962D913C9115972115310551
:1068800009F43FC057968C915797F901811108C0C0
:106890003596E4915896EC935897F9013C9611C0BF
:1068A000813041F43F96E4915896EC935897F90162
:1068B000709607C03D96E4915896EC935897F9016D
:1068C0003E96E4915996EC93599758968C91589727
:1068D000082E000C990B59962C915997821B9109FF
:1068E00027FD93955A962C915A97203441F0829F18
:1068F000C001112426E0969587952A95E1F75B96CD
:106900008C9308952CE632E3FC01368B258B089599
:10691000CF92DF92EF92FF920F931F93CF93DF936B
:106920008C017B016A01CB01FA011995D82F8823CC
:1069300011F1682FC801E9DDF801C189C195FFEFA8
:10694000EF1AFF0AC701F6011995F801882351F0E3
:106950008089C80FC701F6011995D82F682FC80183
:10696000D4DDEDCFD03221F091898389890F01C028
:1069700080898C0F01C080E0DF91CF911F910F9132
:10698000FF90EF90DF90CF9008954EE652E3C0CF96
:10699000CF93DF93FC01248135812617370741F01F
:1069A000EC017583648365DF8CE692E39E8B8D8BAF
:1069B000DF91CF9108954F925F926F927F92AF9245
:1069C000BF92CF92DF92EF92FF920F931F93CF93DC
:1069D000DF93CDB7DEB729013A019B01AC01241941
:1069E0003509460957098A899B89AC89BD89BC014B
:1069F000CD016A197B098C099D090F948730A80184
:106A0000970124193509460957090F94EB30CA013B
:106A1000B9016A0D7B1D8C1D9D1DDF91CF911F91CA
:106A20000F91FF90EF90DF90CF90BF90AF907F904D
:106A30006F905F904F90089580E090E008950895E2
:106A4000CF92DF92EF92FF920F931F93CF93DF933A
:106A50006C017A018B01C0E0D0E0CE15DF0589F032
:106A6000D8016D918D01D601ED91FC910190F081DD
:106A7000E02DC6011995892B11F47E0102C02196E3
:106A8000ECCFC701DF91CF911F910F91FF90EF9055
:106A9000DF90CF900895DC01ED91FC910190F081A1
:106AA000E02D1994CF92EF920F93FC0113AE14AE28
:106AB00015AE04962ADA0F91EF90CF9008950895BD
:106AC0000E94192BFCDF0F94F12BC0E0D0E00F9453
:106AD0007E2C2097E1F30E940000F9CFE9E2F4E078
:106AE00083AF64AF0895EF92FF920F931F93CF93FC
:106AF000DF937A016F3F71058105910509F048F434
:106B000089E294E0C8DF8DE294E0F7DC282F30E0E2
:106B100014C0C0916404D09165044D2F50E0EC2F57
:106B2000F0E08B019C01BF018DE294E000D6C80F1C
:106B3000C0936404D09365049C01C901DF91CF9197
:106B40001F910F91FF90EF900895EF92FF920F9396
:106B50001F93CF93DF938B01C9E2D4E0FBACECAC85
:106B60004E2D50E06F2D70E09C018DE294E035D603
:106B7000F80EFBAEECAEDF91CF911F910F91FF901D
:106B8000EF900895EF92FF920F931F93CF93DF93AF
:106B90008B01C9E2D4E0FBACECAC4E2D50E06F2D84
:106BA00070E09C018DE294E062D6F80EFBAEECAE94
:106BB000DF91CF911F910F91FF90EF9008956FEFAC
:106BC0007FEFC3CF4FEF5FEF8ECFCF938AEE95E08D
:106BD0000E94EC66C82F60E870E08AEE95E0B5DFB1
:106BE000C63138F460E270E080E090E0EBDFCF5F28
:106BF000F7CFCF9108954F925F926F927F928F92CD
:106C00009F92AF92BF92CF92DF92EF92FF920F933B
:106C10001F93CF93DF93CDB7DEB72D970FB6F894C0
:106C2000DEBF0FBECDBF8091E005882309F48AC086
:106C30006091D20B7091D30B072E000C880B990B2F
:106C40000F94212E11E02091D60B3091D70B40915B
:106C5000D80B5091D90B0F94822F18160CF010E01E
:106C60006091C80B7091C90B072E000C880B990B13
:106C70000F94212E2091CC0B3091CD0B4091CE0B57
:106C80005091CF0B0F94822F18160CF410681093AC
:106C90001B04C0908A0CD0908B0CE0908C0CF09070
:106CA0008D0C20E030E0A901C701B6010F947F2DC3
:106CB00087FD05C020E030E040E05FE304C020E055
:106CC00030E040E05FEBC701B6010F94A62C0F94B3
:106CD000EE2DCB010E94D884BC0186E194E00F9494
:106CE000A335C0908E0CD0908F0CE090900CF0905B
:106CF000910C20E030E0A901C701B6010F947F2D6F
:106D000087FD05C020E030E040E05FE304C020E004
:106D100030E040E05FEBC701B6010F94A62C0F9462
:106D2000EE2DCB010E94D884BC0181E194E00F9448
:106D3000A33582E99CE00E940989BC0189E094E0C6
:106D40000F94A3350E94DE67182F81E050D6209162
:106D50001B0427FF03C048E00CE002C042E102E050
:106D60008091610490E0449774F4809163048417E7
:106D700050F027FD34C189E496E17C0123E060E511
:106D80008DE294E03ED9809161048431B0F4809129
:106D90006304823090F0112309F424C18091D10B57
:106DA000882309F41FC189EB95E17C0102E123E00E
:106DB00042E068E68DE294E024D9809161048C3150
:106DC000D0F590911B048090D60B9090D70BA0909B
:106DD000D80BB090D90BC090D20BD090D30B84318C
:106DE00028F480916304883008F033C280916104F4
:106DF000883008F40EC2809161048C3108F410C20E
:106E00008090CC0B9090CD0BA090CE0BB090CF0B80
:106E10008091C80B9091C90B20916104283008F42F
:106E200005C2809161048C3108F407C2809161042D
:106E30008C3108F408C28091500883FF26C08091ED
:106E40008006882311F1809161048433F0F48091ED
:106E500063048A32D0F007E028E04AE26AE28DE279
:106E600094E006DB05E022E04CE262E38DE294E090
:106E7000FFDA04E02AE041E36AE28DE294E0A8DA76
:106E80004BE262E38DE294E07BD88091610485332C
:106E900028F480916304813308F0A7C00E9416682B
:106EA000823048F090916104943328F49091630407
:106EB000923308F0A2C0809161048F3208F05EC066
:106EC00080916304883208F459C00F9400282B0184
:106ED0003C018CE3C82ED12CE12CF12CC301B20172
:106EE000A70196010F94C930CA01B901A701960103
:106EF0000F94C930CA01062FD72E5901AE014F5F3A
:106F00005F4F7A0150E8451651E5550651E0650698
:106F1000710408F48CC0B90128E130E040E050E091
:106F20000F94C93029013A01DF920F93C50168E13E
:106F300070E00F94A2309F938F935F924F928BEAF1
:106F400095E19F938F93FF92EF920F94D2350FB6F6
:106F5000F894DEBF0FBECDBF5AE045165104610460
:106F6000710408F08EC098E0892F880F980F892F40
:106F700081956FE2855AB2DDC70121DE80916104FF
:106F80008632A0F4809163048E3180F008E020E81E
:106F90004EE160E08DE294E06BDA8091610486322C
:106FA00028F4809163048F3108F06DC080916104F2
:106FB000823328F4809163048B3208F00EC18091F3
:106FC0006104813408F03AC280916304873308F485
:106FD00035C26EE380E082DD812FF7DD2FC285E2CE
:106FE00096E1CBCE8FEE95E1E0CE04E02AE441E3DA
:106FF00066E38DE294E0ECD951CFF8E48F9FB001C5
:107000001124072E000C880B990B0F94212E2AE0D7
:1070100037ED43E25CE30F94BD2F0F94F32D262F41
:1070200002E042E367E38DE294E022DA44CF84E6B3
:10703000A816B10498F4DF920F933F932F9381EA3F
:1070400095E19F938F93FF92EF920F94D2350FB6F5
:10705000F894DEBF0FBECDBF95E086CFDF920F93D1
:107060003F932F9389E995E19F938F93FF92EF923E
:107070000F94D2350FB6F894DEBF0FBECDBF96E0A9
:1070800073CF99E071CF60E08DE294E00E94D72F3A
:1070900065E283E023DD68E570E080E090E092DD6A
:1070A00065E28BE01BDD112321F086E194E087DDB2
:1070B00024C080919C0C80FD17C036E1E32E34E0A3
:1070C000F32EF70161917F016623B9F06F3234F43A
:1070D000062E000C770B880B990B04C06FE370E051
:1070E00080E090E06FDDEDCF80919B0C80FDDDCFE7
:1070F0006FEF7FEF8DE895E145DD65E288E2EEDC3C
:1071000069E570E080E090E05DDD65E280E3E6DC6B
:10711000112321F081E194E052DD24C080919C0C88
:1071200081FD17C021E1E22E24E0F22EF7016191EA
:107130007F016623B9F06F3234F4062E000C770B12
:10714000880B990B04C06FE370E080E090E03ADDBB
:10715000EDCF80919B0C81FDDDCF6FEF7FEF8DE850
:1071600095E110DD65E28DE4B9DC6AE570E080E070
:1071700090E028DD65E285E5B1DC112321F089E0AE
:1071800094E01DDD24C080919C0C82FD17C099E025
:10719000E92E94E0F92EF70161917F016623B9F0A1
:1071A0006F3234F4062E000C770B880B990B04C059
:1071B0006FE370E080E090E005DDEDCF80919B0C07
:1071C00082FDDDCF6FEF7FEF82E995E1DBDC61E0EF
:1071D0008DE294E00E94D72FE9CE83E008D462E3E9
:1071E00083E07CDC66E070E080E090E0EBDC81E056
:1071F000FED362E38CE072DC80915A0290915B02D4
:107200000E94A284DCDC65E270E080E090E0DADCE1
:10721000D6CE80917C0B11112DC08111ECCD2AC0EE
:1072200080916304853108F059C0EACD2091AC0B00
:10723000111184C02111F5CD81C080916304853185
:1072400008F0B0C0F3CD80916304853108F0DAC056
:10725000F2CD90FD03C08FE496E102C087E696E18F
:107260007C010CE022E048E068E08DE294E00E94BE
:107270000130BCCDB601DD0C880B990B0F94212E8B
:1072800020E030E040E05FE30F94A62C0F94EE2D59
:10729000CB010E94A2847C01FC0180818032E1F458
:1072A000F7018181803211F401E001C002E0902FEA
:1072B000990F900F892F819567E0815F0FDC83E044
:1072C00090E0801B91098E0D9F1D79DC69E070E0D4
:1072D00080E090E077DC8FCD03E0E9CF20E030E084
:1072E00040E05FE3C501B4010F94A62C0F94EE2D8E
:1072F000CB010E94A2847C01FC0180818032E1F4F8
:10730000F7018181803211F401E001C002E0902F89
:10731000990F900F892F81956CE1815FDFDB83E00E
:1073200090E0801B91098E0D9F1D49DC69E070E0A3
:1073300080E090E047DC64CD03E0E9CFBC01990F29
:10734000880B990B0F94212E20E030E040E05FE3A2
:107350000F94A62C0F94EE2DCB010E94A2847C01E9
:10736000FC0180818032E1F4F7018181803211F4E7
:1073700001E001C002E0902F990F900F892F8195B5
:1073800067E0845AABDB83E090E0801B91098E0DAF
:107390009F1D15DC69E070E080E090E013DC41CDDA
:1073A00003E0E9CF20E030E040E05FE3C501B40155
:1073B0000F94A62C0F94EE2DCB010E94A2847C0189
:1073C000FC0180818032E1F4F7018181803211F487
:1073D00001E001C002E0902F990F900F892F819555
:1073E0006CE1845A7BDB83E090E0801B91098E0D79
:1073F0009F1DE5DB69E070E080E090E0E3DB16CD07
:1074000003E0E9CF0091D10B002309F414CD6CE126
:1074100087E664DBF4E60F9FC001112481589F4F7B
:107420006FEF70E00F94B630CB010E94A284C7DBEF
:1074300065E270E080E090E0C5DBFDCC2D960FB6F4
:10744000F894DEBF0FBECDBFDF91CF911F910F919A
:10745000FF90EF90DF90CF90BF90AF909F908F9074
:107460007F906F905F904F9008950F931F93CF93ED
:10747000DF93CDB7DEB728970FB6F894DEBF0FBE07
:10748000CDBF8A0123E0660F771F2A95E1F7680FC9
:10749000791F48E050E0CE0101960F94063529810E
:1074A0003A81F801808191812817390790F082177D
:1074B000930760F09C818281981758F081E090E0FA
:1074C0003B812381231738F080E005C081E090E004
:1074D00002C08FEF9FEF28960FB6F894DEBF0FBE65
:1074E000CDBFDF91CF911F910F910895EF92FF9241
:1074F0000F931F93CF93DF93EC018B017A018A8561
:107500009B858617970729F08881998141DA1B8727
:107510000A8788859985019681F00E811F81B701C0
:107520008881998132DA080F111D88859985801725
:10753000910718F481E090E010C06E818A81680F95
:1075400097014C818881998134D92E813F81280F00
:10755000311D3F832E8380E090E0DF91CF911F911A
:107560000F91FF90EF9008954F925F926F927F92EC
:107570008F929F92AF92BF92CF92DF92EF92FF9243
:107580000F931F93CF93DF93CDB7DEB72D970FB631
:10759000F894DEBF0FBECDBF6C012A013B0149014B
:1075A00058011B861C86CE0101967C0188E0F701FC
:1075B00011928A95E9F7DB01CA0127E0B695A795F4
:1075C000979587952A95D1F79A838983F42FFF772A
:1075D000FD878F2F80588B838C831A8619864F3FA7
:1075E00051056105710509F018F460E070E026C0EE
:1075F00060911E0470911F048E01075F1F4F970159
:1076000045E35AE380911C0490911D040E943D655E
:1076100097FDEBCF69857A8583E0660F771F8A95A2
:10762000E1F780911C0490911D04680F791F48E0D8
:1076300050E0C7010F9406356F817885611571059B
:1076400019F44B86B60106C0C616D70619F08D850B
:1076500080688B87AE01455F5F4FC401F5011995C6
:107660002D960FB6F894DEBF0FBECDBFDF91CF9140
:107670001F910F91FF90EF90DF90CF90BF90AF9050
:107680009F908F907F906F905F904F9008956F9232
:107690007F928F929F92AF92BF92CF92DF92EF92A2
:1076A000FF920F931F93CF93DF9300D01F92CDB71C
:1076B000DEB76C017B013A015901480119821A8237
:1076C0001B821C82AE014F5F5F4FB301C7010E9456
:1076D0009D657C0149815A816B817C8141155105F1
:1076E0006105710529F084019501C6013DDFE6CFF2
:1076F0000F900F900F900F90DF91CF911F910F91EE
:10770000FF90EF90DF90CF90BF90AF909F908F90C1
:107710007F906F90089521E020932004ECE1F4E045
:10772000918380837383628380E090E008957F92E9
:10773000AF92BF92CF92DF92EF92FF920F931F937F
:10774000CF93DF93CDB7DEB72C970FB6F894DEBF9B
:107750000FBECDBF6C01762EF72F842FE52FB90118
:10776000A801D6011496AD90BC9015979091200475
:10777000911109C02FEB36E1482F672DC60150D873
:1077800080E090E018C0DA82C9827B82FC838D831E
:10779000EE8318861F82FA86E9861C861B8606E71A
:1077A0001AE39E012F5F3F4FC501DEDEB501C60122
:1077B000EFD88F8198852C960FB6F894DEBF0FBE58
:1077C000CDBFDF91CF911F910F91FF90EF90DF9090
:1077D000CF90BF90AF907F900895CF92DF92EF92BD
:1077E000FF920F931F93CF93DF93CDB7DEB72C9704
:1077F0000FB6F894DEBF0FBECDBF7C01C901F70103
:10780000C480D58020912004211107C02FE936E1E2
:10781000C70106D880E090E01BC0FA82E9826B8342
:107820007C834D835E8318861F821A8709871C8696
:107830001B8606E71AE39E012F5F3F4F47E355E69D
:10784000BC01C60124DFB601C701A2D88F8198858B
:107850002C960FB6F894DEBF0FBECDBFDF91CF914F
:107860001F910F91FF90EF90DF90CF900895CF92EE
:10787000DF92EF92FF920F931F93CF93DF93CDB7D9
:10788000DEB72C970FB6F894DEBF0FBECDBF7C01DC
:10789000C901F701C480D58020912004211108C0BE
:1078A0002FE736E1C7010E94103480E090E01BC052
:1078B000FA82E9826B837C834D835E8318861F8204
:1078C0001A8709871C861B8606E71AE39E012F5F2D
:1078D0003F4F4AE355E6BC01C601D9DEB601C701F8
:1078E00057D88F8198852C960FB6F894DEBF0FBEBF
:1078F000CDBFDF91CF911F910F91FF90EF90DF905F
:10790000CF900895CF93DF93EC01262F4CAD6BAD54
:1079100004960E94BB332BAD082E000C990B820FEE
:10792000911D8BAF81E090E0DF91CF9108950F938F
:107930009CE0899F802D112421E0280F20932804AA
:10794000845F8093270490E002964091610450E0A8
:107950008417950714F480E033C0822F90E02091C3
:10796000630430E082179307B4F76623A9F061E05F
:107970008DE294E00E94D72F409128044E5F0BE0E7
:1079800020E860E08DE294E00E94383260E08DE211
:1079900094E00E94D72F05C061E08DE294E00E9440
:1079A000D72F60912704809161046817A0F290910D
:1079B000280480916304891770F280E08FD881E0F9
:1079C0000F910895CF93DF93FC0185ADEF012496CD
:1079D000811105C081E085AFCE010E94772FCE01D5
:1079E000DF91CF910C94AE2F6FEF7FEFCBC8482F74
:1079F00050E020912604022E000C330B421753074F
:107A000081F080932604813031F46AE97FE18DE2D0
:107A100094E00C94C8346AEA77E18DE294E00C9427
:107A2000C8340895EF92FF920F9389E294E0CADF81
:107A30008CE5E82E8DE1F82E00E428E040E060E0DF
:107A40008DE294E00E94013065E273E08DE294E003
:107A50000E94C83421E233E041E169E38DE294E021
:107A60000E94D93365E97BE08DE294E00E94C8343E
:107A700026E233E04CE16AE38DE294E00E94D933E0
:107A800060EF7EE08DE294E00E94C83422E333E0B0
:107A900049E26BE38DE294E00E94D93360EF7EE02F
:107AA0008DE294E00E94C8342EE333E04EE36DE3B0
:107AB0008DE294E00E94D93320E433E04EE362E4A7
:107AC0008DE294E00E94D9338DE294E00E94B22FBF
:107AD0008111AECF64EC79E080E090E00E943884C0
:107AE0006AEA77E18DE294E00F91FF90EF900C94B9
:107AF000C83461E08CE59DE195DF64EC79E080E0DD
:107B000090E00C943884CF92DF92EF92FF920F9323
:107B10001F93CF93DF93EDDFC0912D0400912E04CE
:107B2000D0E0BE016853710977FF02C06F5F7F4FDD
:107B300075956795D62E89E294E044DFCE01C09713
:107B400096958795182FC257D109D695C7954EEEB1
:107B5000C42EC00EDAEFD00F87EDE82E8CE1F82EA0
:107B600003E127E04CE06D2D8DE294E00E940130AE
:107B700083E03DDF20E433E04C2D612F8DE294E083
:107B80000E94D93329E433E04D2F6C2F8DE294E02D
:107B90000E94D9338DE294E00E94B22F8111DCCF94
:107BA00064EC79E080E090E0DF91CF911F910F913C
:107BB000FF90EF90DF90CF900C94388460E070E0FD
:107BC0008AE99FE1A8CD1F93CF93DF93C0912E0444
:107BD000C695C69589E294E0F5DEDC2FDD0F1D2FFA
:107BE0001C0F83E004DF6C2F80E00E946E358AEE6C
:107BF00095E00E94DF356D2F80E00E946E358CEE9F
:107C000096E1F2DE612F80E00E946E358FED96E105
:107C1000EBDE8DE294E00E94B22F8111E2CFDF9182
:107C2000CF911F9108950895CF939CE0899F802D57
:107C3000112421E0280F20932804845F80932704D7
:107C4000E82FF0E032964091610450E0E417F50728
:107C50000CF448C030E04091630450E0241735072D
:107C60000CF040C0C62F682F8EE30E946E3565E48D
:107C700070E080E090E00E94E23561E36C0F062E38
:107C8000000C770B880B990B0E94E23560E270E0E4
:107C900080E090E00E94E2356091D60B7091D70BA6
:107CA0008091D80B9091D90B0F94EE2DCB010E94AF
:107CB000A2840E94DF356FE270E080E090E00E94D5
:107CC000E2350E94DE67811104C080917C0B811136
:107CD00009C08091D20B9091D30B0E94A284CF91C6
:107CE0000C94DF35CF910895CF92DF92EF92FF92FF
:107CF0000F931F93CF93DF931F921F92CDB7DEB7E1
:107D00007B01622F498313DE4981882309F444C033
:107D1000442311F101151105F9F4C7010E940D6703
:107D200026E130E0281B310937FF02C02F5F3F4FAB
:107D30003595279530E82158822F830F87FD0DC098
:107D400060E270E080E090E02A8339830E94E235AF
:107D5000398131502A81F0CF30E8C32ED12CB601C1
:107D6000C7010E94C2357601E81AF90A011511050A
:107D700011F41E2D07C0FF24B701C8010E94A535CC
:107D80001E2D181B173040F060E270E080E090E09C
:107D90000E94E235181BF6CF0F900F90DF91CF9124
:107DA0001F910F91FF90EF90DF90CF9008950F9368
:107DB000CF93DF93982F862FEA01692FB8DD8823B0
:107DC00031F168E770E0CE010E94C235C8E7C81BF8
:107DD000C73040F060E270E080E090E00E94E23561
:107DE000C81BF6CF609127048AE70E946E35602F8A
:107DF000000F770B880B990B0E94E23560E270E070
:107E000080E090E0DF91CF910F910C94E235DF910B
:107E1000CF910F910895CF92DF92EF92FF920F933F
:107E20001F93CF93DF93982F862F6A017901692FD3
:107E30007EDD882309F447C0C701002321F00E949A
:107E40000D67182F03C00E94EC66182FC4E1D0E024
:107E5000C11BD1098C2F880FC80FCC0FD0E0BE01F9
:107E6000C6010E94C235C81B6AE370E080E090E062
:107E70000E94E235C73040F060E270E080E090E0C0
:107E80000E94E235C81BF6CF8AEF189F802D11247F
:107E90006091270480580E946E35C701002349F085
:107EA000DF91CF911F910F91FF90EF90DF90CF90D6
:107EB0009BCDDF91CF911F910F91FF90EF90DF90BD
:107EC000CF900C94DF35DF91CF911F910F91FF90F0
:107ED000EF90DF90CF900895BF92CF92DF92EF9214
:107EE000FF920F931F93CF93DF936C017B010E944E
:107EF0000D67C82FC7010E94EC6604E110E0081B63
:107F000011098C2F90E0BB24B394081719071CF0BB
:107F1000B12CC5E201C0CFE12C2F30E0A9014E5FAA
:107F20005F4F8091610490E04817590744F0295051
:107F300031098091630490E082179307BCF5D0E08B
:107F4000E114F104D9F16AE370E080E090E00E946E
:107F5000E235BB2081F0C45F80916104C81770F1E5
:107F60002C2F30E0295031098091630490E0821772
:107F700093071CF423C0DD2309F1802F880F800FA5
:107F80006C2F880F0E946E3560E270E080E090E018
:107F90000E94E235C701DF91CF911F910F91FF90B1
:107FA000EF90DF90CF90BF900C94DF356C2F80E086
:107FB0000E946E35C60118DDD1E0C2CFDF91CF91AE
:107FC0001F910F91FF90EF90DF90CF90BF90089599
:107FD000EF92FF920F93CF93DF93D82FC62F7901A3
:107FE000682F8C2FA4DC8823F1F0002331F062E0AD
:107FF00070E080E090E00E94E2352D2F4C2F65E18B
:10800000C7010E948F676EE770E00E94A535CEE73A
:10801000C81BC73040F060E270E080E090E00E9452
:10802000E235C81BF6CFDF91CF910F91FF90EF9013
:1080300008958F929F92AF92BF92CF92DF92EF926C
:10804000FF920F936B017C01809022049090230497
:10805000A0902404B0902504A50194010F947F2DD5
:10806000882301F120E030E0A901C701B6010F9497
:108070007F2D882351F0A5019401C701B6010F940B
:108080007F2D87FD04C081E003C080E001C08FEF39
:1080900080932104C0922204D0922304E09224040D
:1080A000F092250480916104813128F48091630469
:1080B000833008F048C080916104853128F48091B4
:1080C0006304843108F04FC0809161048F3308F05D
:1080D00057C0809163048F3208F452C08AE4E82EBE
:1080E00087E1F82E00E123E04FE265E08DE294E0C5
:1080F0000E9401309AE7E92E97E1F92E23E04FE242
:108100006AE58DE294E00E9401308091210440E311
:10811000481B20E3E22E27E1F22E0DE022E06EE67E
:108120008DE294E00E9401308091210441E3481BDC
:1081300036E1E32E37E1F32E22E069E18DE294E0AF
:108140000E9401301DC08091210444E0481B5BEF78
:10815000E52E56E1F52E0CE022E062E48DE294E09B
:108160000E940130A8CF43E1E42E47E1F42E01E064
:1081700023E044E16CE38DE294E00E940130A4CF5F
:108180000F91FF90EF90DF90CF90BF90AF909F90B6
:108190008F900895CF92EF920F93CF93DF93C9E220
:1081A000D4E01B821A8281E693E099838883CC24F1
:1081B000CA94EE24EA9402E522E143E160E172E030
:1081C000CE010E9452358DE693E099838883DF913A
:1081D000CF910F91EF90CF9008955A9887FD52C09C
:1081E0005B9800000000000000005A9A5A98282F5F
:1081F000220F86FD53C05B980000000000000000C5
:108200005A9A5A98922F990F26FD46C05B98000003
:108210000000000000005A9A5A98892F880F96FD96
:1082200039C05B9800000000000000005A9A5A987C
:10823000982F990F86FD2CC05B980000000000006D
:1082400000005A9A5A98892F880F96FD1FC05B9894
:1082500000000000000000005A9A5A98982F990FC9
:1082600086FD12C05B9800000000000000005A9AD2
:108270005A9896FD15C05B980000000000000000B1
:108280005A9A08955B9AADCF5B9AEDCF5B9AE0CF97
:108290005B9AD3CF5B9AC6CF5B9AB9CF5B9AACCFD0
:1082A0005B9AEACF2F923F925F927F929F92AF921A
:1082B000BF92CF92DF92EF92FF920F931F93CF93D3
:1082C000DF937C011B01942E69018AE0481709F4B1
:1082D0007BC0A5E14A134EC0DB011296ED91FC91E3
:1082E00013971281C681D7815D9A88E28A95000032
:1082F000E9F700EE010F80E1582E510E98E2792E39
:1083000088EF6BDF872D8A950000E9F7103208F0BF
:1083100046C0812F8077806860DF812F8295807FC3
:108320005CDF872D8A950000E9F780E856DF80E062
:1083300054DF872D8A950000E9F78AEF4EDF872DFD
:108340008A950000E9F75E01B0E1AB0EB11C8881AF
:10835000807F43DF89918295807F3FDFCA15DB05EF
:10836000B1F7872D8A950000E9F71F5F0F5F1511A0
:10837000C7CF5D989601492DB101C701DF91CF911B
:108380001F910F91FF90EF90DF90CF90BF90AF9033
:108390009F907F905F903F902F900C943B31802F67
:1083A000807780681ADF802F8295807F16DF872D87
:1083B0008A950000E9F780E810DF80E80EDF872D5E
:1083C0008A950000E9F7B9CF559A5D98539A5B9862
:1083D000529A5A9A5D9AC8E28C2F8A950000E9F762
:1083E00088E790E00E94583088EFF7DE8C2F8A955E
:1083F0000000E9F780E2F1DE80E0EFDE8C2F8A9565
:108400000000E9F780E0E9DE80E8E7DE8C2F8A955E
:108410000000E9F780E0E1DE80E1DFDE8C2F8A9565
:108420000000E9F78FE090E00E94583080E2D5DE4E
:1084300080E4D3DE8C2F8A950000E9F780E2CDDE60
:1084400080E6CBDECA950000E9F710E0D8E208E24A
:10845000812F80778068C1DE812F8295807FBDDE8D
:108460008D2F8A950000E9F780E8B7DE80E0B5DE61
:108470008D2F8A950000E9F78AEFAFDE8D2F8A9560
:108480000000E9F7C0E280E0A8DE80E0A6DE9D2FD4
:108490009A950000E9F7C150B1F788EF9EDE802F72
:1084A0008A950000E9F71F5F103209F0D1CF80E014
:1084B00094DE80EC92DE88E28A950000E9F75D9810
:1084C00059CF0E94357541E050E060E070E08111C5
:1084D00003C040E050E0BA014093DC055093DD0555
:1084E0006093DE057093DF051092B60581E08093FE
:1084F000900583E080931F020895CF92DF92EF9260
:10850000FF920F931F93CF93DF930E9432766C01FB
:1085100061E081E00E940D64C091B605D0E081E089
:10852000C81AD108C11117C080917F05811104C0FC
:108530000E94D96781119BC080911F02882359F046
:1085400081E090917F05911180E004E024E046EB0A
:1085500058E26D2F2CDC63E478E08AEC97E00E940F
:108560001B7C809143088F3201F18091500883FF7A
:108570001CC0C130C1F480917F05813021F40E947C
:10858000D96781117CC080911F02882361F081E04E
:1085900090917F05913009F080E000E22EE342EBFC
:1085A00058E26D2F04DC92E001C091E080911F023F
:1085B000882309F454C0760111E01C0F8FEFE816F0
:1085C000F80609F44CC0C91345C060E070E0C7016B
:1085D0000E945B729091500880917F0594FF22C0A9
:1085E0008C1354C00E94D967882309F44FC083E4D8
:1085F00098E00E94DF741092B60582E090E0A0E05F
:10860000B0E08093DC059093DD05A093DE05B09388
:10861000DF0581E0809390051092E10583E080936F
:108620001F0250C08C1304C00E94D96781113DC045
:1086300080911F02882361F081E090917F059C1357
:1086400080E000E025E136E146E958E26D2FC0DC2C
:10865000912F01C09F5F81E0E81AF108AFCFDF5F83
:10866000CF5FD53009F05ECF90937E052BC00E947E
:108670005D6380919005882309F45ECF23C021DFDC
:1086800080919005882309F47ECF1CC080911F0241
:108690008823F1F281E090917F059C1380E001E056
:1086A00025E136E144EA58E2D1CF83E498E00E9424
:1086B000E6700E9457630E949C6C8091900588230D
:1086C00009F4B6CFDF91CF911F910F91FF90EF90FA
:1086D000DF90CF900895CF93DF93EC01CB01BA01E7
:1086E0000F94212E20E030E048EC52E40F94BD2F8F
:1086F0000F94F32D688379838A839B83DF91CF91D5
:108700000895CF93DF93EC01CB01BA010F94212E92
:108710002AE037ED43E25CE30F94BD2F6883798351
:108720008A839B83DF91CF910895CF93DF93EC01F0
:10873000CB01BA010F94212E688379838A839B83AE
:10874000DF91CF910895CF93DF93EC01CB01BA0174
:108750000F94212E20E030E048EC52E40F94BD2F1E
:10876000688379838A839B83DF91CF910895CF9328
:10877000DF93EC01CB01BA010F94212E2AE037EDF3
:1087800043E25CE30F94BD2F688379838A839B83E4
:10879000DF91CF910895CF93DF93EC01CB01BA0124
:1087A0000F94212E2AE037ED43E25CE30F94BD2FB6
:1087B000688379838A839B83DF91CF9108956BE6E9
:1087C00073E48AEB94E40C94716361E873E484E2EB
:1087D00094E40C94716365E973E48EE994E40C9479
:1087E000716363EA73E481E494E40C94716367EB6E
:1087F00073E48EE594E40C9471636BEC73E487E0AE
:1088000094E40C9471630C9483E30C94CAE3CF93C7
:10881000DF9300D01F92CDB7DEB70F94212E2AE050
:1088200037ED43E25CE30F94BD2F69837A838B833A
:108830009C83CE0101960E9448880F900F900F9064
:108840000F90DF91CF910895CF93DF9300D01F92C7
:10885000CDB7DEB70F94212E2AE037ED43E25CE37B
:108860000F94BD2F69837A838B839C83CE010196FD
:108870000E9441850F900F900F900F90DF91CF9144
:108880000895CF93DF9300D01F92CDB7DEB70F943A
:10889000212E20E030E048EC52E40F94BD2F698394
:1088A0007A838B839C83CE0101960E94EF860F9082
:1088B0000F900F900F90DF91CF910895CF93DF939A
:1088C00000D01F92CDB7DEB70F94212E2AE037EDEE
:1088D00043E25CE30F94BD2F69837A838B839C838F
:1088E000CE0101960E94A7870F900F900F900F90D6
:1088F000DF91CF910895CF92DF92EF92FF926B01BB
:108900007C0120E030E0A9010F947F2D87FD05C098
:1089100020E030E040E05FE304C020E030E040E0F1
:108920005FEBC701B6010F94A62C0F94EE2DCB017F
:10893000FF90EF90DF90CF900C94A2840F94212EA3
:10894000DACFCF93DF9300D01F92CDB7DEB70F946D
:10895000F32D0F941F2E69837A838B839C83CE0122
:1089600001960E94EF860F900F900F900F90DF916D
:10897000CF9108950F94212E20E030E048EC52E48E
:108980000F94BD2FDECFCF93DF931F921F92CDB7F1
:10899000DEB789839A830E948C6240E050E0BA017E
:1089A00089819A810F900F90DF91CF910C9432635F
:1089B0000F931F93CF93DF9361E081E00E940D64DA
:1089C000C091B605D0E0C11119C080917F05811119
:1089D00004C00E94D9678111C5C080911F028823FD
:1089E00009F45DC081E090917F05911180E004E081
:1089F00024E047EF58E26D2FDAD951C0C130D1F4ED
:108A000080917F05813021F40E94D9678111B2C025
:108A100080911F02882309F442C081E090917F0574
:108A2000913009F080E003E02EE34EEE58E26D2F26
:108A3000BED935C0C230C9F480917F05823021F49F
:108A40000E94D96781119FC080911F02882339F14C
:108A500081E090917F05923009F080E003E02EE301
:108A600041EE58E26D2FA3D91AC0C330C1F48091F2
:108A70007F05833021F40E94D96781118DC08091D8
:108A80001F02882361F081E090917F05933009F007
:108A900080E003E02EE34CED58E26D2F88D90E9470
:108AA0001B6381111CC0C430E1F480917F058430C8
:108AB00021F40E94D967811178C080911F02882318
:108AC00009F47CC081E090917F05943009F080E04A
:108AD00003E02EE343ED58E26D2F69D96FC014E037
:108AE00001C015E0C1131AC080917F058C1304C02A
:108AF0000E94D967811164C080911F02882369F0A8
:108B000081E090917F059C1380E003E02EE344EC2C
:108B100058E26D2F4CD91C2F01C01C2F81E0810F12
:108B2000C81317C080917F058C1304C00E94D967B9
:108B300081114FC080911F02882359F081E09091EC
:108B40007F059C1380E003E02EE34BEB58E26D2F92
:108B50002ED9DF5FCF5FD53009F035CF1E5F109380
:108B60007E053FC00E945D6380919005882309F4D3
:108B700034CF37C08EE299E406DF809190058823D8
:108B800009F446CF2EC089EF9CE4FDDE809190056C
:108B9000882309F459CF25C086EF9AE4F4DE80914A
:108BA0009005882309F46BCF1CC087EC9FE4EBDEB3
:108BB00080919005882309F480CF13C015E0AECFD3
:108BC0008BE796E4E0DE80919005882309F494CF4A
:108BD00008C088EF97E4D7DE80919005882309F4D8
:108BE000A9CFDF91CF911F910F9108952F923F92BE
:108BF0004F925F926F927F928F929F92AF92BF92AD
:108C0000CF92DF92EF92FF920F931F93CF93DF9358
:108C1000CDB7DEB727970FB6F894DEBF0FBECDBF36
:108C20001C017F836E83E982FA820B831C839C2C58
:108C30008D2CAD82CA01B9010F941F2E2AE037EDA9
:108C400043E25CE30F94BD2F0F94EE2D2B013C010A
:108C5000EE81FF8160817181828193810F941F2E4B
:108C60002AE037ED43E25CE30F94BD2F0F94EE2D25
:108C70005B016C01A418B508C608D708C801B70184
:108C80000F941F2E2AE037ED43E25CE30F94BD2FD3
:108C90000F94EE2D7B018C01E418F50806091709E5
:108CA000FD81FF938F929F928FED882E83E4982E03
:108CB000A30192016E817F81C1010E94AE620F907B
:108CC0000F900F9027960FB6F894DEBF0FBECDBF62
:108CD000DF91CF911F910F91FF90EF90DF90CF9098
:108CE000BF90AF909F908F907F906F905F904F90CC
:108CF0003F902F900895AF92CF92DF92EF92FF9224
:108D00000F931F93CF93DF9361E081E00E940D6486
:108D1000D091B605C0E0D11119C080917F058111B5
:108D200004C00E94D967811191C080911F028823DD
:108D300009F483C081E090917F05911180E004E007
:108D400024E045EF5AE26C2F32D877C0D13031F5AC
:108D500080917F05813021F40E94D96781117EC006
:108D600080911F02882309F468C011E080917F057B
:108D7000813009F010E06091560C7091570C809191
:108D8000580C9091590C0F941F2EDBDD00E09C01D4
:108D90004FEE5AE26C2F812F3ED84FC0D23031F5C2
:108DA00080917F05823021F40E94D967811170C0C3
:108DB00080911F02882309F440C011E080917F0553
:108DC000823009F010E060915A0C70915B0C809138
:108DD0005C0C90915D0C0F941F2EB3DD00E09C01A4
:108DE0004BEE5AE26C2F812F16D827C0D33029F5CD
:108DF00080917F05833021F40E94D967811162C080
:108E000080911F028823C9F011E080917F05833093
:108E100009F010E060915E0C70915F0C8091600C25
:108E20009091610C0F941F2E8CDD00E09C0147EEA9
:108E30005AE26C2F812F0E940B3FCF5FDF5FC5305E
:108E400009F069CF84E080937E0555C00E945D6380
:108E500080919005882309F468CF4DC0A12C4BE682
:108E6000C42E43EBD42E10EDE12E17E0F12E00E0DE
:108E700010E024E630E040E050E066E57CE082EF80
:108E80009AE2B4DE80919005882309F469CF33C05B
:108E9000A12C2BE6C22E23EBD22E10EDE12E17E0F3
:108EA000F12E00E010E024E630E040E050E06AE51A
:108EB0007CE08DEE9AE29ADE80919005882309F499
:108EC00077CF19C0A12C8BE6C82E83EBD82E10EDDE
:108ED000E12E17E0F12E00E010E024E630E040E063
:108EE00050E06EE57CE089EE9AE280DE80919005AC
:108EF000882309F485CFDF91CF911F910F91FF90C7
:108F0000EF90DF90CF90AF9008952F923F924F92C5
:108F10005F926F927F928F929F92AF92BF92CF9209
:108F2000DF92EF92FF920F931F93CF93DF93CDB712
:108F3000DEB727970FB6F894DEBF0FBECDBF1C017A
:108F40007F836E839C2C8D2CA982CA01B9010F945A
:108F5000EE2D9B01AC01EE81FF81608171818281E8
:108F600093812A833B834C835D830F94EE2D2A816A
:108F70003B814C815D815B016C01A21AB30AC40A7A
:108F8000D50AC801B7010F94EE2D2A813B814C818F
:108F90005D817B018C01E21AF30A040B150BF98148
:108FA000FF938F929F928BEE882E83E4982E6E8192
:108FB0007F81C1010E94AE620F900F900F902796A3
:108FC0000FB6F894DEBF0FBECDBFDF91CF911F91DA
:108FD0000F91FF90EF90DF90CF90BF90AF909F9058
:108FE0008F907F906F905F904F903F902F9008955B
:108FF0006F927F928F929F92AF92BF92CF92DF92A9
:10900000EF92FF920F931F93CF93DF9300D01F92A5
:10901000CDB7DEB761E081E00E940D646090B605D7
:10902000712C61101AC080917F05811104C00E94CB
:10903000D967811198C080911F02882309F48AC0E2
:1090400081E090917F05911180E004E024E045EDFE
:109050005AE2672D0E94D73E7DC081E068122CC085
:1090600080917F05813021F40E94D967811183C0EE
:1090700080911F02882309F46DC011E080917F0563
:10908000813009F010E08091C60C9091C70CA0913E
:10909000C80CB091C90C89839A83AB83BC83CE0181
:1090A00001960E94418500E09C0141EC5AE2672D47
:1090B000812F0E940B3F4EC082E0681225C0809134
:1090C0007F05823021F40E94D967811185C080918B
:1090D0001F02882309F43EC011E080917F05823091
:1090E00009F010E060911E0B70911F0B8091200B16
:1090F0009091210B00DC00E09C014DEA5AE2672DC3
:10910000812F0E940B3F26C083E0681223C080910C
:109110007F05833021F40E94D967811175C0809149
:109120001F028823B9F011E080917F05833009F098
:1091300010E06091220B7091230B8091240B909191
:10914000250BD9DB00E09C014DE95AE2672D812F08
:109150000E940B3F7394639485E0781262CF84E0A1
:1091600080937E0568C00E945D638091900588238E
:1091700009F461CF60C020E030E048EC52E4609137
:10918000C60C7091C70C8091C80C9091C90C0F94BB
:10919000BD2F0F94EE2D1F921F921F9225EE822E4F
:1091A00023E4922E5B016C011CE3E12E16E8F12E04
:1091B00001E010E020E030E0A90166EC7CE08BECFF
:1091C0009AE20E94AE620F900F900F9080919005EE
:1091D000882309F44DCF2FC081E00E94CE67A12CD7
:1091E000C12CD12CE12CF12C08E413E420E030E078
:1091F000A9016EE17BE087EB9AE287DE8091900522
:10920000882309F464CF17C081E00E94CE67A12CA7
:10921000C12CD12CE12CF12C08E413E420E030E047
:10922000A90162E27BE085EA9AE26FDE8091900517
:10923000882309F474CF0F900F900F900F90DF9157
:10924000CF911F910F91FF90EF90DF90CF90BF9043
:10925000AF909F908F907F906F900895AF92CF9234
:10926000DF92EF92FF920F931F93CF93DF9361E012
:1092700081E00E940D64D091B605C0E0D1111AC002
:1092800080917F05811104C00E94D967811103C1BB
:1092900080911F02882309F4F5C081E090917F0539
:1092A000911180E004E024E04BE85AE26C2F0E9428
:1092B000D73EE8C0D13029F580917F05813021F477
:1092C0000E94D9678111EFC080911F02882309F4A1
:1092D000D9C011E080917F05813009F010E06091E4
:1092E000780D7091790D80917A0D90917B0D03DB53
:1092F00000E09C014DE75AE26C2F812F0E940B3F4A
:10930000C1C0D23029F580917F05823021F40E94BE
:10931000D9678111E2C080911F02882309F4B2C08D
:1093200011E080917F05823009F010E060917C0DA2
:1093300070917D0D80917E0D90917F0DDCDA00E0C3
:109340009C014FE65AE26C2F812F0E940B3F9AC07E
:10935000D33029F580917F05833021F40E94D967AD
:109360008111D5C080911F02882309F48BC011E0C0
:1093700080917F05833009F010E06091800D70913D
:10938000810D8091820D9091830DB5DA00E09C01F2
:1093900041E65AE26C2F812F0E940B3F73C0D430FC
:1093A00029F580917F05843021F40E94D9678111CD
:1093B000C8C080911F02882309F464C011E0809125
:1093C0007F05843009F010E06091840D7091850D67
:1093D0008091860D9091870D8EDA00E09C0143E527
:1093E0005AE26C2F812F0E940B3F4CC0D53029F5DB
:1093F00080917F05853021F40E94D9678111BBC01F
:1094000080911F02882309F43DC011E080917F05FF
:10941000853009F010E06091940D7091950D809168
:10942000960D9091970D67DA00E09C0149E45AE2AD
:109430006C2F812F0E940B3F25C0D63019F58091EB
:109440007F05863021F40E94D9678111ADC08091DB
:109450001F028823B9F011E080917F05863009F062
:1094600010E06091980D7091990D80919A0D9091F6
:109470009B0D41DA00E09C0145E35AE26C2F812FFD
:109480000E940B3FCF5FDF5FC53009F0F7CE87E06A
:1094900080937E05A1C00E945D6380919005882322
:1094A00009F4F6CE99C081E00E94CE67A12CC12CB0
:1094B000D12CE12C10ECF12E09E714E420E030E08F
:1094C00040E85FE368E77DE084E89AE21EDD809192
:1094D0009005882309F4F8CE7FC081E00E94CE6712
:1094E000A12CC12CD12CE12C10ECF12E09E714E4B5
:1094F00020E030E040E85FE36CE77DE086E79AE259
:1095000004DD80919005882309F405CF65C081E0D2
:109510000E94CE67A12CC12CD12CE12C10ECF12E95
:1095200009E714E420E030E040E85FE360E87DE034
:1095300088E69AE2EADC80919005882309F412CF4C
:109540004BC081E00E94CE67A12CC12CD12CE12C14
:1095500010ECF12E09E714E420E030E040E85FE38E
:1095600064E87DE08AE59AE2D0DC8091900588236A
:1095700009F41FCF31C081E00E94CE67A12CC12C1D
:10958000D12CE12C10ECF12E09E714E420E030E0BE
:10959000A90164E97DE08EE49AE2B7DC8091900550
:1095A000882309F42DCF18C081E00E94CE67A12C3A
:1095B000C12CD12CE12C10ECF12E09E714E420E0B1
:1095C00030E0A90168E97DE08FE39AE29EDC8091BA
:1095D0009005882309F43BCFDF91CF911F910F9124
:1095E000FF90EF90DF90CF90AF9008956F927F92B1
:1095F0008F929F92AF92BF92CF92DF92EF92FF92A3
:109600000F931F93CF93DF9300D01F92CDB7DEB798
:1096100061E081E00E940D646090B605712C6110DC
:109620001AC080917F05811104C00E94D967811101
:10963000BFC080911F02882309F4B2C081E09091DD
:109640007F05911180E004E024E047EA59E2672DAC
:109650000E94D73EA5C021E0621225C080917F05FF
:10966000813021F40E94D9678111AAC080911F0224
:10967000882309F495C011E080917F05813009F0BD
:1096800010E06091240D7091250D8091260D909130
:10969000270D31D900E09C0147E959E2672D812F60
:1096A0000E940B3F7DC082E0681225C080917F053B
:1096B000823021F40E94D96781119CC080911F02E1
:1096C000882309F46DC011E080917F05823009F094
:1096D00010E06091280D7091290D80912A0D9091D4
:1096E0002B0D09D900E09C0147E859E2672D812F35
:1096F0000E940B3F55C023E062122CC080917F0571
:10970000833021F40E94D96781118EC080911F029D
:10971000882309F445C011E080917F05833009F06A
:1097200010E080912C0D90912D0DA0912E0DB091F7
:109730002F0D89839A83AB83BC83CE0101960E944F
:10974000A78700E09C0147E759E2672D812F0E941F
:109750000B3F26C084E0681223C080917F058430CF
:1097600021F40E94D967811199C080911F0288233A
:10977000B9F011E080917F05843009F010E060912C
:10978000300D7091310D8091320D9091330DB3D821
:1097900000E09C0147E659E2672D812F0E940B3FB4
:1097A0007394639425E072123ACF70927E058FC055
:1097B0000E945D6380919005882309F43ACF87C0A9
:1097C00081E00E94CE67A12CC12CD12CE12C10E8A5
:1097D000F12E07E714E420E030E040E85FE364E2C4
:1097E0007DE08FE999E291DB80919005882309F46F
:1097F0003DCF6DC081E00E94CE67A12CC12CD12C41
:10980000E12C10E8F12E07E714E420E030E040E816
:109810005FE368E27DE08FE899E277DB8091900575
:10982000882309F44BCF53C081E00E94CE6720E02B
:1098300030E048EC52E460912C0D70912D0D809138
:109840002E0D90912F0D0F94BD2F0F94EE2D5B01D7
:109850006C012AE0A21AB108C108D1081F921F9218
:109860001F9297EF892E93E4992E1EEAE12E12E8BB
:10987000F12E01E010E02AE030E040E050E06CE240
:109880007DE08FE799E20E94AE620F900F900F90FB
:1098900080919005882309F439CF19C081E00E9496
:1098A000CE67A12CC12CD12CE12C10E8F12E07E7BA
:1098B00014E420E030E040E85FE360E37DE08FE621
:1098C00099E223DB80919005882309F44ECF0F9015
:1098D0000F900F900F90DF91CF911F910F91FF90FC
:1098E000EF90DF90CF90BF90AF909F908F907F9040
:1098F0006F9008952F923F924F925F926F927F9256
:109900008F929F92AF92BF92CF92DF92EF92FF928F
:109910000F931F93CF93DF93CDB7DEB727970FB683
:10992000F894DEBF0FBECDBF1C017F836E83CA01DA
:10993000B901E982FA820B831C839C2C8D2CAD82A9
:109940002AE037ED43E25CE30F94BD2F0F94EE2D38
:109950002B013C012AE037ED43E25CE3EE81FF811D
:1099600060817181828193810F94BD2F0F94EE2DC0
:109970005B016C01A418B508C608D7082AE037EDCA
:1099800043E25CE3C801B7010F94BD2F0F94EE2DA5
:109990007B018C01E418F50806091709FD81FF9386
:1099A0008F929F9281EF882E83E4982EA3019201DB
:1099B0006E817F81C1010E94AE620F900F900F9067
:1099C00027960FB6F894DEBF0FBECDBFDF91CF91C3
:1099D0001F910F91FF90EF90DF90CF90BF90AF90CD
:1099E0009F908F907F906F905F904F903F902F90BF
:1099F00008959F92AF92BF92CF92DF92EF92FF9223
:109A00000F931F93CF93DF9300D01F92CDB7DEB794
:109A100061E081E00E940D649090B605B12C911038
:109A20001AC080917F05811104C00E94D9678111FD
:109A300052C180911F02882309F444C181E09091B2
:109A40007F05911180E004E024E043E25AE26B2DAF
:109A50000E94D73E37C181E098122CC080917F05CB
:109A6000813021F40E94D96781113DC180911F028C
:109A7000882309F427C111E080917F05813009F026
:109A800010E08091880D9091890DA0918A0DB09180
:109A90008B0D89839A83AB83BC83CE0101960E9490
:109AA000EF8600E09C0147E15AE26B2D812F0E9476
:109AB0000B3F08C182E098122CC080917F05823054
:109AC00021F40E94D967811128C180911F02882347
:109AD00009F4F8C011E080917F05823009F010E0B0
:109AE00080918C0D90918D0DA0918E0DB0918F0D68
:109AF00089839A83AB83BC83CE0101960E94EF8653
:109B000000E09C0143E05AE26B2D812F0E940B3F45
:109B1000D9C083E098122CC080917F05833021F456
:109B20000E94D967811113C180911F02882309F413
:109B3000C9C011E080917F05833009F010E0809169
:109B4000900D9091910DA091920DB091930D8983FC
:109B50009A83AB83BC83CE0101960E94EF8600E01E
:109B60009C0141EF59E26B2D812F0E940B3FAAC04F
:109B700084E0981228C080917F05843021F40E94EF
:109B8000D9678111FEC080911F02882309F49AC011
:109B900011E080917F05843009F010E06091540D50
:109BA0007091550D8091560D9091570D0F941F2E69
:109BB0000E94A14400E09C0143EE59E26B2D812FED
:109BC0000E940B3F7FC085E0981228C080917F05DE
:109BD000853021F40E94D9678111F1C080911F0264
:109BE000882309F46FC011E080917F05853009F06A
:109BF00010E06091580D7091590D80915A0D90911F
:109C00005B0D0F941F2E0E94A14400E09C0145EDC6
:109C100059E26B2D812F0E940B3F54C086E09812B1
:109C200028C080917F05863021F40E94D967811178
:109C3000E4C080911F02882309F444C011E08091A0
:109C40007F05863009F010E060915C0D70915D0D2C
:109C500080915E0D90915F0D0F941F2E0E94A14484
:109C600000E09C0147EC59E26B2D812F0E940B3FD5
:109C700029C087E0981226C080917F05873021F4A3
:109C80000E94D9678111D7C080911F028823D1F02B
:109C900011E080917F05873009F010E06091600D40
:109CA0007091610D8091620D9091630D0F941F2E44
:109CB0000E94A14400E09C0149EB59E26B2D812FE9
:109CC0000E940B3FB394939485E0B812A8CE88E02D
:109CD00080937E05CDC00E945D63809190058823AE
:109CE00009F4A7CEC5C081E00E94CE67A12CC12C8B
:109CF000D12CE12C1CE5F12E01EC17E420E030E042
:109D000040E251E468E87DE08DE19AE2F3DD809184
:109D10009005882309F4AACEABC081E00E94CE67EB
:109D2000A12CC12CD12CE12C1CE5F12E01EC17E467
:109D300020E030E048EC52E46CE87DE08DE09AE20F
:109D4000D9DD80919005882309F4BFCE91C081E0D0
:109D50000E94CE67A12CC12CD12CE12C1CE5F12E48
:109D600001EC17E420E030E048EC52E460E97DE0EB
:109D70008AEF99E2BFDD80919005882309F4D4CE63
:109D800077C081E00E94CE67A12C63E0C62E64E418
:109D9000D62E18EBE12E12E8F12E01E010E024E6B9
:109DA00030E040E050E064E57DE08AEE99E20E9418
:109DB000F64580919005882309F4E5CE59C081E0ED
:109DC0000E94CE67A12C43E0C42E44E4D42E18EBAD
:109DD000E12E12E8F12E01E010E024E630E040E050
:109DE00050E068E57DE08CED99E20E94F6458091B7
:109DF0009005882309F4F2CE3BC081E00E94CE6733
:109E0000A12C23E0C22E24E4D22E18EBE12E12E87E
:109E1000F12E01E010E02AE030E040E050E06CE597
:109E20007DE08EEC99E20E94F645809190058823B2
:109E300009F4FFCE1DC081E00E94CE67A12C83E013
:109E4000C82E84E4D82E18EBE12E12E8F12E01E0A2
:109E500010E024E630E040E050E060E67DE080EC99
:109E600099E20E94F64580919005882309F40CCF71
:109E70000F900F900F900F90DF91CF911F910F9146
:109E8000FF90EF90DF90CF90BF90AF909F9008959C
:109E90002F923F924F925F926F927F928F929F92FA
:109EA000AF92BF92CF92DF92EF92FF920F931F93E8
:109EB000CF93DF93CDB7DEB727970FB6F894DEBF09
:109EC0000FBECDBF1C017F836E83CA01B901E98239
:109ED000FA820B831C839C2C8D2CAD8220E030E019
:109EE00048EC52E40F94BD2F0F94EE2D2B013C0152
:109EF00020E030E048EC52E4EE81FF816081718126
:109F0000828193810F94BD2F0F94EE2D5B016C0124
:109F1000A418B508C608D70820E030E048EC52E4A1
:109F2000C801B7010F94BD2F0F94EE2D7B018C015A
:109F3000E418F50806091709FD81FF938F929F9297
:109F40008DEF882E83E4982EA30192016E817F818C
:109F5000C1010E94AE620F900F900F9027960FB62E
:109F6000F894DEBF0FBECDBFDF91CF911F910F914F
:109F7000FF90EF90DF90CF90BF90AF909F908F9029
:109F80007F906F905F904F903F902F9008959F9299
:109F9000AF92BF92CF92DF92EF92FF920F931F93F7
:109FA000CF93DF9300D01F92CDB7DEB761E081E0A1
:109FB0000E940D649090B605B12C91101AC080914A
:109FC0007F05811104C00E94D9678111D4C080919E
:109FD0001F02882309F4C7C081E090917F05911189
:109FE00080E004E024E045E559E26B2D0E94D73E75
:109FF000BAC081E098122CC080917F05813021F495
:10A000000E94D9678111BFC080911F02882309F483
:10A01000AAC011E080917F05813009F010E08091A5
:10A02000680D9091690DA0916A0DB0916B0D8983B7
:10A030009A83AB83BC83CE0101960E94488800E0DE
:10A040009C0141E459E26B2D812F0E940B3F8BC094
:10A0500082E098122CC080917F05823021F40E940A
:10A06000D9678111ACC080911F02882309F47BC09D
:10A0700011E080917F05823009F010E080916C0D35
:10A0800090916D0DA0916E0DB0916F0D89839A83A3
:10A09000AB83BC83CE0101960E94488800E09C01FE
:10A0A0004DE259E26B2D812F0E940B3F5CC083E093
:10A0B00098122CC080917F05833021F40E94D967CB
:10A0C000811199C080911F02882309F44CC011E0CE
:10A0D00080917F05833009F010E08091700D9091A0
:10A0E000710DA091720DB091730D89839A83AB832A
:10A0F000BC83CE0101960E94488800E09C0149E1A2
:10A1000059E26B2D812F0E940B3F2DC084E09812E5
:10A110002AC080917F05843021F40E94D967811183
:10A1200086C080911F028823F1F011E080917F05A5
:10A13000843009F010E08091740D9091750DA0911C
:10A14000760DB091770D89839A83AB83BC83CE0162
:10A1500001960E94488800E09C0145E059E26B2D81
:10A16000812F0E940B3FB394939485E0B81225CFC2
:10A17000B0927E0577C00E945D6380919005882330
:10A1800009F425CF6FC081E00E94CE67A12C65E065
:10A19000C62E64E4D62EE12C1CE3F12E0CE116E46D
:10A1A00020E030E040EA50E468E67DE08BE499E2AC
:10A1B0006FDE80919005882309F426CF53C081E09B
:10A1C0000E94CE67A12C45E0C42E44E4D42EE12C9D
:10A1D0001CE3F12E0CE116E420E030E040EA50E40C
:10A1E0006CE67DE087E399E253DE80919005882359
:10A1F00009F439CF37C081E00E94CE67A12C25E059
:10A20000C22E24E4D22EE12C1CE3F12E0CE116E444
:10A2100020E030E040EA50E460E77DE083E299E24C
:10A2200037DE80919005882309F44CCF1BC081E074
:10A230000E94CE67A12C85E0C82E84E4D82EE12CA4
:10A240001CE3F12E0CE116E420E030E040EA50E49B
:10A2500064E77DE08FE099E21BDE80919005882322
:10A2600009F45FCF0F900F900F900F90DF91CF9177
:10A270001F910F91FF90EF90DF90CF90BF90AF9024
:10A280009F9008950F93CF93DF9361E081E00E9448
:10A290000D64D091B605C0E0D1111AC080917F0540
:10A2A000811104C00E94D96781118BC080911F0267
:10A2B000882309F47EC081E090917F05911180E0B0
:10A2C00004E024E04CE55BE26C2F0E94D73E71C0B5
:10A2D000D130D9F480917F05813021F40E94D96773
:10A2E000811177C080911F02882309F462C081E048
:10A2F00090917F05913009F080E003E02EE345E581
:10A300005BE26C2F0E94D73E54C0D230D9F48091CA
:10A310007F05823021F40E94D967811164C0809149
:10A320001F02882309F445C081E090917F05923097
:10A3300009F080E003E02EE34EE45BE26C2F0E9424
:10A34000D73E37C0D330D1F480917F05833021F4DC
:10A350000E94D967811151C080911F02882349F161
:10A3600081E090917F05933009F080E003E02EE3D7
:10A3700047E45BE26C2F0E94D73E1BC0D430C9F487
:10A3800080917F05843021F40E94D96781113FC0FC
:10A3900080911F02882369F081E090917F059430BD
:10A3A00009F080E003E02EE34DE35BE26C2F0E94B6
:10A3B000D73ECF5FDF5FC53009F06ECFC0937E051B
:10A3C0002FC00E945D6380919005882309F46ECFB1
:10A3D00027C08EEC95E50E94C344809190058823A8
:10A3E00009F480CF1DC083ED95E50E94C3448091A0
:10A3F0009005882309F493CF13C088ED95E50E945A
:10A40000C34480919005882309F4A6CF09C08DED3F
:10A4100095E50E94C34480919005882309F4B8CF44
:10A42000DF91CF910F910895CF92DF92EF92FF923B
:10A43000CF93C82F0E94AF2A6B017C0124EA30E73A
:10A440004DE75FE36091CD057091CE058091CF051A
:10A450009091D0050F947F2D87FD05C04AEF50E005
:10A4600060E070E003C040E050E0BA01C40ED51EC9
:10A47000E61EF71EC092C905D092CA05E092CB0530
:10A48000F092CC05C0932002CF91FF90EF90DF9027
:10A49000CF9008952F923F924F925F926F927F924A
:10A4A0008F929F92AF92BF92CF92DF92EF92FF92E4
:10A4B0001F93CF93DF93CDB7DEB72A970FB6F894EB
:10A4C000DEBF0FBECDBF1C01162F0E94D9678823A7
:10A4D00029F01092E6050E945D63DAC08091DC05E8
:10A4E0009091DD05A091DE05B091DF058F839887FF
:10A4F000A987BA87892B8A2B8B2B09F491C0E4E0BA
:10A500001E9FD0011124BE83AD83FD01E657F34F9A
:10A51000408051806280738020E030E04AE754E45C
:10A52000C301B2010F94A62C6B017C0180915502EE
:10A530008823F9F01130A9F058F01230D1F4C0900E
:10A540004502D0904602E0904702F090480211C0C8
:10A55000C0903D02D0903E02E0903F02F090400259
:10A5600008C0C0904102D0904202E0904302F090B7
:10A5700044026F81788589859A850F94212E2091D8
:10A58000CD053091CE054091CF055091D0050F9467
:10A59000BD2F9B01AC01C301B2010F94A62C4B014E
:10A5A0005C018D819E818657934F9E838D83DC0154
:10A5B0008D929D92AD92BC9213978F819885A985BB
:10A5C000BA85B7FF1AC020E030E04AE754E4C3017F
:10A5D000B2010F94A52C6B017C019B01AC01C5015C
:10A5E000B4010F947F2D87FF16C0AD81BE81CD923F
:10A5F000DD92ED92FC9213970EC0A7019601C50162
:10A60000B4010F94822F181634F4ED81FE81C082BC
:10A61000D182E282F382812F07DF81E080931F02E3
:10A620001092DC051092DD051092DE051092DF0518
:10A6300080911F02882361F124E0129FF001112410
:10A64000E657F34F80819181A281B38189839A83F8
:10A65000AB83BC832DEC3CEC4CEC5DE36091CD0511
:10A660007091CE058091CF059091D0050F94822FE7
:10A6700087FD05C0CE0101960E94DF8505C060E21E
:10A68000CE0101960E945786BC01C1010E946C3F19
:10A690002A960FB6F894DEBF0FBECDBFDF91CF91E3
:10A6A0001F91FF90EF90DF90CF90BF90AF909F9061
:10A6B0008F907F906F905F904F903F902F90089574
:10A6C00060E084ED9BE2E6CE61E08DEC9BE2E2CEC1
:10A6D00062E086EC9BE2DECECF93DF9300D01F9248
:10A6E000CDB7DEB70E94D967882329F01092E6051E
:10A6F0000E945D635DC06091DC057091DD05809115
:10A70000DE059091DF05611571058105910569F1FF
:10A710000F94212E2091CD053091CE054091CF058B
:10A720005091D0050F94BD2F9B01AC016091960C08
:10A730007091970C8091980C9091990C0F94A62C85
:10A740006093960C7093970C8093980C9093990C4F
:10A7500083E06ADE81E080931F021092DC05109294
:10A76000DD051092DE051092DF0580911F0288231F
:10A77000F9F02091690530916A0540916B0550917F
:10A780006C056091960C7091970C8091980C90914B
:10A79000990C0F94A52C69837A838B839C83CE01BB
:10A7A00001960E94DF85BC0185E69BE20E946C3F1A
:10A7B0000F900F900F900F90DF91CF91089521E0AF
:10A7C0002093E6056093CD057093CE058093CF0569
:10A7D0009093D00540E050E0BA01809167059091D8
:10A7E00068050C94326360E070E080E291E4E7CFAA
:10A7F00060E070E080E89FE3E2CF6DEC7CEC8CECF5
:10A800009DE3DDCFFF920F931F93CF93DF93F82E3D
:10A81000709368056093670561E081E00E940D64B4
:10A82000D091B605C0E091E081E0F816A9F1F816E4
:10A8300028F082E0F81609F45DC08AC0D111FBC08F
:10A840009923D9F080917F051816BCF04091DC0562
:10A850005091DD056091DE057091DF054F5F5F4F20
:10A860006F4F7F4F4093DC055093DD056093DE050D
:10A870007093DF058F5F80937F0580911F0288238F
:10A8800009F44AC100E010E021E041E06FEB7BE217
:10A890008C2F0E94743E40C1D111CDC09923D9F0B4
:10A8A00080917F051816BCF04091DC055091DD05C4
:10A8B0006091DE057091DF054F5F5F4F6F4F7F4FF7
:10A8C0004093DC055093DD056093DE057093DF0552
:10A8D0008F5F80937F0580911F02882309F41CC13C
:10A8E00000E010E021E041E068EB7BE28C2F0E9469
:10A8F000743E12C1D1119FC09923D9F080917F0578
:10A900001816BCF04091DC055091DD056091DE0524
:10A910007091DF054F5F5F4F6F4F7F4F4093DC05B6
:10A920005093DD056093DE057093DF058F5F8093A4
:10A930007F0580911F02882309F4EEC000E010E03B
:10A9400021E041E061EB7BE28C2F0E94743EE4C089
:10A950004091960C5091970C6091980C7091990CC5
:10A960004093690550936A0560936B0570936C057D
:10A97000D1112CC09923D9F080917F051816BCF015
:10A980004091DC055091DD056091DE057091DF0599
:10A990004F5F5F4F6F4F7F4F4093DC055093DD0556
:10A9A0006093DE057093DF058F5F80937F05809154
:10A9B0001F02882309F4E8C000E010E021E041E034
:10A9C00067EA7BE28C2F0E94743EDEC083E0F812BF
:10A9D00032C06091D60B7091D70B8091D80B9091BB
:10A9E000D90B2091930B211126C00F94EE2D2091AD
:10A9F0002B0230912C0262177307ECF4D130C9F4AA
:10AA000080917F05813021F40E94D96781118EC029
:10AA100080911F02882369F081E090917F05913039
:10AA200009F080E004E024E047E95BE26C2F0E943B
:10AA3000D73E82E072C0D130D9F480917F05813059
:10AA400021F40E94D967811179C080911F02882367
:10AA500009F462C081E090917F05913009F080E0B7
:10AA600004E024E04DE85BE26C2F0E94D73E54C026
:10AA7000D230D9F480917F05823021F40E94D967C9
:10AA8000811164C080911F02882309F445C081E0D0
:10AA900090917F05923009F080E003E02EE343E8D7
:10AAA0005BE26C2F0E94D73E37C0D330D1F4809147
:10AAB0007F05833021F40E94D967811151C08091B4
:10AAC0001F02882349F181E090917F05933009F0BE
:10AAD00080E003E02EE34AE75BE26C2F0E94D73E62
:10AAE0001BC0D430C9F480917F05843021F40E94CA
:10AAF000D96781113FC080911F02882369F081E0EE
:10AB000090917F05943009F080E003E02EE34FE65A
:10AB10005BE26C2F0E94D73E85E0CF5FDF5F90E065
:10AB2000C53009F081CE80937E0532C00E945D63FE
:10AB300080919005882309F46BCF2AC00E945D6341
:10AB400080919005882309F480CF22C083EF93E59C
:10AB50000E94C34480919005882309F493CF18C0C4
:10AB600088EF93E50E94C34480919005882309F4FF
:10AB7000A6CF0EC08DEF93E50E94C344809190054F
:10AB8000882309F4B8CF04C083E0F812C5CF21CFE1
:10AB9000DF91CF911F910F91FF9008954FEF60E6E5
:10ABA00073E580E02FCE4FEF64E673E581E02ACEB7
:10ABB0004FEF68E673E582E025CE4FEF6CE673E574
:10ABC00083E020CE0F93CF93DF9361E081E00E947A
:10ABD0000D64D091B605C0E0D1111AC080917F05F7
:10ABE000811104C00E94D96781118BC080911F021E
:10ABF000882309F47EC081E090917F05911180E067
:10AC000004E024E048E35BE26C2F0E94D73E71C071
:10AC1000D130D9F480917F05813021F40E94D96729
:10AC2000811177C080911F02882309F462C081E0FE
:10AC300090917F05913009F080E003E02EE34EE231
:10AC40005BE26C2F0E94D73E54C0D230D9F4809181
:10AC50007F05823021F40E94D967811164C0809100
:10AC60001F02882309F445C081E090917F0592304E
:10AC700009F080E000E22EE340E25BE26C2F0E94EC
:10AC8000D73E37C0D330D1F480917F05833021F493
:10AC90000E94D967811151C080911F02882349F118
:10ACA00081E090917F05933009F080E000E22EE38F
:10ACB00042E15BE26C2F0E94D73E1BC0D430C9F446
:10ACC00080917F05843021F40E94D96781113FC0B3
:10ACD00080911F02882369F081E090917F05943074
:10ACE00009F080E000E22EE34DEF5AE26C2F0E9463
:10ACF000D73ECF5FDF5FC53009F06ECFC0937E05D2
:10AD00002FC00E945D6380919005882309F46ECF67
:10AD100027C082E491E50E94C34480919005882376
:10AD200009F480CF1DC08AE29BE20E94AC62809150
:10AD30009005882309F493CF13C08FE19BE20E9412
:10AD4000AC6280919005882309F4A6CF09C08EE0FB
:10AD50009BE20E94AC6280919005882309F4B8CFF1
:10AD6000DF91CF910F910895CF93DF93EC01CB0149
:10AD7000BA010F94212E0F94EE2D79836883DF9111
:10AD8000CF91089564EB76E585E597E50C947163C2
:10AD90000F931F93CF93DF9361E081E00E940D64D6
:10ADA000C091B605D0E081E0C1112CC08823D9F054
:10ADB00080917F051816BCF04091DC055091DD05AF
:10ADC0006091DE057091DF054F5F5F4F6F4F7F4FE2
:10ADD0004093DC055093DD056093DE057093DF053D
:10ADE0008F5F80937F0580911F02882309F441C003
:10ADF00000E010E020E041E063E37DE28D2F0E945F
:10AE0000743E37C0C130D1F480917F05813021F488
:10AE10000E94D967811137C080911F02882349F1B0
:10AE200081E090917F05913009F080E000E22EE30F
:10AE300048E25DE26D2F0E94D73E1BC0C230C9F4CC
:10AE400080917F05823021F40E94D967811122C050
:10AE500080911F02882369F081E090917F059230F4
:10AE600009F080E000E22EE344E15DE26D2F0E94F4
:10AE7000D73EDF5FCF5F80E0D53009F095CF83E02C
:10AE800080937E050DC0C093260B8091900588238A
:10AE900019F206C0C093260B809190058823C1F259
:10AEA000DF91CF911F910F9108950F94212E0F9450
:10AEB000EE2DCB010C94A284EF92FF920F931F937F
:10AEC000CF93DF93CDB7DEB72B970FB6F894DEBFE5
:10AED0000FBECDBF7C0140916E05842F042E000C67
:10AEE000990B20916F05223051F0233019F022E6A2
:10AEF0003DE20AC047FF06C02EE63DE205C020E85D
:10AF00003DE202C027E73DE29F934F933F932F938B
:10AF10008E010F5F1F4F1F930F930F94D2354091F7
:10AF20002702509128024F50510997010F900F901E
:10AF30000F900F900F900F904E155F050CF49A0133
:10AF40003093D30B2093D20B80E00E947898C801F5
:10AF50000E9429652B960FB6F894DEBF0FBECDBFB9
:10AF6000DF91CF911F910F91FF90EF900895E091A5
:10AF70006E05EE0FFF0BEE52F44F808191819CCF56
:10AF80005F926F927F928F929F92AF92BF92CF9279
:10AF9000DF92EF92FF920F931F93CF93DF93582E80
:10AFA00080936F0560936E0561E081E00E940D64FF
:10AFB000D091B605C0E081E027EB622E27E5722E26
:10AFC000D11138C08823D9F080917F051816BCF0C4
:10AFD0004091DC055091DD056091DE057091DF0543
:10AFE0004F5F5F4F6F4F7F4F4093DC055093DD0500
:10AFF0006093DE057093DF058F5F80937F058091FE
:10B000001F02882309F492C022E0521649F083E01F
:10B01000581203C064E47DE205C064E37DE202C02F
:10B0200064E57DE200E010E021E041E08C2F0E9429
:10B03000743E7CC0D130D9F480917F05813021F4F9
:10B040000E94D96781117BC080911F02882309F477
:10B050006DC081E090917F05913009F080E004E0BF
:10B0600024E04FEB5DE26C2F0E94D73E5FC0D230F0
:10B07000D9F480917F05823021F40E94D967811133
:10B0800066C080911F02882309F450C081E090912E
:10B090007F05923009F080E000E22EE343EB5DE2B1
:10B0A0006C2F0E94D73E42C0D330D1F480917F05EF
:10B0B000833021F40E94D967811154C080911F020E
:10B0C0008823A1F181E090917F05933009F080E021
:10B0D00000E22EE347EA5DE26C2F0E94D73E26C0D5
:10B0E000D43021F580917F05843021F40E94D96706
:10B0F000811143C080911F028823C1F011E080912B
:10B100007F05843009F010E0E0916E05EE0FFF0B33
:10B11000EE52F44F808191810E94A28400E09C0154
:10B1200049E85DE26C2F812F0E940B3FCF5FDF5F0C
:10B1300080E0C53009F044CFC0937E0551C00E9425
:10B140005D6380919005882309F47ECF49C080918A
:10B150007A0590917B05B0DE80919005882309F4F3
:10B1600090CF3EC080917C0590917D05A5DE8091B9
:10B170009005882309F4A2CF33C081E00E94CE67F6
:10B1800060916E05660F770B6E52744FFB01A080C5
:10B19000B180C501BB0CAA0BBB0B5C016D01F8E7CC
:10B1A000AF1AB108C108D1081F927F926F9282EC4A
:10B1B000882E86E5982E1AEAE12EF12C00E010E0A8
:10B1C00028E730E040E050E088E99DE20E94AE626E
:10B1D0000F900F900F9080919005882309F48ACFEB
:10B1E000DF91CF911F910F91FF90EF90DF90CF9063
:10B1F000BF90AF909F908F907F906F905F900895D9
:10B2000060E081E0BDCE8F929F92AF92BF92CF92CD
:10B21000DF92EF92FF920F931F93CF93DF934C0136
:10B220005B016A0160E085E00E940D64D091B60583
:10B23000F12C82E0E82ED1111AC080911F028823E0
:10B2400021F180911E02823041F0833019F469EEC1
:10B250007CE205C067ED7CE202C069EF7CE200E0C1
:10B2600010E021E041E08F2D0E94743E0EC0D130ED
:10B2700061F480911F02882341F000E010E020E09B
:10B2800041E0B4018F2D0E94743EA114B10481F0FD
:10B29000D23081F480911F02882309F46EC000E04F
:10B2A00010E020E041E0B5018F2D0E94743E65C0A2
:10B2B000C2E001C0C3E0C114D10491F0DC130FC09F
:10B2C00080911F02882351F000E010E020E041E06F
:10B2D000B6018F2D0E94743ECD2F01C0CD2FCF5FC0
:10B2E00021E030E0A114B10411F420E030E081E06D
:10B2F00090E0C114D10411F480E090E0820F931F1C
:10B30000029781F0DC130DC080911F02882349F061
:10B3100000E010E020E041E062E17DE28F2D0E943C
:10B32000743ECF5FDC1314C080911F02882371F03C
:10B3300000E010E021E040E067E07DE28F2D0E9418
:10B34000743E60916D058F2D0E94143EE0921F02A5
:10B35000F394DF5F85E0F8126ECFCF5FC0937E0578
:10B36000DF91CF911F910F91FF90EF90DF90CF90E1
:10B37000BF90AF909F908F900895C3E0C114D10407
:10B3800009F0ADCFADCF4EEC5CE26EEB7CE285EB2D
:10B390009CE239CF40E050E065EA7CE28CE99CE237
:10B3A00032CF40E050E06DE87CE28EE79CE22BCFAC
:10B3B00040E050E06FE67CE282E69CE224CF46E586
:10B3C0005CE265E47CE285E39CE21DCF40E050E076
:10B3D00067E27CE28EE19CE216CF40E050E06EE056
:10B3E0007CE281E09CE20FCF40E050E064EF7BE242
:10B3F00083EF9BE208CF40E050E064EE7BE28BED10
:10B400009BE201CF611160931E0240936D05082EEF
:10B41000000C990BAA0BBB0B8B30910580F5FC013E
:10B420008827EA56FF4F8F4F0D9407318AEC99E534
:10B430001CC08DEE99E519C08FED99E516C086EE1A
:10B4400099E513C08BEF99E510C084EF99E50DC025
:10B4500088ED99E50AC081ED99E507C01092260BA9
:10B4600088EC96E502C083EC99E5009741F021E075
:10B470002093E60540E050E0BA010C9432630C944E
:10B4800057638091D105882321F01092E6050E9430
:10B490005D630C94793D9091500893FB882780F967
:10B4A00093FF06C081E090918006911101C080E079
:10B4B000089540E061E080E0A5DF8DE89EE20F9412
:10B4C0006E1C0C94DAD2E7DF882319F080915008C3
:10B4D00082FD0C94459389E89EE20F946E1CF9CF8F
:10B4E0001092141610926F0280915008806280931F
:10B4F00050080E944D936FEF8BE79EE20E94B36964
:10B500000C9457630F93CF93DF9361E081E00E9427
:10B510000D64D091B605C0E08C2F8D0FC9F48091D9
:10B520007F05811104C00E94D967811133C08091C9
:10B530001F02882341F181E090917F05911180E005
:10B5400004E024E046E75EE26C2F0E94D73E1BC079
:10B550008130C9F480917F05813021F40E94D96740
:10B5600081111FC080911F02882369F081E09091B2
:10B570007F05913009F080E000E22EE34BE65EE2C9
:10B580006C2F0E94D73ECF5FC53031F682E08093AA
:10B590007E050CC00E945D6380919005882339F27E
:10B5A00005C09EDF809190058823E1F2DF91CF9165
:10B5B0000F910895EF92FF920F931F93CF93DF9314
:10B5C00061E081E00E940D64C091B60510E0C111F8
:10B5D00018C080917F05811104C00E94D967811134
:10B5E00095C180911F02882361F081E090917F05D1
:10B5F000911180E004E024E04FE55EE2612F0E94BB
:10B60000D73E0E941B63D82F9091500893FBEE24E5
:10B61000E0F893FF03C03FDFF82E01C0F12CDD23DB
:10B6200009F459C0C130D9F480917F05813021F4EB
:10B630000E94D967811171C180911F02882309F48A
:10B6400098C181E090917F05913009F080E000E29F
:10B650002EE343E55EE2612F0E94D73E8AC1C230ED
:10B66000D9F480917F05823021F40E94D96781113D
:10B670005BC180911F02882309F47BC181E0909116
:10B680007F05923009F080E003E02EE348E45EE2BB
:10B69000612F0E94D73E6DC1C33009F057C0809121
:10B6A0007F05833021F40E94D967811147C18091C1
:10B6B0001F02882309F45DC181E090917F059330DA
:10B6C00009F080E003E02EE343E45EE2612F0E9494
:10B6D000D73ED4E05BC0C130D9F480917F05813082
:10B6E00021F40E94D967811133C180911F02882300
:10B6F00009F441C181E090917F05913009F080E02B
:10B7000000E22EE346E35EE2612F0E94D73E33C1A2
:10B71000C230F1F480917F05823021F40E94D96714
:10B7200081111DC180911F02882309F424C181E089
:10B7300090917F05923009F080E003E02EE34DE226
:10B740005EE2612F0E94D73ED3E020C0D4E001C06A
:10B75000D3E0CD131BC080917F058C1304C00E94E1
:10B76000D96781110AC180911F02882371F081E09D
:10B7700090917F059C1380E003E02EE341E25EE2BE
:10B78000612F0E94D73EDC2F01C0DC2F81E08D0F9E
:10B79000C81318C080917F058C1304C00E94D9671C
:10B7A0008111F5C080911F02882361F081E09091A2
:10B7B0007F059C1380E003E02EE343E15EE2612F0E
:10B7C0000E94D73E82E08D0F4091D20B5091D30B57
:10B7D0009091930B911107C020912B0230912C0274
:10B7E00042175307DCF0C81333C080917F058C13D8
:10B7F00004C00E94D9678111D4C080911F028823A0
:10B8000039F181E090917F059C1380E000E22EE306
:10B810004BEF5DE2612F0E94D73E1AC0C81318C0DB
:10B8200080917F058C1304C00E94D9678111C2C02A
:10B8300080911F02882361F081E090917F059C1325
:10B8400080E003E02EE34BEE5DE2612F0E94D73EE5
:10B85000DD5FCD1318C080917F058C1304C00E945A
:10B86000D9678111B1C080911F02882361F081E006
:10B8700090917F059C1380E003E02EE34DED5DE2A7
:10B88000612F0E94D73E91E09D0FEE20E9F0F1106C
:10B8900035C0C91331C080917F058C1304C00E944C
:10B8A000D96781119BC080911F02882329F181E013
:10B8B00090917F059C1380E003E02EE34FEC5DE266
:10B8C000612F0E94D73E18C0C91316C080917F0512
:10B8D0008C1302C00E94D96780911F02882361F0F7
:10B8E00081E090917F059C1380E000E22EE344EC20
:10B8F0005DE2612F0E94D73E92E09D0F1F5FCF5FF8
:10B90000153009F064CE90937E0571C0D6D6809133
:10B910009005882309F465CE6AC0CBDD809190053F
:10B92000882309F489CE63C082E89AE50E94C34463
:10B9300080919005882309F49CCE59C08BE39EE545
:10B940000E94C34480919005882309F4B0CE4FC073
:10B95000BADD80919005882309F4C7CE48C082EEF5
:10B9600095E50E94C34480919005882309F4DACEBE
:10B970003EC0D4E00BCFD3E009CF81E390E60E9434
:10B98000C34480919005882309F4EDCE30C089E945
:10B9900091E60E94C34480919005882309F402CF68
:10B9A00026C08BE09EE2D8D580919005882309F4CB
:10B9B00024CF1DC080E099E50E94C344809190058A
:10B9C000882309F435CF13C081E49AE50E94C3446B
:10B9D00080919005882309F446CF09C08DE792E451
:10B9E0000E94C34480919005882309F45CCFDF91C5
:10B9F000CF911F910F91FF90EF9008956091D00B20
:10BA000070E080E00C94869360916402709165020E
:10BA1000072E000C880B990B0F94212E2AE037ED8E
:10BA200043E25CE30F94BD2F609360027093610268
:10BA300080936202909363020895CF93DF93EC01A9
:10BA4000CB01BA010F94212E0F94F32D6883DF915F
:10BA5000CF91089540E050E0BA0189EE9DE502D60D
:10BA60001092700510927105109272051092730574
:10BA700081E08093E605089540E050E0BA018DEE44
:10BA80009DE5F0D510927005109271051092720527
:10BA90001092730581E08093E60508956DE17DE5E0
:10BAA00083E59DE51EC60F94212E0F94F32D862F5E
:10BAB0000C947C84EF92FF920F931F93CF93DF93AC
:10BAC00000D01F92CDB7DEB7082F7B010E94D96747
:10BAD000882321F01092E605F0D570C08091DC0536
:10BAE0009091DD05A091DE05B091DF050097A105DD
:10BAF000B105D1F11092DC051092DD051092DE0542
:10BB00001092DF0521E020931F02E02FF0E020914A
:10BB10009B0C30E0002E02C0359527950A94E2F781
:10BB200020FF0AC0EE0FFF1FE656F44F208131813F
:10BB3000280F391F31832083092E000CAA0BBB0B61
:10BB40004091700550917105609172057091730577
:10BB5000840F951FA61FB71F8093700590937105E2
:10BB6000A0937205B093730580911F02882331F171
:10BB700084E0089F800111240C5C124F60917005D5
:10BB80007091710580917205909173050F94212E2B
:10BB90009B01AC01F80160817181828193810F94D6
:10BBA000BD2F69837A838B839C8360E2CE010196EB
:10BBB0000E945786BC01C7010E946C3F0F900F90F6
:10BBC0000F900F90DF91CF911F910F91FF90EF9009
:10BBD00008956CE07FE280E06DCF61E07FE281E07C
:10BBE00069CF4F925F926F927F928F929F92AF92A6
:10BBF000BF92CF92DF92EF92FF920F931F93CF935A
:10BC0000DF93F901D8019E2C9A01550F440B550B77
:10BC1000EB01A880B9806501BB0CEE08FF08560156
:10BC20006701A21AB30AC40AD50A2F01FF0F6608DA
:10BC3000770883017201E21AF30A040B150B9F9235
:10BC4000BF93AF93E2EC8E2EE6E59E2E87D40F9045
:10BC50000F900F90DF91CF911F910F91FF90EF9078
:10BC6000DF90CF90BF90AF909F908F907F906F901C
:10BC70005F904F9008956F927F928F929F92AF92B4
:10BC8000BF92CF92DF92EF92FF920F931F93CF93C9
:10BC9000DF9361E081E0C1D5D091B605C0E02EEF21
:10BCA000622E2CE5722ED1111AC080917F05811170
:10BCB00004C00E94D967811121C180911F0288238D
:10BCC00009F413C181E090917F05911180E004E0B7
:10BCD00024E04CEF5EE26C2F0E94D73E06C1D130CB
:10BCE00011F580917F05813021F40E94D96781117F
:10BCF0000CC180911F02882309F4F7C011E08091E4
:10BD00007F05813009F010E080915A0290915B022A
:10BD10000E94A28400E09C0140EF5EE26C2F812F24
:10BD20000E940B3FE2C0D23011F580917F05823036
:10BD300021F40E94D9678111FAC080911F028823E3
:10BD400009F4D3C011E080917F05823009F010E042
:10BD50008091D20B9091D30B0E94A28400E09C01B1
:10BD600042EE5EE26C2F812F0E940B3FBEC0D330AB
:10BD700011F580917F05833021F40E94D9678111EC
:10BD8000EBC080911F02882309F4AFC011E08091BD
:10BD90007F05833009F010E08091C80B9091C90BAA
:10BDA0000E94A28400E09C014AED5EE26C2F812F8C
:10BDB0000E940B3F9AC0D43001F580917F058430FA
:10BDC00021F40E94D9678111DCC080911F02882371
:10BDD00009F48BC011E080917F05843009F010E0F8
:10BDE0008091D00B0E947C8400E09C0146EC5EE2D6
:10BDF0006C2F812F0E940B3F78C0D53011F58091B8
:10BE00007F05853021F40E94D9678111DEC08091C1
:10BE10001F02882309F469C011E080917F058530F5
:10BE200009F010E080916402909165020E94A28462
:10BE300000E09C014CEB5EE26C2F812F0E940B3FD7
:10BE400054C0D630D9F480917F05863021F40E9409
:10BE5000D9678111CCC080911F02882309F445C0A5
:10BE600081E090917F05963009F080E003E02EE3B9
:10BE700041EB5EE26C2F0E94D73E37C0D730D1F441
:10BE800080917F05873021F40E94D9678111BCC061
:10BE900080911F02882349F181E090917F059730BE
:10BEA00009F080E003E02EE346EA5EE26C2F0E9498
:10BEB000D73E1BC0D830C9F480917F05883021F46B
:10BEC0000E94D9678111ADC080911F02882369F05B
:10BED00081E090917F05983009F080E003E02EE347
:10BEE00047E95EE26C2F0E94D73ECF5FDF5FC5302F
:10BEF00009F0D9CE89E080937E059FC0DED3809182
:10BF00009005882309F4D9CE98C0E12C00E010E018
:10BF100027EE33E04AE050E06AE572E086EF9EE209
:10BF200060DE80919005882309F4E3CE86C081E02D
:10BF30000E94CE67E12C04E215E622E231E040E007
:10BF400050E062ED7BE089EE9EE24BDE8091900551
:10BF5000882309F4F2CE71C081E00E94CE67E12C03
:10BF600007E215E627E830E040E050E068EC7BE0CF
:10BF70008EED9EE236DE80919005882309F401CF94
:10BF80005CC081E00E94CE67A090D00BB12CC12C88
:10BF9000D12C1F927F926F928EE4882E8DE5982E81
:10BFA000E12CF12C8701EA9420E030E0A90160ED5A
:10BFB0007BE080ED9EE2D2D20F900F900F908091A7
:10BFC0009005882309F401CF38C0E12C04E01DE579
:10BFD00027EE33E04AE050E064E672E081EC9EE256
:10BFE00000DE80919005882309F411CF26C094D2F9
:10BFF00040E050E0BA018AE29DE534D3809190059B
:10C00000882309F428CF19C087D240E050E0BA0154
:10C010008CE39DE527D380919005882309F438CFE0
:10C020000CC07AD240E050E0BA0185E894E61AD319
:10C0300080919005882309F447CFDF91CF911F911C
:10C040000F91FF90EF90DF90CF90BF90AF909F90B7
:10C050008F907F906F9008951092D10B0E9412994B
:10C0600026C32F923F924F925F926F927F928F9250
:10C070009F92AF92BF92CF92DF92EF92FF920F9377
:10C080001F93CF93DF9361E081E0C7D32090B60583
:10C09000312C6EEF462E6CE5562EC7E2D5E674E2E3
:10C0A000672E75E6772E211019C080917F058111CA
:10C0B00003C07FD78111ABC080911F02882309F490
:10C0C00074C081E090917F05911180E004E024E04C
:10C0D0004AE45FE2632D0E94D73E67C081E02812E8
:10C0E00021C080917F05813019F463D7811196C0FA
:10C0F00080911F02882309F458C011E080917F05C8
:10C10000813009F010E08091D20B9091D30B0E9406
:10C11000A28400E09C014CE35FE2632D812F0E942A
:10C120000B3F43C092E0291220C080917F058230EE
:10C1300019F43FD781119AC080911F028823A9F179
:10C1400011E080917F05823009F010E08091C80BEA
:10C150009091C90B0E94A28400E09C0144E35FE23D
:10C16000632D812F0E940B3F20C083E028121DC049
:10C1700080917F05833019F41CD781119EC0809176
:10C180001F02882391F011E080917F05833009F030
:10C1900010E08091D00B0E947C8400E09C0140E282
:10C1A0005FE2632D812F0E940B3F8091D20B909113
:10C1B000D30B2091C80B3091C90B232B11F4892B81
:10C1C000E9F094E0291218C080917F05843019F4B9
:10C1D000F0D6811195C080911F02882369F081E01B
:10C1E00090917F05943009F080E000E22EE347E172
:10C1F0005FE2632D0E94D73E85E001C084E0339466
:10C20000239495E039124FCF80937E057FC055D29D
:10C2100080919005882309F44FCF78C081E0BED685
:10C22000A090D20BB090D30B0B2C000CCC08DD08E7
:10C230001F927F926F9242EC842E46E5942E12E27A
:10C24000E12EFF24F39400E010E020E030E0A901AB
:10C2500062ED7BE083E49FE281D10F900F900F901D
:10C2600080919005882309F443CF50C081E096D691
:10C27000A090C80BB090C90B0B2C000CCC08DD08AB
:10C280001F92DF93CF9322EC822E26E5922E17E8A1
:10C29000E12EF12C00E010E020E030E0A90168EC94
:10C2A0007BE088E39FE25AD10F900F900F9080912E
:10C2B0009005882309F440CF29C081E06FD6A09073
:10C2C000D00BB12CC12CD12C1F925F924F928EE4D7
:10C2D000882E8DE5982EE12CF12C8701EA9420E040
:10C2E00030E0A90160ED7BE08AE29FE237D10F9058
:10C2F0000F900F9080919005882309F440CF06C0DD
:10C30000ABDE80919005882309F465CFDF91CF9152
:10C310001F910F91FF90EF90DF90CF90BF90AF9063
:10C320009F908F907F906F905F904F903F902F9055
:10C3300008950F931F93CF93DF9361E081E06DD257
:10C34000D091B605C0E0D11116C080917F05811152
:10C3500003C02FD681119AC080911F02882309F44F
:10C360003CC081E090917F05911180E004E024E0E1
:10C370004EE95FE22FC0D130B1F480917F0581306A
:10C3800019F417D6811189C080911F02882329F1E1
:10C3900081E090917F05913009F080E003E02EE389
:10C3A0004CE85FE217C0D230C1F480917F05823043
:10C3B00019F4FFD581117EC080911F02882369F096
:10C3C00081E090917F05923009F080E003E02EE358
:10C3D0004DE75FE26C2F0E94D73E2DD1182FD3304E
:10C3E000D1F480917F05833019F4E3D581116FC0BA
:10C3F00080911F02882309F47CC081E090917F0521
:10C40000933009F080E000E22EE34EE65FE26C2F0D
:10C410000E94D73E6EC081116FC0D430B1F48091BC
:10C420007F05843019F4C5D5811158C080911F0251
:10C43000882319F181E090917F05943009F080E024
:10C4400000E22EE340E65FE215C0D530B1F4809102
:10C450007F05853009F449C080911F02882369F067
:10C4600081E090917F05953009F080E000E22EE3B5
:10C470004FE45FE26C2F0E94D73E86E0CF5FDF5F24
:10C48000C53009F060CF80937E0541C016D1809100
:10C490009005882309F460CF3AC03ED040E050E0D8
:10C4A000BA0188ED94E4DED080919005882309F4E8
:10C4B0006BCF2DC031D040E050E0BA0185E894E662
:10C4C000D1D080919005882309F476CF20C0C9D2BD
:10C4D00080919005882309F48BCF19C0C5D2809133
:10C4E0009005882309F4A2CF12C063D5811106C03C
:10C4F000B3CF112309F4C1CF84E0C0CF0E94D0B8DC
:10C5000081E0EFD180919005882309F4A5CFDF91D8
:10C51000CF911F910F910895809191058630D8F4A5
:10C5200096E0899FF0011124EE56FA4F2091D7052D
:10C530003091D805318320834091DC055091DD0591
:10C540006091DE057091DF054283538364837583B8
:10C550008F5F8093910508950D946E1C2F923F92EA
:10C560004F925F926F927F928F929F92AF92BF9203
:10C57000CF92DF92EF92FF920F931F93CF93DF93AF
:10C5800000D000D0CDB7DEB71C012B833C834D8398
:10C590005E8369837A83C0DF83E080931F023092D9
:10C5A0008F0520928E0569817A8170938D05609345
:10C5B0008C052B813C814D815E81209388053093D1
:10C5C000890540938A0550938B05E0928405F0928B
:10C5D00085050093860510938705A092DC05B0922F
:10C5E000DD05C092DE05D092DF059092D8058092DD
:10C5F000D7058C8D9D8D90938305809382058E8DBC
:10C600008093810526960FB6F894DEBF0FBECDBF8E
:10C61000DF91CF911F910F91FF90EF90DF90CF901E
:10C62000BF90AF909F908F907F906F905F904F9052
:10C630003F902F9008958091A20D90919F0D891B9E
:10C640008F7071F49091500892FB882780F992FDC9
:10C6500008C081E090910716913019F080E00895AC
:10C6600081E008952091D7053091D8052817390722
:10C67000E9F09093D8058093D7054093DC0550935B
:10C68000DD056093DE057093DF058E52974621F439
:10C690001092E605109291050E94133E82E080936D
:10C6A0001F0281E0809390051092E105089540E01B
:10C6B00050E0BA018EE297E6D5CFE0919105EE23E6
:10C6C00079F0E150E093910586E0E89FF0011124B4
:10C6D000EE56FA4F40E050E0BA0180819181C2CF1E
:10C6E000E6CF0F931F93CF93DF93FC01EB01809173
:10C6F000DC059091DD05A091DE05B091DF05B7FF67
:10C7000008C01092DC051092DD051092DE05109233
:10C71000DF058091840590918505A0918605B091F3
:10C7200087054091DC055091DD056091DE05709133
:10C73000DF0584179507A607B70744F48093DC0547
:10C740009093DD05A093DE05B093DF0580911F0275
:10C75000882301F18091880590918905A0918A052F
:10C76000B0918B054091DC055091DD056091DE05AF
:10C770007091DF058C019D01040F151F261F371FC7
:10C78000C901B8011995BC0180918E0590918F0562
:10C790000E946C3F8091D105811108C08091810574
:10C7A0008823B1F180911F02882391F180918C053B
:10C7B00090918D050097B1F0009188051091890541
:10C7C00020918A0530918B054091DC055091DD0563
:10C7D0006091DE057091DF05400F511F621F731FCE
:10C7E000FE011995E0918205F0918305309741F0A3
:10C7F00080918105811103C08091D1058111199526
:10C80000D8D3882329F0DF91CF911F910F9155CF75
:10C81000DF91CF911F910F910895282F1092D60587
:10C820008091DC059091DD05A091DE05B091DF05DA
:10C8300081309048A105B10540F01092DC051092BE
:10C84000DD051092DE051092DF058091E00588235A
:10C8500031F08091DC0580937F05109290058091E6
:10C860007E051816FCF4082E000C990B821B91090A
:10C8700020917F05022E000C330B2817390794F006
:10C8800097FF02C080E090E080937F05092E000CA6
:10C89000AA0BBB0B8093DC059093DD05A093DE050E
:10C8A000B093DF0580917F056623C1F09091B605B6
:10C8B000891714F48093B6052091B605022E000C5A
:10C8C000330B2C5F3F4F482F082E000C550B2417BD
:10C8D000350734F484508093B60508958093B605E7
:10C8E0000895882361F063E972E084E690E00F9494
:10C8F00074276AEB72E084E690E00D94742768EB8D
:10C9000071E084E190E00D9474278F929F92AF9232
:10C91000BF92CF92DF92EF92FF924BD3882359F0D0
:10C920001092E605FF90EF90DF90CF90BF90AF9010
:10C930009F908F90C2CE81E08093E605C090DC0589
:10C94000D090DD05E090DE05F090DF05C114D10444
:10C95000E104F10409F450C01092DC051092DD05E9
:10C960001092DE051092DF05B6010D2C000C880B2D
:10C97000990B0F94212E20913C0D30913D0D40914B
:10C980003E0D50913F0D0F94BD2F2091640C3091BE
:10C99000650C4091660C5091670C0F94A62C4B01CE
:10C9A0005C0120E030E040E050EC0F94822F87FDE6
:10C9B00023C020E030E040EA50E4C501B4010F9408
:10C9C0007F2D1816CCF080919B0C82FF0AC08091BD
:10C9D0009E0B90919F0BC80ED91ED0929F0BC092B8
:10C9E0009E0B8092640C9092650CA092660CB092A3
:10C9F000670C82E080931F0280911F028823D9F088
:10CA000084E69CE00E944185BC0183EA9FE20E948B
:10CA10006C3F6091640C7091650C8091660C9091F4
:10CA2000670CFF90EF90DF90CF90BF90AF909F90FA
:10CA30008F900C941940FF90EF90DF90CF90BF90B3
:10CA4000AF909F908F90089580E00C9478980C940C
:10CA5000C59821E0209380050F94731C10928005E7
:10CA600008950E9468B53DCF0E94FFC23ACFFC01F5
:10CA700080810895FC01849108954F925F926F9296
:10CA80007F928F929F92AF92BF92CF92DF92EF925E
:10CA9000FF920F931F93CF93DF936C017B015A0199
:10CAA0002901672B31F088248394912CC0E0D0E0D9
:10CAB00019C0F8011182108227C03701680C791C57
:10CAC00076946794E3012197A201BE01C601F501A6
:10CAD00019951816190654F0892BC9F04301FFEF78
:10CAE0008F1A9F0AE814F90440F702C07E01FACFBA
:10CAF000CE15DF0530F4CE0102968816990620F097
:10CB00002196F801D183C0838FEF9FEF05C0F80114
:10CB1000D183C08380E090E0DF91CF911F910F918E
:10CB2000FF90EF90DF90CF90BF90AF909F908F904D
:10CB30007F906F905F904F9008958F929F92AF92E9
:10CB4000BF92CF92DF92EF92FF920F931F93CF93FA
:10CB5000DF93EC016B017A01FB01199587FD06C09B
:10CB6000082F10E020E030E0219620C1982F907E21
:10CB7000903CC1F4082F0F7110E020E030E0480134
:10CB8000590186E0880C991CAA1CBB1C8A95D1F718
:10CB9000CE010196F60119958F7395018401082B3A
:10CBA000229604C1982F907F903E19F58F70882EA1
:10CBB000912CA12CB12C16E0880C991CAA1CBB1C32
:10CBC0001A95D1F7CE010196F60119958F73882A2F
:10CBD00006E0880C991CAA1CBB1C0A95D1F7CE0153
:10CBE0000296F60119958F7395018401082B2396FF
:10CBF000DDC0982F987F903F81F58770882E912C0B
:10CC0000A12CB12CF6E0880C991CAA1CBB1CFA952F
:10CC1000D1F7CE010196F60119958F73882AA6E007
:10CC2000880C991CAA1CBB1CAA95D1F7CE010296B0
:10CC3000F60119958F73882AB6E0880C991CAA1CF6
:10CC4000BB1CBA95D1F7CE010396F60119958F73E7
:10CC500095018401082B2496A9C0982F9C7F983FAA
:10CC6000E9F58370882E912CA12CB12C56E0880C0C
:10CC7000991CAA1CBB1C5A95D1F7CE010196F6014E
:10CC800019958F73882A66E0880C991CAA1CBB1C16
:10CC90006A95D1F7CE010296F60119958F73882A0D
:10CCA00076E0880C991CAA1CBB1C7A95D1F7CE01A2
:10CCB0000396F60119958F73882AE6E0880C991C73
:10CCC000AA1CBB1CEA95D1F7CE010496F601199572
:10CCD0008F7395018401082B259668C0982F9E7F3D
:10CCE0009C3F09F04AC08170882E912CA12CB12C58
:10CCF00086E0880C991CAA1CBB1C8A95D1F7CE0132
:10CD00000196F60119958F73882A96E0880C991C74
:10CD1000AA1CBB1C9A95D1F7CE010296F601199573
:10CD20008F73882A26E0880C991CAA1CBB1C2A95A4
:10CD3000D1F7CE010396F60119958F73882A36E054
:10CD4000880C991CAA1CBB1C3A95D1F7CE010496FD
:10CD5000F60119958F73882A46E0880C991CAA1C45
:10CD6000BB1C4A95D1F7CE010596F60119958F7334
:10CD700095018401082B269619C0982F907C903835
:10CD800049F4082F007C003871F42196CE01F60199
:10CD90001995F7CF082F0E7F0D3F28F02196CE0171
:10CDA000F6011995F7CF00E010E09801E114F104C5
:10CDB00029F0F7010083118322833383CE01DF91B1
:10CDC000CF911F910F91FF90EF90DF90CF90BF9088
:10CDD000AF909F908F9008951F93CF93DF9300D0D3
:10CDE0001F92CDB7DEB710E0AE014F5F5F4F67E334
:10CDF00075E6A3DE49815A816B817C81452B462BE8
:10CE0000472B11F01F5FF0CF812F0F900F900F90E5
:10CE10000F90DF91CF911F9108951F93CF93DF93D0
:10CE200000D01F92CDB7DEB710E0AE014F5F5F4F6D
:10CE30006AE375E682DE49815A816B817C81452BEC
:10CE4000462B472B11F01F5FF0CF812F0F900F90D3
:10CE50000F900F90DF91CF911F9108951092D605FA
:10CE60008091D1051092D105882341F040E050E037
:10CE7000BA018AED9AE5F6DB0C94DE3D20915A0268
:10CE800030915B024091DC055091DD056091DE053B
:10CE90007091DF05C901840F951F2436310571F4A7
:10CEA000473051056105710514F0069732C04A3FBD
:10CEB0005F4F6F4F7F4F54F506962BC024363105D8
:10CEC00024F48536910514F504C08436910524F4C4
:10CED0001DC08A3091053CF0883E43E094072CF059
:10CEE00087EE93E002C08AE090E02817390761F0EE
:10CEF00090935B0280935A021092DC051092DD053C
:10CF00001092DE051092DF050C94FB3584E690E06C
:10CF1000E3CF8A30910504F78AE090E0E9CFCF9320
:10CF2000DF931F92CDB7DEB780910108811103C056
:10CF300083E498E02FC0211103C081E098E02AC06B
:10CF40008DE0815048F0440F411DE82FF0E0ED5B8B
:10CF5000F74F90814927F5CF8091C8058417A9F034
:10CF60004093C80581E098E0698336DF90E06981ED
:10CF7000861B910997FF02C080E090E08093D9055D
:10CF80001092DA0588E0809321028091DA0590E022
:10CF90008F5F974F0F90DF91CF9108958093D605C3
:10CFA0001092D2051092D3051092D4051092D50597
:10CFB00008958091D1051092D1050895CF92DF9206
:10CFC000EF92FF920F931F930E94AF2A0091C40526
:10CFD0001091C5052091C6053091C7056B017C01F4
:10CFE000C01AD10AE20AF30AF7FC13C02091C30564
:10CFF00020952093C305DC01CB018A549C4FAF4F91
:10D00000BF4F8093C4059093C505A093C605B09308
:10D01000C70581E09091C305911101C080E01F9187
:10D020000F91FF90EF90DF90CF900895809150087E
:10D0300082FF09C083FF04C080918006811106C071
:10D0400020E02093E9058091E905089580910B0681
:10D0500090910C06A0910D06B0910E060097A105C7
:10D06000B10571F3BC01CD016D597F4F8F4F9F4FBB
:10D0700024E630E040E050E00F94C93060910706AC
:10D08000709108068091090690910A060F94C930A4
:10D09000D8CFCF9393E090931F0281111092E805AF
:10D0A0000E94AF2ADC01CB018C509E4FAF4FBF4F87
:10D0B0008093E2059093E305A093E405B093E50522
:10D0C00068E873E182E090E00F947427C6E0C150F5
:10D0D00049F00F94092762E070E080E090E00E9440
:10D0E000E02AF5CFCF910895AF92BF92CF92DF9211
:10D0F000EF920F931F93CF93DF9300D01F92CDB782
:10D10000DEB7809120028F3F09F444C00E94AF2A0D
:10D110000091C9051091CA052091CB053091CC052D
:10D12000DC01CB01801B910BA20BB30BB7FD32C00E
:10D1300090919F0D8091A20D8F5F8F70981751F184
:10D14000E091200284E0E802F0011124EB58FC4F4A
:10D1500020E030E040E752E4608171818281938178
:10D160000F94862D69837A838B839C83A12CB12CA9
:10D170006501E12C8E010F5F1F4F26E93CE042E97B
:10D180005CE06EE87CE08AE89CE00E949EE18FEF24
:10D19000809320020F900F900F900F90DF91CF910E
:10D1A0001F910F91EF90DF90CF90BF90AF900895B7
:10D1B0000F931F930E94AF2A0091E2051091E3059F
:10D1C0002091E4053091E505DC01CB01801B910B3A
:10D1D000A20BB30BB7FD11C08091030181FB99270E
:10D1E00090F981E089279091030192FF82609091EC
:10D1F000000196FF84608093E8058091E8058170C6
:10D200009091E80591FD82609091B705891741F1F1
:10D210008130A9F028F0823041F0833059F01EC0EF
:10D22000913089F09230A9F019C0992361F09330C0
:10D2300081F014C0913069F0923081F404C09923D8
:10D2400041F0933059F49091DB0591509093DB05B8
:10D2500005C09091DB059F5F9093DB058093B70538
:10D260001F910F910895CF93DF930E94DE3DE4E07C
:10D27000F1E080818D7F8083C5E0D1E08881809559
:10D28000827043E051E0DA018C9380818B7F808350
:10D290008881809584708C9321E031E0D9018C9154
:10D2A0008F7B8C9380910201809580748093000124
:10D2B00080818E7F8083888180958170FA01808350
:10D2C00082E08093E70574DF1092DB05DF91CF9158
:10D2D000089581E09091EA05911101C080E00895E0
:10D2E000CF93DF932091010621111EC0FC01019014
:10D2F0000020E9F73197EF01C81BD90BC731D105E1
:10D3000034F031972081207C2038D9F3F4CFBC0150
:10D31000DD27AE018AEE95E00F94B835C651DA4F9D
:10D32000188283E080931F02DF91CF910895CF93FD
:10D33000DF93CDB7DEB78E8190910106891780F01B
:10D34000809301069E01275F3F4F4F81588566E11C
:10D3500070E08AEE95E00F94013683E080931F021F
:10D36000DF91CF9108950F931F93CF93DF938C019B
:10D3700067FF03C01092010660E08091010690E013
:10D38000262F062E000C330B281739070CF160935B
:10D390000106C8010F941A35F801E80FF91FEF01D3
:10D3A000C01BD10BC731D10534F031978491807CFB
:10D3B0008038D9F3F4CFDD27AE01B8018AEE95E0CD
:10D3C0000F943B35C651DA4F188283E080931F02D9
:10D3D000DF91CF911F910F9108954F925F926F92BD
:10D3E0007F928F929F92AF92BF92CF92DF92EF92F5
:10D3F000FF920F931F9378DEDBDE8091E80582FFBA
:10D4000015C08091C205811113C091E09093C205AF
:10D4100020911416211103C08091800589278093E3
:10D42000D1051092141681E034DE02C01092C205BC
:10D4300080910301809581701091E7058117B9F003
:10D440008093E705882309F4A6C164EF71E080E0CA
:10D4500090E00E9438840E945F75123009F096C1F6
:10D460000E942F7683E080931F020E94DE3D0E947F
:10D47000AF2A6B017C018091BE059091BF05A09100
:10D48000C005B091C105A7019601281B390B4A0BB5
:10D490005B0B57FF05C08091E105882309F427C283
:10D4A000D701C6018C599F4FAF4FBF4F8093BE0528
:10D4B0009093BF05A093C005B093C1056091DB05B3
:10D4C000062E000C770B77FF03C0719561957109EB
:10D4D000062E000C770B880B990B0F94212E2B0135
:10D4E0003C0120E030E040E050E40F94822F87FFC1
:10D4F00005C08091D105811183C093C08091D6056C
:10D50000882309F456C08090D2059090D305A0904E
:10D51000D405B090D50581149104A104B104E1F1C2
:10D5200020E030E040E05FE3C301B2010F94BD2F83
:10D530002B013C01C701B601681979098A099B09C9
:10D540000F941F2E9B01AC01C301B2010F94862DD5
:10D5500020E030E04AE754E40F94BD2F4B015C011A
:10D5600020E030E040EA52E40F94822F87FF0FC0A2
:10D5700020E030E040EF51E4C501B4010F94822F68
:10D5800087FD0AC02AE030E040E050E009C024E610
:10D5900030E040E050E004C021E030E040E050E006
:10D5A000C092D205D092D305E092D405F092D50571
:10D5B00004C021E030E040E050E0A091DB050A2EFD
:10D5C000000CBB0B0F942E3122E030E040E050E025
:10D5D0000F94EB308091DC059091DD05A091DE0584
:10D5E000B091DF05820F931FA41FB51F8093DC0548
:10D5F0009093DD05A093DE05B093DF051092DB0567
:10D60000D701C6018856954CAF4FBF4F8093BA05DE
:10D610009093BB05A093BC05B093BD0581E08093BA
:10D620001F022091D7053091D80547E62E323407E6
:10D6300041F480912102882309F4C0C08150809375
:10D6400021022D57324471F48091DA059091D90569
:10D65000891740F490912102992309F4BFC0915099
:10D660009093210280916F0081FB222720F981FF96
:10D6700005C080916F008D7F80936F008091B20C08
:10D680009091B30CA091B40CB091B50C222329F069
:10D6900020916F00226020936F003AE0B695A79525
:10D6A000979587953A95D1F7009721E0A207B105A4
:10D6B00020F08FEF9FEFA0E0B0E096958795209146
:10D6C0001F02211105C03091E10531110CC151C07B
:10D6D000009741F04091B8055091B9054817590796
:10D6E00008F047C08091E105811117C0223008F091
:10D6F0008DC080916604811107C081E0809366042B
:10D700008DE294E00E94772F8DE294E00E94AE2F8C
:10D7100081E08093E0058093E10583E00E94F73C7F
:10D7200061E08DE294E00E94D72FE091D705F0915F
:10D73000D80519951092E0058091E105811172C01C
:10D740001092D1050E94AF2ADC01CB018C199D09F2
:10D75000AE09BF090091B8051091B90520E030E08D
:10D76000081719072A073B0720F49093B9058093FF
:10D77000B8058091D7059091D8058E52974609F447
:10D78000A3C08091E60581119FC072C060E08CEE5D
:10D790009FE2E9DD67CE8BD5123009F463CE60E0FD
:10D7A0008FED9FE2E0DD8091D7059091D8058E52F4
:10D7B000974609F457CE0E94576354CE8CE080936D
:10D7C00021028091B8059091B90501979093B90510
:10D7D0008093B80581E080931F0233CF96E0909349
:10D7E000210291E090931F028F5F8093DA05D701A9
:10D7F000C6018856954CAF4FBF4F8093BA059093A2
:10D80000BB05A093BC05B093BD052CCF243030F0F0
:10D81000243009F06ECF10921F026BCF81E080930D
:10D820001F0267CF8DE294E00E94B22F91E0811138
:10D8300001C090E09093E105992309F481CF0E9403
:10D84000AF2ADC01CB018C199D09AE09BF09C0903C
:10D85000B805D090B905E12CF12CC816D906EA0616
:10D86000FB0608F044C09093B9058093B8053FC00B
:10D870008091BA059091BB05A091BC05B091BD0502
:10D88000C81AD90AEA0AFB0AF7FE0E945763809178
:10D89000E10581112CC080911F02813091F083300D
:10D8A00031F51F910F91FF90EF90DF90CF90BF90D7
:10D8B000AF909F908F907F906F905F904F900C945F
:10D8C000133E10921F0213C048E9C40E4AE3D41E4F
:10D8D000E11CF11CC092BA05D092BB05E092BC05D8
:10D8E000F092BD05D4CF009709F417CFF3CE1F9166
:10D8F0000F91FF90EF90DF90CF90BF90AF909F90EF
:10D900008F907F906F905F904F90089561E02BDD36
:10D910000C945763CF93DF931F921F92CDB7DEB75E
:10D9200089839A83A0DC89819A81F0DF0F900F9020
:10D93000DF91CF910C94E33D8091500882FD05C0AA
:10D9400080910716823061F410C080910108811126
:10D9500003C083E498E002C081E098E061E0C0CCBD
:10D96000813031F082EB9FE205C082ED9FE202C080
:10D9700086EC9FE26FEFF7CC8EE297E69093D805A6
:10D980008093D705089561E0FC0180810E94D42C2A
:10D990008FEF0C94148ECF93DF93EC018A810E9459
:10D9A000D58D60E08881DF91CF910C94D42C8F923B
:10D9B0009F92AF92BF92EF92FF920F931F93CF93DC
:10D9C000DF93EC018B017A010E94AF2A4B015C01CD
:10D9D0002CE2820E21E0921EA11CB11C0E94EE8D51
:10D9E0008B838F3F61F40E94AF2ADC01CB01881941
:10D9F0009909AA09BB09B7FDF1CF81E10DC08E3F9E
:10DA000051F4B701C8010E94F58D0E94EE8D0E946D
:10DA1000EE8D11E003C08FE0898310E0CE01B3DF0B
:10DA2000812FDF91CF911F910F91FF90EF90BF90C9
:10DA3000AF909F908F900895CF92DF92EF92FF92D8
:10DA40006A017B010E94AF2AC60ED71EE81EF91E8E
:10DA50000E94EE8D8F3F61F00E94AF2ADC01CB0166
:10DA60008C199D09AE09BF09B7FDF2CF80E001C056
:10DA700081E0FF90EF90DF90CF900895EF92FF92BA
:10DA80001F93CF93DF9300D01F92CDB7DEB77C01F9
:10DA9000162F29833A834B835C837DDF48E552E070
:10DAA00060E070E0C701C8DF812F80640E94148E9F
:10DAB0008C810E94148E8B810E94148E8A810E9418
:10DAC000148E89810E94148E112311F087E801C001
:10DAD00085E90E94148E1C3011F40E94EE8D10E036
:10DAE0000E94EE8DF701838387FF04C01F3F11F072
:10DAF0001F5FF6CF0F900F900F900F90DF91CF9197
:10DB00001F91FF90EF9008958F929F92AF92BF92D6
:10DB1000CF92DF92EF92FF920F931F93CF93DF93F9
:10DB2000EC01162F1C82198248830E94AF2A6B01D8
:10DB30007C0120EDC20E27E0D21EE11CF11CA8954D
:10DB400061E088810E94D42C61E088810E94982C39
:10DB50000E94E68D85E08A830E94D58D0AE08FEFD2
:10DB60000E94148E0150D9F7A89520E030E0A90159
:10DB700060E0CE0183DF8B83813061F00E94AF2AA9
:10DB8000DC01CB018C199D09AE09BF09B7FDEDCFB2
:10DB900081E055C0A8952AEA31E040E050E068E015
:10DBA000CE016CDF853011F481E009C004E00E94F1
:10DBB000EE8D8B830150D9F78A3A51F482E08C8341
:10DBC000A8958C81823081F0812C912C540111C058
:10DBD0000E94AF2ADC01CB018C199D09AE09BF0957
:10DBE000B7FDD9CF82E02BC0812C912CA12C80E4F1
:10DBF000B82E20E030E0A90167E3CE013FDFA501A8
:10DC0000940169E2CE013ADF8B83882361F00E94A0
:10DC1000AF2ADC01CB018C199D09AE09BF09B7FD04
:10DC2000E8CF8AE00CC08C818230D1F420E030E073
:10DC3000A9016AE3CE0122DF882329F088E08983E5
:10DC4000CE01A1DE16C00E94EE8D807C803C11F4D6
:10DC500083E08C830E94EE8D0E94EE8D0E94EE8DFB
:10DC6000CE0191DE173018F41A8381E003C088E1F9
:10DC7000898380E0DF91CF911F910F91FF90EF900A
:10DC8000DF90CF90BF90AF909F908F9008950F93AB
:10DC90001F93CF93DF93EC0189018C81833039F09E
:10DCA00089E0440F551F661F771F8A95D1F79A01A7
:10DCB000AB0161E1CE01E2DE811109C040E052E03A
:10DCC000B801CE01DF91CF911F910F9170CE84E00A
:10DCD0008983CE0158DE80E0DF91CF911F910F91B3
:10DCE0000895CF93DF93EC01862FBA010E94198E1D
:10DCF0008FEF0E94148E8FEF0E94148E0E94EE8D83
:10DD00008B83982F9F71953031F083E18983CE0109
:10DD10003ADE80E001C081E0DF91CF9108950F935A
:10DD20001F93CF93DF93EC0189018C81833039F00D
:10DD300089E0440F551F661F771F8A95D1F79A0116
:10DD4000AB0168E1CE019ADE81111EC0A8016EEF21
:10DD5000CE01C7DF8823E1F048E552E060E070E0E3
:10DD6000CE016ADE882371F020E030E0A9016DE089
:10DD7000CE0184DE81110AC00E94EE8D811106C0A1
:10DD800011E007C087E103C086E001C086E1898316
:10DD900010E0CE01F8DD812FDF91CF911F910F911F
:10DDA0000895CF93DF931F92CDB7DEB7209116165B
:10DDB00030911716CE0101962115310519F0821BFD
:10DDC000930B02C08C5196410F90DF91CF91089533
:10DDD000FC01238121110C94897F089580915008C2
:10DDE000847F8B7F8093500810920706109208065C
:10DDF0001092090610920A0610920B0610920C0659
:10DE000010920D0610920E0610927C061092BB0620
:10DE10008EE091E0ECEBF6E0DF019C011D922150D9
:10DE20003040E1F78FEF809300080895FC0120E077
:10DE30003EE2DB014C91403241F0283011F4308356
:10DE40003196DB014C91408331962F5F6F5F7F4F9E
:10DE50002B3079F7108208952F923F924F925F9264
:10DE60006F927F928F929F92AF92BF92CF92DF92EA
:10DE7000EF92FF920F931F93CF93DF93CDB7DEB74F
:10DE8000C356D1090FB6F894DEBF0FBECDBF8C01CB
:10DE90005B014A014DB65EB6312C7E0187E5E80E86
:10DEA000F11C9BE1292E41E058E0BE016F5F7F4FDE
:10DEB000C5010E94F97D18160CF005C18C85282F2C
:10DEC0002871203109F074C090910606915092306B
:10DED00008F46EC06DB67EB6BE016F5F7F4FC7019E
:10DEE000A5DF0115110521F0F8018081811173C0B2
:10DEF00021E081E090E0F70101900020E9F73197FF
:10DF0000EE19FF09E80FF91F32968DB79EB78E1BE9
:10DF10009F0B0FB6F8949EBF0FBE8DBFEDB7FEB737
:10DF200031966F01211102C0B80102C065E873E0AB
:10DF3000C6010F94A335B701C6010F948D3565E86E
:10DF400073E0C6010F948D351CAE1FAE21E0A70112
:10DF5000B501CE01CC960E94858181110DC08091C2
:10DF60000606811109C00E94ED898CED91E30E94A3
:10DF7000DF89C7010E94AB8CFE01FC96DE01919601
:10DF8000822D01900D928A95E1F740E050E0BE01AC
:10DF90006F5D7F4FC60160DFCE01819619DFCE0134
:10DFA000CC9616DF0FB6F8947EBE0FBE6DBE7BCF4B
:10DFB0009981992309F487C0953E09F474CF9E3264
:10DFC00009F471CF909101089E3209F46CCF8A70E8
:10DFD00009F069CF0AC0F80101900020E9F73197F4
:10DFE000CF01801B910B20E086CF81E0203109F02A
:10DFF00080E09091500880FB94F990935008811133
:10E0000008C08985873409F04ECF8A858E3709F498
:10E010004ACF80910606813021F068F08230B9F154
:10E0200042CF8091040690910506019690930506D3
:10E030008093040638CFBE016F5F7F4F83E498E082
:10E04000F5DE0115110511F0680105C083E4C82E45
:10E0500088E0D82E08C0F60181916F018823B1F3C2
:10E060000E94548CF8CFF60181916F01882319F03A
:10E070000E94548CF8CF80E20E94548C6D8D7E8D6E
:10E080008F8D98A14AE050E00E94618D0CCFBE01B7
:10E090006F5F7F4F83E498E0C9DE8114910441F003
:10E0A00063E478E0C4010F947A35892B51F40BC0F6
:10E0B000832D90E02091020630910306821793078A
:10E0C00011F03394F0CE0FB6F8945EBE0FBE4DBE85
:10E0D000CD59DF4F0FB6F894DEBF0FBECDBFDF9135
:10E0E000CF911F910F91FF90EF90DF90CF90BF9055
:10E0F000AF909F908F907F906F905F904F903F90E8
:10E100002F900895CF93DF93CDB7DEB76B970FB6FF
:10E11000F894DEBF0FBECDBF1092060640E050E07F
:10E12000BA0185EE97E00E94A87E8BE1E5EEF7E06C
:10E13000DE01119601900D928A95E1F740E050E0E2
:10E14000BE016F5F7F4F80E090E086DECE010196DA
:10E150003FDE6B960FB6F894DEBF0FBECDBFDF91EA
:10E16000CF9108950F931F93CF93DF93CDB7DEB771
:10E170002D970FB6F894DEBF0FBECDBF80918006FD
:10E18000882391F0BE016F5F7F4F8DE796E00E947C
:10E190001B7C8E010F5F1F4FF80181918F01882337
:10E1A00039F00E94548CF8CF82ED91E30E94DF8910
:10E1B0008AE00E94548C2D960FB6F894DEBF0FBEF5
:10E1C000CDBFDF91CF911F910F910895CF92DF9234
:10E1D000EF92FF920F931F93CF93DF93CDB7DEB7EC
:10E1E000EDB6FEB6DC010D900020E9F79D01281B7D
:10E1F000390B2C5F3F4F4DB75EB7421B530B0FB629
:10E20000F8945EBF0FBE4DBF0DB71EB70F5F1F4F17
:10E210009F938F938CE891E39F938F931F930F931A
:10E220000F94D235680154E0C50ED11C0F900F90A9
:10E230000F900F900F900F90F6018081882349F086
:10E24000082E000C990B0F94FE34F60181936F0198
:10E25000F3CFC8010F94731C88E891E30F946E1CF0
:10E260000FB6F894FEBE0FBEEDBEDF91CF911F91A9
:10E270000F91FF90EF90DF90CF900895809150081C
:10E2800083FF03C0846080935008089510921D0B93
:10E29000809150088F7D8B7F809350080E944B5A4D
:10E2A000882321F08DE796E00C94897F0895EEDFB6
:10E2B00080915008877F8093500808950F931F9393
:10E2C000CF93DF938B01EA01DB016D917C910E947A
:10E2D0001B7CD801ED91FC919081888191110EC039
:10E2E0008936B0F48FE28083F801808191810196B4
:10E2F0009183808388818F5F88830AC0893680F705
:10E300003196D801ED93FC9388818F5F8883E1CFAC
:10E31000DF91CF911F910F9108950F931F93CF938A
:10E32000DF9300D0CDB7DEB79C012F5F3F4F3B831B
:10E330002A832FE2FC01208381E0898310E00BE136
:10E340008091BB06181770F4019FC0011124AE0123
:10E350004F5F5F4FBE016E5F7F4F8454994FAEDFBA
:10E360001F5FEECF89818B3570F4AE014F5F5F4F39
:10E37000BE016E5F7F4F8DE796E0A0DF8A819B81B3
:10E3800001979B838A83EA81FB8110820F900F9013
:10E390000F90DF91CF911F910F91089580915008B8
:10E3A00082FF1FC089E590E30E94DF896091070624
:10E3B000709108068091090690910A064AE050E0A3
:10E3C0000E94568D8FE20E94548C60910B067091D2
:10E3D0000C0680910D0690910E064AE050E00C94D8
:10E3E000618D88E490E30C94DF89EF92FF920F93A4
:10E3F0001F93CF93DF938C01FC0101900020E9F77C
:10E400003197EF01C81BD90B10927D066EE470E0C6
:10E410000F9498357C01009729F4FE013197E00FA5
:10E42000F11F0EC060E270E00F9498358C010F5F11
:10E430001F4F6AE270E0C7010F949835FC013197D5
:10E440008DE081838AE082831382B8018DE796E0B4
:10E450000E94188480917D06882361F00E94F089D3
:10E4600081E390E3DF91CF911F910F91FF90EF90A7
:10E470000C94DF89DF91CF911F910F91FF90EF9066
:10E4800008958DE796E00E943E7F8DE796E00E941A
:10E49000897F809150088D7F8E7F809350081092E5
:10E4A0000706109208061092090610920A0681E0EB
:10E4B0008093160B08950F931F93CF93DF93CDB7DF
:10E4C000DEB76B970FB6F894DEBF0FBECDBF8B01E2
:10E4D00022E020930606909303068093020640E014
:10E4E00050E0BA018AEC97E00E94A87E8BE1EAEC4A
:10E4F000F7E0DE01119601900D928A95E1F7A801EF
:10E50000BE016F5F7F4F80E090E0A6DCCE010196F8
:10E510005FDC6B960FB6F894DEBF0FBECDBFDF9108
:10E52000CF911F910F910895CF93DF93CDB7DEB7B1
:10E530006B970FB6F894DEBF0FBECDBF81E080931E
:10E540000606109205061092040640E050E0BA015B
:10E550008AEC97E00E94A87E8BE1EAECF7E0DE010E
:10E56000119601900D928A95E1F740E050E0BE01CE
:10E570006F5F7F4F80E090E06FDCCE01019628DC7A
:10E5800080910406909105066B960FB6F894DEBF55
:10E590000FBECDBFDF91CF9108952F923F924F9242
:10E5A0005F926F927F928F929F92AF92BF92CF9223
:10E5B000DF92EF92FF920F931F93CF93DF93CDB72C
:10E5C000DEB76C970FB6F894DEBF0FBECDBF5C010F
:10E5D0004C8F2DB63EB619821C82FB0180819E01B4
:10E5E0002F5F3F4F49018F3239F08AEC97E0F501F8
:10E5F000918380838B0162C085EE97E0F501918362
:10E6000080838B010F5F1F4F0115110509F456C060
:10E610004DB65EB66FE270E0C8010F9498353C01CC
:10E620000817190708F04AC07C01E01AF10AFF2414
:10E63000C70101962DB73EB7281B390B0FB6F894CA
:10E640003EBF0FBE2DBF8DB79EB701966C01A701CF
:10E65000B8010F94B835F601EE0DFF1D10823C8D08
:10E66000332319F0C6010E94AB8CF50160817181E2
:10E6700021E0A601C4010E948581811113C0B60169
:10E6800084E190E30E94F3898EE20E94548C8AE038
:10E690000E94548C0FB6F8945EBE0FBE4DBE00E0D3
:10E6A00010E00CC0F5019182808283010F5F1F4F43
:10E6B0000FB6F8945EBE0FBE4DBEA6CFC40188DB78
:10E6C000C8010FB6F8943EBE0FBE2DBE6C960FB6B5
:10E6D000F894DEBF0FBECDBFDF91CF911F910F9198
:10E6E000FF90EF90DF90CF90BF90AF909F908F9072
:10E6F0007F906F905F904F903F902F9008950F9371
:10E700001F93CF93DF931F921F92CDB7DEB7209157
:10E71000500823FF27C0BC0140E0CE0101963DDF39
:10E720008C010097F9F0BC0189819A810E945F8277
:10E73000B801882381F083E890E30E94F3898AE09E
:10E740000E94548C10920706109208061092090637
:10E7500010920A0607C08BE690E30E94F3898EE2CE
:10E760000E94548C0F900F90DF91CF911F910F91C9
:10E770000895EF92FF920F931F93CF93DF9300D0F2
:10E78000CDB7DEB72091500823FF07C1F42EE62E47
:10E790008C010E944B5A882309F451C0FF2009F4D0
:10E7A0005BC080917C06882359F00E94F08983E445
:10E7B00091E30E94DF8980E090E00F94AE2AEDC0E3
:10E7C0008FE096E0AADDE0917C0684E0E89FF0010E
:10E7D0001124E858F94F8091070690910806A091FE
:10E7E0000906B0910A0680839183A283B3830E94B5
:10E7F000ED89B8018AE291E30E94F38980917C0659
:10E8000099E6899FB0011124615F794F8FE191E30F
:10E810000E94F3894091070650910806609109060D
:10E8200070910A0689E191E30E94548A8AE00E946D
:10E83000548C80917C068F5F80937C0625C0FF20DE
:10E8400039F00E94ED8989E091E30E94DF891CC0C4
:10E8500010927C0622E001C021E02B830E94ED890A
:10E8600084E091E30E94DF892B81213009F492C07A
:10E8700088EF90E30E94DF89B80180EF90E30E9467
:10E88000F3898AE00E94548C01DD40E0B801CE019A
:10E89000019683DE8C01009709F47FC069817A813B
:10E8A000EE2009F44BC021E0AC018DE796E00E9418
:10E8B0008581882309F43EC080918E0690918F0651
:10E8C000A0919006B091910680930B0690930C0650
:10E8D000A0930D06B0930E0610920706109208063C
:10E8E0001092090610920A06B80182EE90E30E9487
:10E8F000F38940910B0650910C0660910D067091C2
:10E900000E068AED90E30E94548A8AE00E94548C9D
:10E910008BEC90E30E94DF89B80180E090E0CBDDD2
:10E9200080910108811102C0C80102C081E098E015
:10E9300060E02DC0B80187EB90E30BC026E5AC0189
:10E940008DE796E00E94858181110CC0B80183EAB1
:10E9500090E30E94F3898EE20E94548C8AE00E9428
:10E96000548C1BC080915008816080935008B8017E
:10E9700080E090E0A0DD1092160BB80181E990E3F1
:10E980000E94F3898AE00E94548C60E0C8010E94D2
:10E99000706903C08EEF90E36DCF0F900F900F90D2
:10E9A000DF91CF911F910F91FF90EF9008952091EB
:10E9B000500822602093500840E060E0DACE0F93C8
:10E9C0001F93CF93DF93CDB7DEB76B970FB6F89455
:10E9D000DEBF0FBECDBF8C0119821C828091CD0796
:10E9E000811103C065EE77E002C06AEC77E021E0B8
:10E9F000A801CE0101960E9485818823F1F08BE168
:10EA0000FE013196AAECB7E001900D928A95E1F7EC
:10EA1000A091BB06AA30D8F481E08A0F8093BB0690
:10EA20008BE18A9FD0011124A454B94FEAECF7E09E
:10EA300001900D928A95E1F70AC00E94ED89B80114
:10EA40008EEF9FE20E94F3898AE00E94548CCE01EF
:10EA50000196BED96B960FB6F894DEBF0FBECDBF40
:10EA6000DF91CF911F910F9108958091BB0688236C
:10EA7000C9F081508093BB06882359F090E001973C
:10EA80002BE1289FF001299FF00D1124E454F94F48
:10EA900002C0E5EEF7E08BE1AAECB7E001900D9241
:10EAA0008A95E1F78091BB0608958BE1E5EEF7E0EA
:10EAB000AAECB7E001900D928A95E1F70895809154
:10EAC0005008877F809350088091E807882321F0C1
:10EAD00085EE97E00E94897F45E360E086EB96E053
:10EAE00013D8811105C00E94ED8984EC91E32AC0FE
:10EAF00041E066EB76E088E996E07DD481110DC0B7
:10EB000040E066EB76E088E996E075D4811105C0B7
:10EB10000E94F08980EB91E315C068E976E085EE0C
:10EB200097E0E5D6811105C00E94F0898FE991E355
:10EB300009C0809150088860809350080E94ED8938
:10EB400083E991E30E94DF89B0DF83E080931F02B5
:10EB50000895AF92BF92CF92DF92EF92FF921F93F0
:10EB6000CF93DF93CDB7DEB7A8970FB6F894DEBF8B
:10EB70000FBECDBF8091000887FD61C08091500815
:10EB800082FD5DC083FF9BDF8091500883FF54C0EE
:10EB900080910008082E000C990BC0969F938F93CC
:10EBA00088E290E39F938F936E0181E2C80ED11C9F
:10EBB000DF92CF920F94D23540E050E0BA0185EE5B
:10EBC00097E00E94A87E0F900F900F900F900F90EB
:10EBD0000F90FE0131967F0140E050E0B70185EED5
:10EBE00097E00E94F97D18163CF5F701019000208E
:10EBF000E9F731971E2F1E19115068F05701A10E29
:10EC0000B11C17FDBA94F501808190E00F94FE3499
:10EC1000F5018083F1CF8A858E37F1F245E050E02F
:10EC2000B601C7010F94AA35892BB1F6C601CEDA19
:10EC3000809100088F5F01C08FEF80930008A89635
:10EC40000FB6F894DEBF0FBECDBFDF91CF911F91FD
:10EC5000FF90EF90DF90CF90BF90AF90089510920B
:10EC6000000823CF61CC0E94DAD28DE796E00E94A3
:10EC7000897F80917C06882329F1815080937C06CE
:10EC800029E6829FC001112441E061E0815F994F34
:10EC900070DDE0917C0684E0E89FF0011124E858E3
:10ECA000F94F4081518162817381409307065093EF
:10ECB00008066093090670930A068DE796E00E94A5
:10ECC000A87EDCCAE3DA0E94B4D20F94BB270F946B
:10ECD00000286D3371058105910520F08AEF9FE2D0
:10ECE0000F946E1C1092E9050C949C6C1092E50731
:10ECF0001092E8071092CA071092CD0780E090E0CA
:10ED0000FC01E454F94F108213824B968E3021E0BF
:10ED10009207B1F789E18093B7061092BA06109274
:10ED2000AF0610927D06109280060895CF93DF9370
:10ED30008DE796E04DD8CAECD7E06B97CE0148D866
:10ED400086E0CC3BD807C9F78AEC97E041D885EE3E
:10ED500097E0DF91CF913CC8CF93809155088823ED
:10ED6000B9F14091580A5091590A60915A0A70912C
:10ED70005B0A28E538E080915608909157080E9478
:10ED80008F6EC82F811102C0C0E023C0409151088E
:10ED900050915208609153087091540841155105E3
:10EDA0006105710591F028E538E080915608909151
:10EDB00057080E948F6E882339F3109251081092E1
:10EDC000520810925308109254081092550801C02E
:10EDD000C1E08C2FCF910895CF92DF92EF92FF92F6
:10EDE000CF936B017C01C42F8091580A9091590AEE
:10EDF000A0915A0AB0915B0A8C159D05AE05BF051E
:10EE0000C9F0AADF811102C080E018C028E538E00F
:10EE1000B701A60180915608909157080E94476E4D
:10EE2000882391F3C092580AD092590AE0925A0A64
:10EE3000F0925B0A81E0C11180935508CF91FF9059
:10EE4000EF90DF90CF900895CF92DF92EF92FF92F4
:10EE50000F931F93CF93DF93FC0181859285A38548
:10EE6000B4850196A11DB11D84179507A607B707A4
:10EE700010F480E060C08789803149F4BB27A72F58
:10EE8000962F852FC388D488E588F6880FC08032F6
:10EE900081F783899489A589B6896A017B01C7E0D6
:10EEA000F694E794D794C794CA95D1F78C0D9D1D1D
:10EEB000AE1DBF1DE9016A017B018F014091580A17
:10EEC0005091590A60915A0A70915B0A841795070C
:10EED000A607B70731F040E0BC01CD017DDF8823F4
:10EEE00041F2F8018789803179F4B701A6015527ED
:10EEF00066277727440F551FFA01E85AF74F80819C
:10EF00009181A0E0B0E012C0B701A6014F7755276C
:10EF100066277727440F551F440F551FFA01E85AFB
:10EF2000F74F80819181A281B381BF7088839983DB
:10EF3000AA83BB8381E0DF91CF911F910F91FF9056
:10EF4000EF90DF90CF9008954F925F926F927F92F3
:10EF5000AF92BF92CF92DF92EF92FF920F931F93E7
:10EF6000CF93DF9300D01F92CDB7DEB78C014983DA
:10EF70005A836B837C835901C12CD12C7601412C9F
:10EF800082E0582E612C712C49815A816B817C81E1
:10EF90009E012F5F3F4FC80157DF882341F1D30106
:10EFA000C201F801058404C0880F991FAA1FBB1F66
:10EFB0000A94D2F7C80ED91EEA1EFB1E49815A8157
:10EFC0006B817C818789803139F481E0483F5F4FD4
:10EFD0006105710538F4D8CF81E0483F5F4F6F4F2E
:10EFE0007F4090F2F501C082D182E282F3820F90DD
:10EFF0000F900F900F90DF91CF911F910F91FF9085
:10F00000EF90DF90CF90BF90AF907F906F905F9028
:10F010004F9008954F925F926F927F928F929F923E
:10F02000AF92BF92CF92DF92EF92FF920F931F9316
:10F03000CF93DF93EC016A017B0128013901423053
:10F0400051056105710510F480E064C089859A85D9
:10F05000AB85BC850196A11DB11D84179507A60738
:10F06000B70790F38F89803149F48D2C9E2CAF2CFB
:10F07000BB248B899C89AD89BE890FC0803221F762
:10F080008B889C88AD88BE88DB01CA0157E0B695A5
:10F09000A795979587955A95D1F7880E991EAA1E20
:10F0A000BB1E41E0C501B40197DE882369F29F8948
:10F0B000903161F4DD24EE24FF249601220F331FEA
:10F0C000F901E85AF74F5182408211C0E894C7F81D
:10F0D000DD24EE24FF249601220F331F220F331F5D
:10F0E000F901E85AF74F40825182628273829A890D
:10F0F000923080F04D815E816F817885840E951EFF
:10F10000A61EB71E8092510890925208A0925308F2
:10F11000B0925408DF91CF911F910F91FF90EF9023
:10F12000DF90CF90BF90AF909F908F907F906F9027
:10F130005F904F9008952F923F924F925F926F92FF
:10F140007F928F929F92AF92BF92CF92DF92EF9277
:10F15000FF920F931F93CF93DF93CDB7DEB72F9717
:10F160000FB6F894DEBF0FBECDBF1C014D835E838A
:10F170006F8378873B872A87FC0181859285A385E9
:10F18000B4858C019D010F5F1F4F2F4F3F4F0C87A0
:10F190001D872E873F87AA85BB85CD90DD90ED909A
:10F1A000FC90C114D104E104F10431F0BFEFCB1A9B
:10F1B000DB0AEB0AFB0A10C0F101C080D180E280BB
:10F1C000F380F1E0F9870D811E812F8138850130B0
:10F1D00011052105310509F0198646015701412C19
:10F1E000512C3201F10181859285A385B4854816A1
:10F1F00059066A067B0608F04EC00C851D852E85D3
:10F200003F85081519052A053B0550F482E0882E34
:10F21000912CA12CB12C92E0C92ED12CE12CF12CF7
:10F220009E012F5F3F4FB501A401C1010DDE882370
:10F2300091F149815A816B817C81D501C40101968C
:10F24000A11DB11D452B462B472B19F06C017D01EB
:10F250000FC0AC01BD014C195D096E097F090D811C
:10F260001E812F813885401751076207730741F0CF
:10F270001FEF411A510A610A710A4C015D01B2CFB8
:10F280000FEF1FEF2FEF3FE0B501A401C101C2DE78
:10F290008D83811113C01D823DC02401350121E001
:10F2A000421A51086108710895018401B301A20155
:10F2B000C101B0DE882379F353014201C814D90497
:10F2C000EA04FB0450F3AA85BB854D915D916D91D5
:10F2D0007C914115510561057105A9F4EA85FB850D
:10F2E000C082D182E282F382F985FF2399F00FEF89
:10F2F000C01AD00AE00AF00AD101CD92DD92ED9257
:10F30000FC92139707C097018601C10183DE81112A
:10F31000E5CFC1CF8D812F960FB6F894DEBF0FBE1B
:10F32000CDBFDF91CF911F910F91FF90EF90DF90B4
:10F33000CF90BF90AF909F908F907F906F905F9095
:10F340004F903F902F900895AF92BF92CF92DF924F
:10F35000EF92FF920F931F93CF93DF9300D01F92F2
:10F36000CDB7DEB75C016A017B0182E090E0A0E0EE
:10F37000B0E0F50180839183A283B3839E012F5F68
:10F380003F4FB701A601C5015FDD882321F100E0F1
:10F3900010E09801B701A601C5013CDE8823D9F031
:10F3A000C980DA80EB80FC80F5018789803149F4DF
:10F3B00081E0F8EFCF16FFEFDF06E104F10460F41F
:10F3C000DDCF81E098EFC9169FEFD906E9069FE0EF
:10F3D000F90610F4D3CF80E00F900F900F900F90AC
:10F3E000DF91CF911F910F91FF90EF90DF90CF9021
:10F3F000BF90AF9008954F925F926F927F928F92DD
:10F400009F92AF92BF92FF920F931F93CF93DF9380
:10F41000EC01142F70935708609356081F8A82E0FE
:10F4200090E0A0E0B0E088839983AA83BB83109228
:10F4300055081092510810925208109253081092D9
:10F4400054088FEF9FEFDC018093580A9093590A7C
:10F45000A0935A0AB0935B0A442371F1453008F037
:10F46000E0C040E060E070E0CB01B6DC882309F446
:10F47000D8C020E1129FA0011124485B574FFA0128
:10F48000E254FE4F80818F7709F0CBC03C9680819B
:10F490009181A281B38184369105A105B10508F45B
:10F4A000C0C0349780809180A280B3808114910481
:10F4B000A104B10421F4B5C0812C912C540140E089
:10F4C000C501B40189DCF82E882309F4AAC0809113
:10F4D0006308909164088115924009F0A2C0909150
:10F4E0006808992309F49DC0209166083091670847
:10F4F000232B09F496C080916508882309F491C0F4
:10F500009A8B8C831D8690E061E070E02D85E22F60
:10F51000AB01022E02C0440F551F0A94E2F7841774
:10F52000950731F031E0320F3D87283078F379C00C
:10F5300020916E0830916F082115310519F040E0D7
:10F5400050E008C020917C0830917D0840917E08F1
:10F5500050917F082D833E834F83588780916608A2
:10F560009091670824013501480E591E611C711CD9
:10F570004B8A5C8A6D8A7E8A0091690810916A08BC
:10F58000198F088FA0916808B0E00F942431460EBF
:10F59000571E681E791E4A8E5B8E6C8E7D8E85E0AE
:10F5A000000F111F8A95E1F701501E4F012F1127FF
:10F5B0000695400E511E611C711C4E865F86688A3E
:10F5C000798A20916B0830916C082115310521F062
:10F5D000890120E030E008C0009178081091790896
:10F5E00020917A0830917B08B501A401441955098E
:10F5F00066097709400F511F621F731F04C076957B
:10F60000679557954795EA95D2F749875A876B874B
:10F610007C87453F8FE058076105710520F48CE039
:10F620008F8BF12C15C0453F5F4F6105710510F4BC
:10F6300080E10DC08091840890918508A091860892
:10F64000B09187088A8F9B8FAC8FBD8F80E28F8BA4
:10F650008F2DDF91CF911F910F91FF90BF90AF90B1
:10F660009F908F907F906F905F904F900895CF9371
:10F67000DF93EC019C012C5F3F4F41E050E060E0E4
:10F6800070E0898D9A8D57DD882399F04D895E89C8
:10F690006F89788D452B462B472B59F44C815D8122
:10F6A0006E817F814D8B5E8B6F8B788F9981906897
:10F6B0009983DF91CF910895CF92DF92EF92FF92DD
:10F6C0000F931F93CF93DF93DC0151964D915D9182
:10F6D0006D917C915497403E5F4F6F41710510F0E2
:10F6E00010E067C0EC01C3DF8823D1F335DB182FAE
:10F6F0008823B1F3E98DFA8D8C819D81AE81BF8124
:10F700000297A109B109058404C0880F991FAA1F97
:10F71000BB1F0A94D2F7C684D784E088F188C80E4C
:10F72000D91EEA1EFB1E81E080935508C092580A3C
:10F73000D092590AE0925A0AF0925B0A80E092E075
:10F74000E8E5F8E0DF019C011D9221503040E1F72F
:10F7500001E0E98DFA8D8481081798F428E538E0F6
:10F76000B701A601400F511D611D711D8091560802
:10F77000909157080E948F6E882309F4B1CF0F5FD4
:10F78000E8CF40E052E060E070E0058404C0440F40
:10F79000551F661F771F0A94D2F789899A89AB890A
:10F7A000BC89480F591F6A1F7B1F498B5A8B6B8B73
:10F7B0007C8B812FDF91CF911F910F91FF90EF9064
:10F7C000DF90CF900895CF93DF93EC0141E061117A
:10F7D00001C040E06C857D858E859F85FDDA88239C
:10F7E00041F0888920E2829FC0011124885A974FF6
:10F7F00002C080E090E0DF91CF910895FC0120E00D
:10F8000090E08EE23081303269F0283029F4DB015B
:10F81000A90FB11D8C939F5FDB01A90FB11D308132
:10F820003C939F5F2F5F31962B3061F7FB01E90F0F
:10F83000F11D10820895CF93DF93FC0123812111E4
:10F8400002C080E010C02250223028F48FE2FB0179
:10F850008083118207C0EB0160E0B5DF009789F378
:10F86000BE01CCDF81E0DF91CF9108952BE030E243
:10F870002150FB01E20FF11D30832111F9CFDC0192
:10F8800097E03A2FEB2F8D9181110AC0DA013C935A
:10F890001196EC9381E0FB019081903239F525C0FF
:10F8A0008F32A1F38E3229F49A30F9F028E09AE0F1
:10F8B000E8CFE0EFF1E33491332321F031963813B0
:10F8C000FACF13C0921788F0813278F08F3769F041
:10F8D00031E0320FFB01E20FF11D2FE9280F2A3131
:10F8E00008F480528083232FCCCF80E008950F93BB
:10F8F0001F93CF93DF93FC012381222311F080E03B
:10F9000043C08B01EC01FB018789803131F18032EA
:10F91000B1F783E08B83F801428D538D648D758D33
:10F920004D8B5E8B6F8B788F9E012F5E3F4FC80192
:10F930000BDB882321F31A8F098F81E089831886D6
:10F9400019861A861B861C821D821E821F82188AB7
:10F950001C861D861E861F8617C082E08B831D8A2B
:10F960001E8A1F8A188EFB01808D918DA0E0B0E069
:10F9700025E0880F991FAA1FBB1F2A95D1F7898BF5
:10F980009A8BAB8BBC8BD7CFDF91CF911F910F910F
:10F9900008952F923F924F925F926F927F928F9233
:10F9A0009F92AF92BF92CF92DF92EF92FF920F930E
:10F9B0001F93CF93DF9300D01F92CDB7DEB79C8308
:10F9C0008B834B015A01DC0113968C91811103C08A
:10F9D0008FEF9FEFE1C0EB81FC81818180FFF8CF49
:10F9E000EB81FC8181899289A389B4894085518505
:10F9F00062857385841B950BA60BB70BA50160E090
:10FA000070E084179507A607B70708F45C01750135
:10FA10008B819C8104969A838983612C92E0792E54
:10FA2000E114F10409F48AC0AB81BC8118964D91B0
:10FA30005D916D917C911B976A01B1E0DB22EB81B6
:10FA4000FC8123811A012B0189E056944794379455
:10FA500027948A95D1F7818D928D223061F4FC0133
:10FA6000828D938DA48DB58DBC01CD01620D731D6A
:10FA7000841D951D49C0DC0114961C911150122162
:10FA8000C114D104F9F411111DC0452B462B472B8D
:10FA900059F4EB81FC8185899689A789B08D84838F
:10FAA0009583A683B7830EC0AB81BC8114964D911C
:10FAB0005D916D917C91179729813A81C5D98823F1
:10FAC00009F486CFEB81FC81218D328D8481958173
:10FAD000A681B7810297A109B109F901058404C083
:10FAE000880F991FAA1FBB1F0A94D2F74685578516
:10FAF00060897189840F951FA61FB71FBC01CD01B6
:10FB0000610F711D811D911D93012C193D09870104
:10FB10002E153F0508F489010115F2E01F0779F55C
:10FB20002091580A3091590A40915A0A50915B0A23
:10FB3000621773078407950719F421C0C5012CC00B
:10FB40009401AB01BC0180915608909157080E9426
:10FB5000476E882309F43CCF800E911EEB81FC8117
:10FB600080859185A285B385800F911FA11DB11D50
:10FB700080879187A287B387E01AF10A51CF40E0CE
:10FB80002BD9882309F424CFB601685A774FA801EE
:10FB9000C4010F947135E0CF0F900F900F900F902C
:10FBA000DF91CF911F910F91FF90EF90DF90CF9059
:10FBB000BF90AF909F908F907F906F905F904F908D
:10FBC0003F902F900895CF93DF931F92CDB7DEB76C
:10FBD00041E050E0BE016F5F7F4FDBDE019719F41B
:10FBE000898190E002C08FEF9FEF0F90DF91CF915E
:10FBF0000895DF92EF92FF920F931F93CF93DF93BD
:10FC0000FC012381223060F0008511852285338537
:10FC10000F71112722273327012B022B032B11F001
:10FC20008FEF5DC04115510511F0FA0110827A0184
:10FC3000EB018C018DE0D82E40E250E0BE01C801FE
:10FC4000A8DE8032910539F021E0892B09F420E00B
:10FC5000822F819544C028812223C9F1253E11F0CD
:10FC60002E3231F4E114F10439F3F7011082E4CFBC
:10FC7000E114F10441F13B853F733F3021F54A8D9A
:10FC80005B8D452B01F52F713FEF320F3530D8F4E6
:10FC900030E021503109D29EC001D39E900D112435
:10FCA000D701A80FB91FFE0120E0AD01253088F46F
:10FCB00031813D932F5F32962D30C1F7288126FF89
:10FCC00002C0FA0115862B8523FDB6CF08C080E05F
:10FCD00006C02B3010F43481ECCF3681EACFDF91AF
:10FCE000CF911F910F91FF90EF90DF9008951F9398
:10FCF000CF93DF93FC012381223018F480E090E061
:10FD000023C0EC01408551856285738585E0769539
:10FD10006795579547958A95D1F7142F1F70CF0196
:10FD200052DF97FDEBCF88859985AA85BB854F96D5
:10FD3000A11DB11D88879987AA87BB87F0E21F9F05
:10FD4000C0011124885A974FDF91CF911F910895D8
:10FD50008F929F92AF92BF92CF92DF92EF92FF92DB
:10FD60000F931F93CF93DF93EC018B81811102C01E
:10FD700080E077C009891A892B893C890417150707
:10FD800026073707A8F36A017B01823029F4C88669
:10FD9000D986EA86FB860DC0C114D104E104F104C2
:10FDA00051F4188619861A861B861C821D821E82B3
:10FDB0001F8281E056C088849984AA84BB84E98D1F
:10FDC000FA8D258530E0275F3F4FB501A4014150F2
:10FDD000510961097109022E04C0769567955795FE
:10FDE00047950A94D2F7D701C6010197A109B10935
:10FDF00004C0B695A795979587952A95D2F784174D
:10FE00009507A607B70720F089288A288B2849F488
:10FE10004D895E896F89788D4C835D836E837F8386
:10FE200004C0841B950BA60BB70B4C015D018E0122
:10FE30000C5F1F4F81149104A104B10409F4A7CFF2
:10FE40004C815D816E817F819801898D9A8D0E94A0
:10FE5000247791E0891A9108A108B1088111EACFAD
:10FE600087CFDF91CF911F910F91FF90EF90DF909F
:10FE7000CF90BF90AF909F908F9008950F931F9356
:10FE8000CF93DF93EC018B818823D9F1898187FFA0
:10FE900032C061E0CE0197DC8C01009791F1FC014A
:10FEA0008081853E71F18B81823040F489899A8905
:10FEB000AB89BC89848F958FA68FB78F8D899E89DA
:10FEC000AF89B88DF801938F828FB58BA48BE091A9
:10FED0005C0AF0915D0A309759F0B8016A5E7F4F75
:10FEE000C80148961995F801808D918D938B828B6E
:10FEF00089818F778983DF91CF911F910F910C9426
:10FF0000AC7681E0888380E0DF91CF911F910F91E3
:10FF10000895CF93DF93EC01B1DF1B82DF91CF9186
:10FF200008954F925F926F927F928F929F92AF92BD
:10FF3000BF92EF92FF920F931F93CF93DF9300D066
:10FF40001F92CDB7DEB7FC0183818130E1F481815E
:10FF500081FF19C081899289A389B4898417950783
:10FF6000A607B70780F0892B8A2B8B2B09F474C066
:10FF70004A015B017F014084518462847384CF0114
:10FF8000E7DE811102C080E068C0F701818D928DAB
:10FF900081149104A104B10469F4458956896789E3
:10FFA000708DD2D9882379F3F701158A168A178ABA
:10FFB000108E39C0F70144815581668177819E0199
:10FFC0002F5F3F4F0E9424778823E9F249815A81AD
:10FFD0006B817C81F701818D928DFC012789203115
:10FFE00039F4483FFFEF5F0761057105E0F407C092
:10FFF000483F2FEF520762072FE07207A0F4A4D901
:020000021000EC
:10000000882309F4C0CFF701448155816681778147
:100010000FEF1FEF2FEF3FE0818D928D0E940A7846
:10002000882309F4B0CFF701818A928AA38AB48A1F
:10003000818180688183C70121DF882309F4A3CFF0
:10004000B501A401481459046A047B0410F4B301F7
:10005000A201C7017DDE01C081E00F900F900F90DB
:100060000F90DF91CF911F910F91FF90EF90BF9074
:10007000AF909F908F907F906F905F904F9008957A
:100080001F93CF93DF93EC01142F80E2689FF00160
:1000900011249F01285A374FD9011B968C918171E9
:1000A00021F0842F827109F057C08091580A9091F5
:1000B000590AA0915A0AB0915B0A8C879D87AE8736
:1000C000BF87688BE85AF74F4489558960E070E034
:1000D000BA01552744274D8B5E8B6F8B788F828DAD
:1000E000938DA0E0B0E0482B592B6A2B7B2B4D8BD6
:1000F0005E8B6F8B788FD9011B968C91887151F430
:10010000848D958DA68DB78D898B9A8BAB8BBC8B8F
:1001100081E00CC0803101F59E012F5E3F4F898D3B
:100120009A8D0E94A4778823B9F084E08B83812F75
:100130008F7089831C821D821E821F8218861986F9
:100140001A861B8614FF0BC040E050E0BA01CE01B6
:10015000E8DE811104C00FC01B8280E00CC015FFD7
:1001600009C049895A896B897C89CE01DF91CF9179
:100170001F91EECD81E0DF91CF911F910895BF9245
:10018000CF92DF92EF92FF920F931F93CF93DF9363
:100190008C01EB016A01E22E898D9A8DF801928F14
:1001A000818F40E050E0BA01CE01D2DDF12C88858C
:1001B0009985AA85BB8549895A896B897C89841769
:1001C0009507A607B707C0F525E0B695A7959795BB
:1001D00087952A95D1F7F82FFF70BF2ECE0187DDC6
:1001E000DC01892B09F486C08C91882319F0853EA7
:1001F000B9F47DC0F1100EC04091580A5091590ACF
:1002000060915A0A70915B0AF801448755876687A6
:100210007787B08A8C91882369F0FF24F394C7CF45
:100220004BE050E0BD01C6010F946435892B09F005
:10023000BECF5AC0FF24F3948E2D8274823409F00D
:1002400059C0FF2049F0F801B08861E0C801BBDA6D
:10025000EC01892B69F44EC08B81823009F44AC0CD
:10026000CE012ADA882309F445C0C8E5D8E0B12CCC
:1002700080E2FE0111928A95E9F78BE0F601DE013A
:1002800001900D928A95E1F7E0915C0AF0915D0A88
:10029000309739F0BE01625F7F4FCE0140961995CD
:1002A00008C081E298E2998B888B80E098E09F8774
:1002B0008E87888999899B8B8A8B998F888F8E8569
:1002C0009F859F8B8E8B0E94AC76882399F04E2D54
:1002D0006B2DC801DF91CF911F910F91FF90EF908F
:1002E000DF90CF90BF90CCCEE7FEF1CF03C0F110EE
:1002F00094CF82CF80E0DF91CF911F910F91FF903B
:10030000EF90DF90CF90BF9008953F924F925F9211
:100310006F927F928F929F92AF92BF92CF92DF9215
:10032000EF92FF920F931F93CF93DF93CDB7DEB77A
:10033000C354D1090FB6F894DEBF0FBECDBF5C0128
:100340006B0124965FAF4EAF2497522E1C8E1F8EEA
:1003500019821C826115710511F410E074C0FC0152
:1003600083818111FACF2496EEADFFAD2497808171
:100370008F32F1F4F60183818250823058F0618D22
:10038000728DCE010196B3DA882339F38E010F5FA7
:100390001F4F01C086012496EEADFFAD24978081EA
:1003A0008F3239F431962496FFAFEEAF2497F3CF16
:1003B0008B017E01FCE1EF0EF11C3701CE010196AD
:1003C0004C014E2C3F2CAE014E5B5F4FBE01695C71
:1003D0007F4F24968EAD9FAD249748DA882309F489
:1003E000BCCF2496EEADFFAD249780818F3231F4DF
:1003F00031962496FFAFEEAF2497F3CF8823D9F040
:1004000021E0AE01495C5F4FB801C701B8DE882327
:1004100009F4A3CF0C151D0511F0C8017ADDE6140F
:10042000F70431F0942D832D8701E92EF82ECBCFE0
:10043000982D892DF9CF252DAE01495C5F4FB8016C
:10044000C5019DDE182FCE0101960E94E86ECE01F7
:100450004C960E94E86E812FCD5BDF4F0FB6F8946B
:10046000DEBF0FBECDBFDF91CF911F910F91FF90E7
:10047000EF90DF90CF90BF90AF909F908F907F9044
:100480006F905F904F903F900895CF93DF93EC0172
:1004900040E050E0BA0145DD882369F061E0CE011B
:1004A00092D9009741F025EEFC0120831B82DF9159
:1004B000CF910C94AC7680E0DF91CF9108951F939B
:1004C000CF93DF93CDB7DEB76B970FB6F894DEBF4F
:1004D0000FBECDBFAB0119821C8222E0BC01CE0150
:1004E000019613DF182F882321F0CE010196CDDF6E
:1004F000182FCE0101960E94E86E812F6B960FB6E1
:10050000F894DEBF0FBECDBFDF91CF911F9108954C
:100510002F923F924F925F926F927F928F929F9213
:10052000AF92BF92CF92DF92EF92FF920F931F9301
:10053000CF93DF9300D01F92CDB7DEB78C014B0174
:100540003A01DC0113968C9113978130C1F4119616
:100550008C9181FF14C082FF18C0F8014189528933
:100560006389748980859185A285B38584179507F1
:10057000A607B70751F0C801EBDB811106C081E087
:10058000D8018C938FEF9FEF3CC1530184C0D801F9
:1005900059968D919C915A97FC0154805A946A0106
:1005A0007B0129E0F694E794D794C7942A95D1F774
:1005B0005C207A01F1E0FF22552009F478C080E048
:1005C00092E08E199F0965018A159B0508F46C015C
:1005D000D80159962D913C915A9714968D919D91E1
:1005E0000D90BC91A02D0297A109B109F9010584D4
:1005F00004C0880F991FAA1FBB1F0A94D2F7468513
:10060000578560897189840F951FA61FB71F9C01AC
:10061000AD01250D311D411D511D19012A01C114C6
:1006200032E0D30609F08AC08091580A9091590AA5
:10063000A0915A0AB0915B0A82159305A405B505ED
:1006400069F4109255088FEF9FEFDC018093580AF0
:100650009093590AA0935A0AB0935B0A9401B2018D
:10066000A10180915608909157080E948F6E8823AF
:1006700009F485CFF80180859185A285B3858C0D1D
:100680009D1DA11DB11D80879187A287B3878C0C0A
:100690009D1CAC18BD08D80118964D915D916D91C7
:1006A0007C911B97A114B10409F071CF7DC0E114B6
:1006B000F10409F084CF14964D915D916D917C9178
:1006C0001797411551056105710559F455968D919E
:1006D0009D910D90BC91A02D0097A105B10541F50C
:1006E00021C09E012F5F3F4F0E942477882309F489
:1006F00046CF89819A81AB81BC81F801218D328DF1
:10070000F9012789203139F4883FFFEF9F07A105C0
:10071000B10540F40DC0883F2FEF9207A2072FE0EC
:10072000B20730F0C8010E94377B811148CF27CF34
:10073000F80184839583A683B78341CFE114F10444
:1007400019F5D80118964D915D916D917C911B978B
:1007500051968D919D910D90BC91A02D48175907F0
:100760006A077B0788F00E94AC76882309F407CFDC
:1007700081E0809355082092580A3092590A40929D
:100780005A0A50925B0A08C041E0C201B1010E94BE
:10079000EC76882309F4F3CEA601B401C701885A88
:1007A000974F0F94713566CF5196CD90DD90ED90B7
:1007B000FC90549711968C91C416D506E606F70660
:1007C00040F4F801418B528B638B748B806881837A
:1007D0000DC020915C0A30915D0A232B39F0611421
:1007E000710421F08068D80111968C93F801818101
:1007F00083FD02C0C30105C0C80140DB8111FACFEF
:10080000BECE0F900F900F900F90DF91CF911F9160
:100810000F91FF90EF90DF90CF90BF90AF909F909F
:100820008F907F906F905F904F903F902F900895A2
:10083000FB0101900020E9F73197AF01461B570BF0
:1008400067CECF93C82F0E9407A7CC2351F02498DE
:100850002C9A65E070E080E090E00E94E02A149A13
:1008600003C0249A2C981498CF91089580E0E9CF82
:10087000CF92DF92EF92FF926B017C0183E3C81667
:10088000D104E104F10470F082E3C81AD108E10850
:10089000F10862E370E080E090E00E94E02A0E94AC
:1008A000A69AECCFC701B6010E94E02AFF90EF9014
:1008B000DF90CF900C94A69ADC01FB01460F571FE6
:1008C000E417F507C1F081912D913C9111973827DC
:1008D00098E0B901660F771F37FF06C09B0181E2E0
:1008E000282780E1382701C09B01915091F711968C
:1008F0003C932E93E5CF0895282F843640F064E68C
:100900000F9496306AE00F949630905D01C090E2AB
:100910009093620A2A3048F03AE0822F632F0F94B6
:1009200096300F949630905D01C090E29093630AE8
:10093000822F6AE00F949630905D9093640A82E66D
:100940009AE008959C0197FD0EC08436910584F0CD
:1009500064E670E00F94B630CB016AE070E00F946B
:10096000B630805D06C03195219531098DE201C018
:1009700080E28093620A2A30310564F0EAE0F0E018
:10098000C901BF010F94B630CB01BF010F94B6303F
:10099000805D01C080E28093630AC9016AE070E073
:1009A0000F94B630805D8093640A82E69AE00895E1
:1009B000AC01952F991F9927991F29F022273327DA
:1009C000241B350B01C09A01483E5340ACF0C901CD
:1009D00068EE73E00F94B630CB01EAE0F0E0BF01BF
:1009E0000F94B630805D8093610AC90164E670E0BF
:1009F0000F94B630CB0112C0243631050CF19111A1
:100A000002C080E201C08DE28093610AC90164E600
:100A100070E00F94B630CB01EAE0F0E0BF010F9434
:100A2000B630805D8093620AC901BF010F94B63071
:100A3000CB01BF010F94B630805D8093630A16C06E
:100A400080E28093610A8093620A2A3031053CF08B
:100A500091118DE28093620AEAE0F0E0E5CF911116
:100A600002C080E201C08DE28093630AC9016AE09E
:100A700070E00F94B630805D8093640A81E69AE05E
:100A800008958F929F92AF92BF92CF92DF92EF9292
:100A9000FF92CF93FC01C080D180E280F38020E000
:100AA00030E04AE754E4C701B6010F94BD2F4B0173
:100AB0005C0120E030E0A901C701B6010F947F2D51
:100AC00087FD05C020E030E040EA50E404C020E0AB
:100AD00030E040EA50ECC501B4010F94A62C20E0B0
:100AE00030E040E251E40F94862D0F94EE2D6B011F
:100AF0007C0197FD10C020E137E240E050E00F9408
:100B0000EB30CA01B9012AE030E040E050E00F9438
:100B1000EB30605D09C0F094E094D094C094C11CA7
:100B2000D11CE11CF11C6DE260935F0AC701B601A4
:100B300028EE33E040E050E00F94EB308AE0882E5E
:100B4000912CA12CB12CCA01B901A50194010F94DB
:100B5000EB30605D6093600AC701B60124E630E0C7
:100B600040E050E00F94EB30CA01B901A5019401B7
:100B70000F94EB30605D6093610A8EE28093620AAD
:100B8000C701B601A50194010F94EB30C62FCA012D
:100B9000B901A50194010F94EB30605D6093630A85
:100BA000C05DC093640A8FE59AE0CF91FF90EF900B
:100BB000DF90CF90BF90AF909F908F9008958F92CD
:100BC0009F92AF92BF92CF92DF92EF92FF92FC0181
:100BD000C080D180E280F38020E030E048EC52E435
:100BE000C701B6010F94BD2F4B015C0120E030E03E
:100BF000A901C701B6010F947F2D87FD05C020E034
:100C000030E040EA50E404C020E030E040EA50EC3C
:100C1000C501B4010F94A62C20E030E040E251E47D
:100C20000F94862D0F94EE2D9B0177FF06C022278F
:100C30003327261B370B8DE201C08BE280935F0ABE
:100C4000C90168EE73E00F94B630CB01EAE0F0E042
:100C5000BF010F94B630805D8093600AC90164E6DD
:100C600070E00F94B630CB01BF010F94B630805DB9
:100C70008093610AC901BF010F94B630282FCB01C0
:100C8000BF010F94B630805D8093620A8EE280933C
:100C9000630A205D2093640A8FE59AE0FF90EF904D
:100CA000DF90CF90BF90AF909F908F9008958F92DC
:100CB0009F92AF92BF92CF92DF92EF92FF92CF932B
:100CC000C62FFC01C080D180E280F38020E030E4B8
:100CD0004CE156E4C701B6010F94BD2F4B015C01F6
:100CE00020E030E0A901C701B6010F947F2D87FDF8
:100CF00005C020E030E040EA50E404C020E030E0ED
:100D000040EA50ECC501B4010F94A62C20E030E07D
:100D100040E251E40F94862D0F94EE2D6B017C017F
:100D2000611571058105910561F097FF0CC0F09484
:100D3000E094D094C094C11CD11CE11CF11C6DE264
:100D400003C060E201C06C2F60935F0AC701B60167
:100D500028EE33E040E050E00F94EB308AE0882E3C
:100D6000912CA12CB12CCA01B901A50194010F94B9
:100D7000EB30605D6093600A8EE28093610AC70188
:100D8000B60124E630E040E050E00F94EB30CA01B9
:100D9000B901A50194010F94EB30605D6093620A84
:100DA000C701B601A50194010F94EB30C62FCA010B
:100DB000B901A50194010F94EB30605D6093630A63
:100DC000C05DC093640A8FE59AE0CF91FF90EF90E9
:100DD000DF90CF90BF90AF909F908F9008958F92AB
:100DE0009F92AF92BF92CF92DF92EF92FF92FC015F
:100DF000C080D180E280F38020E030E0A901C7010B
:100E0000B6010F947F2D87FF08C0C701B601905827
:100E100020E030E040E251E406C020E030E040E273
:100E200051E4C701B6010F94BD2F20E030E040EA45
:100E300050E40F94A62C20E030E040E251E40F94FF
:100E4000862D0F94EE2D6B017C016031F7E27F0758
:100E50008105910584F020E137E240E050E00F94F5
:100E6000EB30CA01B9012AE030E040E050E00F94D5
:100E7000EB30605D01C060E26093600A88EEC816E6
:100E800083E0D806E104F10494F0C701B60128EE2E
:100E900033E040E050E00F94EB30CA01B9012AE0A2
:100EA00030E040E050E00F94EB30605D01C060E264
:100EB0006093610AE4E6CE16D104E104F10494F0F3
:100EC000C701B60124E630E040E050E00F94EB307B
:100ED000CA01B9012AE030E040E050E00F94EB3065
:100EE000605D01C060E26093620AFAE0CF16D1044F
:100EF000E104F1049CF08AE0882E912CA12CB12C05
:100F0000C701B601A50194010F94EB30CA01B901E4
:100F1000A50194010F94EB30605D01C060E2609325
:100F2000630AC701B6012AE030E040E050E00F94C8
:100F3000EB30605D6093640A80E69AE0FF90EF908A
:100F4000DF90CF90BF90AF909F908F9008958F9239
:100F50009F92AF92BF92CF92DF92EF92FF92CF9388
:100F6000FC01C080D180E280F38020E030E04AE7DD
:100F700054E4C701B6010F94BD2F4B015C0120E082
:100F800030E0A901C701B6010F947F2D87FD05C090
:100F900020E030E040EA50E404C020E030E040EAE5
:100FA00050ECC501B4010F94A62C20E030E040E2E3
:100FB00051E40F94862D0F94EE2D6B017C0197FF69
:100FC0000AC0F094E094D094C094C11CD11CE11CE0
:100FD000F11C8DE201C08BE280935E0AC701B6016D
:100FE00020E137E240E050E00F94EB308AE0882EB9
:100FF000912CA12CB12CCA01B901A50194010F9427
:10100000EB30605D60935F0AC701B60128EE33E004
:1010100040E050E00F94EB30CA01B901A501940102
:101020000F94EB30605D6093600AC701B60124E65F
:1010300030E040E050E00F94EB30CA01B901A50167
:1010400094010F94EB30605D6093610A8EE28093AF
:10105000620AC701B601A50194010F94EB30C62FB7
:10106000CA01B901A50194010F94EB30605D609352
:10107000630AC05DC093640A8EE59AE0CF91FF9049
:10108000EF90DF90CF90BF90AF909F908F9008959A
:101090008F929F92AF92BF92CF92DF92EF92FF9288
:1010A000CF93FC01C080D180E280F38020E030E06B
:1010B000A901C701B6010F947F2D87FF08C0C701A2
:1010C000B601905820E030E04AE754E406C020E042
:1010D00030E04AE754E4C701B6010F94BD2F20E089
:1010E00030E040EA50E40F94A62C20E030E040E2EB
:1010F00051E40F94862D0F94EE2D6B017C01603A24
:10110000F6E87F07F1E08F07910584F020EA36E8E2
:1011100041E050E00F94EB30CA01B9012AE030E021
:1011200040E050E00F94EB30605D01C060E26093FE
:101130005E0A80E1C81687E2D806E104F10494F063
:10114000C701B60120E137E240E050E00F94EB30F8
:10115000CA01B9012AE030E040E050E00F94EB30E2
:10116000605D01C060E260935F0AE8EECE16E3E0E6
:10117000DE06E104F10494F0C701B60128EE33E085
:1011800040E050E00F94EB30CA01B9012AE030E0B2
:1011900040E050E00F94EB30605D01C060E260938E
:1011A000600AC701B60124E630E040E050E00F9449
:1011B000EB308AE0882E912CA12CB12CCA01B90108
:1011C000A50194010F94EB30605D6093610A8EE29B
:1011D0008093620AC701B601A50194010F94EB3018
:1011E000C62FCA01B901A50194010F94EB30605DCF
:1011F0006093630AC05DC093640A8EE59AE0CF9164
:10120000FF90EF90DF90CF90BF90AF909F908F9026
:1012100008958F929F92AF92BF92CF92DF92EF92FA
:10122000FF92FC01C080D180E280F38020E030E0BA
:101230004AE754E4C701B6010F94BD2F4B015C018E
:1012400020E030E0A901C701B6010F947F2D87FD92
:1012500005C020E030E040EA50E404C020E030E087
:1012600040EA50ECC501B4010F94A62C20E030E018
:1012700040E251E40F94862D0F94EE2D6B017C011A
:1012800097FF0AC0F094E094D094C094C11CD11C84
:10129000E11CF11C8DE201C080E280935E0AF0E166
:1012A000CF16F7E2DF06E104F10494F0C701B601BE
:1012B00020E137E240E050E00F94EB30CA01B90181
:1012C0002AE030E040E050E00F94EB30605D01C078
:1012D00060E260935F0A88EEC81683E0D806E104F6
:1012E000F10494F0C701B60128EE33E040E050E08D
:1012F0000F94EB30CA01B9012AE030E040E050E041
:101300000F94EB30605D01C060E26093600AC7013A
:10131000B60124E630E040E050E00F94EB308AE084
:10132000882E912CA12CB12CCA01B901A5019401E0
:101330000F94EB30605D6093610AC701B601A501AF
:1013400094010F94EB306B017C01672B682B692BA8
:1013500089F08EE28093620ACA01B901A501940165
:101360000F94EB30605D6093630A80E38C0D809393
:10137000640A1AC0CA01B901A50194010F94EB30A7
:10138000611571058105910539F02EE22093620AFD
:10139000605D6093630A05C080E28093630A809376
:1013A000620A80E28093640A8EE59AE0FF90EF90F3
:1013B000DF90CF90BF90AF909F908F900895CF9384
:1013C000DF93FC018491EF012196882319F06CD200
:1013D000FE01F8CFDF91CF91089587E092E3EFCF40
:1013E0008DE092E3ECCF0F931F93CF93DF931F9287
:1013F0001F92CDB7DEB769837A83E1DF6981062F5B
:101400007A81172FF80181918F01882311F04CD236
:10141000F9CF0F900F90DF91CF911F910F91089509
:10142000CF93DF93EB01CBDF6AE070E0CE01DF9179
:10143000CF912DC3CF92DF92EF92FF926A017B0191
:10144000BEDF4AE050E0C701B601FF90EF90DF90A9
:10145000CF900CC3CF92DF92EF92FF926A017B0193
:10146000AEDF42E050E0C701B601FF90EF90DF90A1
:10147000CF909AC3CF92DF92EF92FF926A017B01E5
:101480009EDF42E050E0C701B601FF90EF90DF9091
:10149000CF908AC3CF93DF93EB0191DF6AE070E0D6
:1014A000CE01DF91CF9108C3CF92DF92EF92FF92EE
:1014B0006A017B0184DF4AE050E0C701B601FF907A
:1014C000EF90DF90CF90F2C2811103C080E092E3F1
:1014D00002C084E092E373CFF7DF8AE0E5C10C94A9
:1014E000D16E81E0089581E008958F929F92AF922E
:1014F000BF92CF92DF92EF92FF920F931F93CF9301
:10150000DF931F921F92CDB7DEB76C0159018B019B
:101510007B01E40EF51E0E151F0561F1F6018080BA
:101520009180F80161918F016983C4016A830F94EE
:10153000D6386A81681779F0C4010F94DE38C40187
:101540000F94D6389981891731F047DF84E192E30F
:1015500036DF81E010C041E050E0BE016F5F7F4F99
:10156000C501AAD9F601408151814F5F5F4F518378
:101570004083D1CF80E00F900F90DF91CF911F91EA
:101580000F91FF90EF90DF90CF90BF90AF909F9022
:101590008F9008958F929F92AF92BF92CF92DF92D9
:1015A000EF92FF920F93CF93DF931F92CDB7DEB7E9
:1015B0005C016B017A014901F501808191810F94F1
:1015C000D6388983002311F0F601808341E050E092
:1015D000BE016F5F7F4FC4016FD9F501408151811A
:1015E0004F5F5F4F51834083FFEFCF1ADF0A81E0E7
:1015F000E81AF10809F780E00F90DF91CF910F9181
:10160000FF90EF90DF90CF90BF90AF909F908F9022
:10161000089598E288E10FB6F894A8958093600049
:101620000FBE9093600008951F920F920FB60F9215
:1016300011240BB60F920F931F932F933F934F9349
:101640005F936F937F938F939F93AF93BF93CF934A
:10165000DF93EF93FF9300918C0AD0918B0A11E0F6
:101660001D0F1F77C091C6009091670A492F092E60
:10167000000C550B660B770B4C30510508F046C03B
:10168000FA018827EF55FF4F8F4F0D940731CD3466
:1016900041F0CE34B9F481E005C0CA3330F0CD3426
:1016A00071F582E08093670A4AC0C03308F047C0F2
:1016B000C03209F444C0CD3211F541C0C13329F024
:1016C000C43329F0C032D9F43AC083E0EBCF88E0CC
:1016D000E9CFC03321F0C13391F486E0E3CF84E059
:1016E000E1CFC83361F485E0DDCFC23341F487E058
:1016F000D9CFC13321F489E0D5CFC03311F08BE0CD
:10170000D1CF8AE0CFCFCA30D1F417C0CA30B9F4F4
:101710008091160B882389F0973049F09A3059F060
:10172000953059F410926F021092141606C081E0A1
:101730008093170B02C00F94652A1092670A101746
:1017400031F0ED2FF0E0E557F54FC283D12FD09364
:101750008B0AFF91EF91DF91CF91BF91AF919F9154
:101760008F917F916F915F914F913F912F911F9139
:101770000F910F900BBE0F900FBE0F901F901895FA
:101780001F920F920FB60F9211240BB60F922F9348
:101790008F939F93EF93FF9380916A0A2091690A38
:1017A000281791F0E82FF0E0E759F54F92818F5F0D
:1017B0008F719093C60080936A0A9091C0009064E4
:1017C0009093C000281305C08091C1008F7D809345
:1017D000C100FF91EF919F918F912F910F900BBEC0
:1017E0000F900FBE0F901F9018959B01AC011092A7
:1017F000C000211581EE380741055105C1F08091E7
:10180000C00082608093C00060E079E08DE390E0EA
:101810000F94EB30CA01B901615071098109910936
:1018200022E030E040E050E00F94EB3002C020E1D5
:1018300030E03093C5002093C4008091C1008061E6
:101840008093C1008091C10088608093C100809125
:10185000C10080688093C1008091C1008F7D80931A
:10186000C1001092680A089580918B0A90918C0AA9
:10187000891759F0E92FF0E0E557F54F82819F5F16
:101880009F7790938C0A90E008958FEF9FEF0895D3
:10189000EBE8FAE0808181830895EBE8FAE080814B
:1018A0009181891B8F77089591E09093680A9091B8
:1018B000C10095FD04C09091C00095FD40C02091ED
:1018C000690A2F5F2F710FB607FC34C090916A0A26
:1018D000291322C09091C00095FF1DC090916A0A03
:1018E0004091690A491791F0E92FF0E0E759F54F67
:1018F00032819F5F9F713093C60090936A0A309146
:10190000C00030643093C000491305C09091C100FD
:101910009F7D9093C100DACFE091690AF0E0E7592A
:10192000F54F82832093690A8091C1008062809381
:10193000C100089590916A0A2913EECFFBCF8093DE
:10194000C6008091C00080648093C00008958DE03F
:10195000ABDF8AE0A9CFCF93DF93EC018991882395
:1019600011F0A2DFFBCFDF91CF91F1CF8F929F9249
:10197000AF92BF92EF92FF921F93CF93DF93CDB7B9
:10198000DEB7A0970FB6F894DEBF0FBECDBF6115CE
:1019900071058105910579F110E0842E912CA12C1F
:1019A000B12CEE24E394F12CEC0EFD1EE10EF11CA3
:1019B00017FDFA94A50194010F94C930F7016083D3
:1019C000B901CA011F5F611571058105910549F7CC
:1019D000115010F1E1E0F0E0EC0FFD1FE10FF11DFF
:1019E00017FDFA9580818A3010F097E301C090E3EB
:1019F000890F5ADFEDCF80E3A0960FB6F894DEBFD3
:101A00000FBECDBFDF91CF911F91FF90EF90BF90A0
:101A1000AF909F908F9048CFA0960FB6F894DEBFFE
:101A20000FBECDBFDF91CF911F91FF90EF90BF9080
:101A3000AF909F908F900895CF92DF92EF92FF9298
:101A40006B017C0197FF0AC08DE22EDFF094E094D9
:101A5000D094C094C11CD11CE11CF11C4AE0C70108
:101A6000B601FF90EF90DF90CF9080CF41155105E8
:101A700011F4862F19CF4A30510509F4DDCF76CF06
:101A8000AB01682F880F770B880B990BEFCFAB0159
:101A9000BC01990F880B990BE9CFAB01BC01990FE1
:101AA000880B990BE3DF53CFE1DF51CF411551058F
:101AB00011F4862FF9CE5ACFAB01BC0180E090E043
:101AC000F5CFF4DF44CF8F929F92AF92BF92CF9227
:101AD000DF92EF92FF92CF936B017C01B42E20E056
:101AE00030E0A9010F947F2D87FF06C08DE2DCDE78
:101AF000F7FAF094F7F8F094C0E060E070E080E06E
:101B00009FE3CB1541F02DEC3CEC4CEC5DE30F94E6
:101B1000BD2FCF5FF6CF9B01AC01C701B6010F947B
:101B2000A62C6B017C010F94F32D4B015C014AE064
:101B30001DDFCC2379F1C501B4010F941F2E9B0149
:101B4000AC01C701B6010F94A52C6B017C018EE29C
:101B5000ABDE20E030E040E251E4C701B6010F9473
:101B6000BD2F4B015C010F94EE2D6B01770FEE083A
:101B7000FF08C701B60160DFC701B6010F94212E2F
:101B80009B01AC01C501B4010F94A52C6B017C0134
:101B9000C150F9F6CF91FF90EF90DF90CF90BF90BA
:101BA000AF909F908F9008958ECF909164009B7F0F
:101BB00090936400982F906A96959CBD80FD03C019
:101BC00091E0863009F490E09DBD0895209A289A0E
:101BD000219A2398229A209A81E0E7CF8FEF8EBD39
:101BE0000DB407FEFDCF8EB5089561157105D9F0CE
:101BF000615071092FEF2EBDFC014FEF9F01281B93
:101C0000390B2617370738F40DB407FEFDCF2EB574
